:020000040000FA
:04000000D1EF75F0D7
:08000800056ED8CF06F0E0CF31
:1000100007F00001E9CF0DF0EACF08F0E1CF09F0D9
:10002000E2CF0AF0D9CF0BF0DACF0CF0F3CF14F017
:10003000F4CF15F0FACF16F000C00FF001C010F0A9
:1000400002C011F003C012F004C013F0F2AA2CEFAA
:1000500000F0F2B4CAEF3AF0A0A432EF00F0A1B47D
:10006000ECEF3CF00FC000F010C001F011C002F046
:1000700012C003F013C004F00E8E0DC0E9FF08C0DB
:10008000EAFF09C0E1FF0AC0E2FF0BC0D9FF0CC0C4
:10009000DAFF14C0F3FF15C0F4FF16C0FAFF0550D5
:1000A00007C0E0FF06C0D8FF1000F2CF0EF0F29EAE
:1000B000C20FF66E000EF7220900F5500EBEF28E4A
:1000C00012004000400065218521E731073284217C
:1000D0006419E629483A2C532C53EB428E53AE5BFD
:1000E0008E53CF5BCF5B306CCE5BB1741385CE5B30
:1000F0004D4B8F53AF53AF5BCF5BF063316C1164EB
:10010000326C30640F640F5CCE53CE533164CF5BDE
:10011000AF5B8D5B2B4B68322A4BE521C9424832DD
:10012000CA42EA42CA42EA4A683A893A48320A4B23
:100130000943AB536A4BC421A9424311683A272AA9
:100140006C4BCA3A0A432311A521473A0632A94209
:100150002311C629693A2832CA42693A0C4B717494
:100160004D4BCF5B91744F748C530D64748D2C4345
:100170000C434E4B8E534D4B6D53EF63D4846E53F3
:10018000F063EF63CE5B8D536C4B6D4BCF5B8E5347
:10019000106C4D532B4B272A883AE5290B53A52188
:1001A0004832A93ACA42A942683AEB4ACA422B4BA2
:1001B0006B536B4B2A4BE5218419E2086419893A89
:1001C0000B432722EA3A6419C6290732683AE6291E
:1001D000CA424832EF6B8A3AAA426D5B8D5B2E6C45
:1001E0008C53ED6393955295AF7CD07CEE63EB42DC
:1001F000EB3A2D4B4E534D53CB422C53AE5B0C4B35
:10020000AE5B50746C53CA3AEB422C436D536D5342
:100210006D53EB426D5BEA42E9424732072A283AC6
:100220002832483A0B53EA4A4C53EA4A683AEA42BF
:10023000ED63C83A2A4BC94264196419072A473248
:10024000472A68328511272A472A2B4B68324C4BA4
:10025000A93A2C4B0F6C893A4C53128D118D729523
:100260009295719571957195B29D939D338DAE5B0D
:100270006D532C4B6D530C4BEB4A6D53AE5B0C4BDB
:10028000AD53EF636D53EB42CB42AB3A2C4BCF5B9C
:100290002C4B2C4B0B4BCA3AEB42CA42AA42E731D9
:1002A000483A483AAA4AAA42CA42EA4AE629A93A38
:1002B000AC5BE5214E6C2B5323114419A5218832E8
:1002C000C942682A472AA93A682A0722683289322D
:1002D000282A4832CB42EB4ACE633295D084F08450
:1002E000308D7095B19D9195D29DB39DEE634D5328
:1002F000AE5B4F6C749D2F742B534B532F6CF28459
:100300006D532C4B4D53CB42AA3ACA42CB42CF63DA
:100310000C4BCB428A3AEB42893A4832683AC629BA
:100320008942693A07320732A942A83A6F74E94212
:10033000E8420522E93AA83AC5216419C62968327B
:10034000883206228832072AC621A6196932693204
:10035000693A0B4B8A3AEB4A2B4B8C5BAC5BD39DD7
:1003600071952F85B19DB19D919DF184CA426E53C7
:10037000CB420B4B939DD4A5B39D72951185907480
:10038000A93AEB420C4BCB424932AA3AAA3AEB4A81
:10039000CB422C53CA42EB42693A683AA942283A06
:1003A000483A483A894289420A4B4B5346324A53AB
:1003B000252AE842E9426B53273264196419472A17
:1003C000C51967324311483A2732C621CA42893AD1
:1003D000EB4ACA4249328A3A0B4B4E74729DB29D27
:1003E000CB5B2C64D39DD2A551954F74CA42EB4A86
:1003F000EB4ACA42AF84D2A5D2A5F2A57295A83A1B
:10040000C93ACA42CB42AA3A8A3AAA3ACB42CB422A
:10041000CB42EB4AEB4A893ACA422832493A08327F
:1004200089426942CA4A89420B53AC5B67324A4BE4
:10043000094BE9428B53262AE621E629E629A4192D
:10044000C521E621631167326732C73A8A532943CF
:100450002A4B2A4BAC5BAC5B4D6C4D74CE7CAE7CB6
:100460000843AB5B4E6C5195929DB3A532954E748B
:100470002B53CD63529DB2A550952C6CE8422B4B6B
:100480006932693AEB426932482A0B432C4B2C4BB8
:100490004C53CA42CA42893A693ACA4A6942E73168
:1004A000CA4ACA4AAA4A2732CA422A4B6B530A434B
:1004B0004B53A83A4A4BC100E629A629A621641944
:1004C00084198419A419262A87320C5C2C640C5CCC
:1004D000AF746E6CAF74CF7CCF7C508D2F85718DD7
:1004E000518D4F6CEA420E6C118D5195929DB3A5C2
:1004F00035B6D3A534B634B6939DC942EA4AEB4229
:100500008A3A493ACA3A6D53AA3A6D53AA3AAA3A74
:100510002C4BC942C942EA4AEA524C5B0732693A5B
:100520000B53CA4A6942A942272A0A4B0A4B883A06
:10053000883A272AE629C200031145190732E6291D
:1005400063194632E529272AEC5BEC5BF074518590
:100550006E6C11852D648F743185508D3085318D91
:10056000328DEA42CB42CA42CD63939DAF7C8E7CF2
:1005700014AE75BE75BEF3ADD084EA4AAA42AA3A5B
:1005800069326932EB424D536D534C53CB42693261
:100590006932EA42C9428942EA52EA4A0832EB52D7
:1005A000A9420B53483A0B53072AA93A2B53062A60
:1005B000CA42EA42A942AA42241144198521C52906
:1005C00064198419C521C93A8C532A43CC536F6CE2
:1005D000D0740E64AC538F74D07C518D528D939532
:1005E0008C5B2C5331748A3A8942B5A536B635B640
:1005F000B7C6B6BE54B60C6C2E74893AEA428A3A33
:10060000082AAA42282ACB428E5B0B4B8D5BCA423A
:10061000893AC93AA93AA94268420B53483A8942F1
:10062000483A6942A94ACA4ACA4A0B4BA9426C5B7A
:100630000B4B893A2C538942810003114419431909
:10064000231102094732E621EA3ACA3AEE632F64DF
:10065000AD538C538B4BCC5B6E74AF7C907C907C99
:100660000C53AB422E5BEC528B424D5B1395F6ADB7
:1006700036AED4A556B6CC630A4BEB4AEC4A0C4BCB
:10068000693A6A3A6932893AEB4A6C530B4BEB424E
:10069000A93AEA428832A83A883A8942483A273247
:1006A000483AEB52483AEB4A8942EB522732A621AC
:1006B00028326519CA4AA208E310E310641923110D
:1006C000021184212732E7210A432B4B2C4B2C4B60
:1006D0004C4B2B434B4B2C6C108D118DCF6B727C84
:1006E0003795989DD4843695117C938CF073117452
:1006F0006E5B5174EF63CE63CA429AC6AB42D7AD0C
:10070000EF63C721CA42EA426C5B6832893ACA3A4F
:10071000EB428932272A072A683AAA42C629EA4ABE
:100720000B5369428842A8420A530A53683A683216
:10073000272A282A0732C208A208241924192419B2
:10074000810085214419AA3AAE5B0B43AA3ACA3A02
:10075000EB42CA3A2B4B5195929DB49D8A42D58C5F
:100760003795948493841595F9B59ACEF9B5B48CE0
:10077000F173569D19B6B7ADF073359DAC4AB38C85
:100780008B424D5BEB4A8D5BCA42EB4A2832893A79
:10079000893A4832A621283A693A8942483A283AA1
:1007A000A9428942883A4B53E94AA84AEA4AC942CF
:1007B000272AC6214419C629441944212419241979
:1007C0000311C6290311072AEB42EA42893AAE5BBC
:1007D000AE5BEE63949534AE929D939D0C530E5395
:1007E000B8A5B9A59484D4849484B484F58C9484F5
:1007F0003274D48C369D569D779DB7A5B7A598A524
:1008000031748E634C534C532B53EA4A2B53072AB3
:100810006832272A2832493A283A483A283A283A68
:100820008942AA42E9422A53C94A4A53A83AA83AF5
:10083000883AA521E208E310E31065210311483A44
:1008400003112419C208272AAA3ACA420B4370741A
:10085000CD5B8C53528DEF84CE84D084AE636F5BBE
:10086000B47C7895F6841685D67CD67CF684D584BF
:100870007BB6168DF684F584F584F67CF684368D89
:100880006E538B426D632C530B4BEB4A4C53EA4235
:100890002B4B48328942AA4A0B536521A629E629E7
:1008A00028328942E94A4B534B53873AE942A83AE6
:1008B000062A683A43192319E631C629852165219C
:1008C0002419E310E210272A883289326C4BAD5389
:1008D0008C4B6F6C317DAE74519531952B530C4B15
:1008E000747C388DD784F784D684D684388DD684AA
:1008F000168DF684D684168D168D178DD684378D79
:10090000326C0D4B3174EB42CB42AA3A4832272A63
:10091000693A283228328A4ACB524521AA4AA9424A
:10092000893AEB4AA942893AEA4A8942EA4AC942E3
:10093000CA4AEA5264214421031164214419A208DD
:10094000C308E310E3100622882AA8324B436B4BFE
:100950002E5C2E5CF0742D64F084F18CCA422E5310
:10096000B67C999DB67C1785F784388D5895F684AA
:10097000B99D999DF68CF78C58953895D784389504
:10098000B58C2E53EC424D53CA428A3A4832483213
:10099000693A894208324942AA4A8629EB52CA4A30
:1009A0006942CB4A89420B4B2B534C53EB4AEA4AE0
:1009B000A942E6316421C210A1086842E21044193C
:1009C000E310E310E210882A2622672AE93A6B4BEB
:1009D0006B438C4BED5BD074F184EE63693A2E531C
:1009E000957CDAA5346CF363136C757C3895589557
:1009F000F68C747CD26BD26BD68C5895799DDAAD1F
:100A0000D6944F5BCC42106C082AA93A072A072AD1
:100A1000E729893A894249424842A629EB5269426C
:100A2000AA4ACB4A0B4BA942CA424832893AA5216D
:100A3000C62964192311A1080632C6298108A10814
:100A4000441944192319A9322B432B434B4B8C5384
:100A50000A3B4B430E5C0E644F74717CA7190E4B1E
:100A6000B05BF1637053B15B6F53B05BAC3AB16391
:100A70004E53B063D063D16BCD42ED42F263B15BB4
:100A80002F533274A72929320B4B893A2832483226
:100A9000693ACA4AAA4AE731283AA629AA4AEB5231
:100AA000CA4A2B530B4B2B53EA4A2732A9426519EA
:100AB000C20823196419C629A5298521A10844194A
:100AC0008100C2080319893AAD538D53EA42482A7E
:100AD000CA3A0B43CE5BEA4289420F6C282AF06B7C
:100AE0002D532D532A320D4BAB3ACB42EC42CB3A2D
:100AF0004D53B484D4845374326C11643585F163DE
:100B0000F163D06B2519C729AC63A5218621A521E6
:100B1000473A68426942AA4A69424942EB520B533A
:100B20000B4B0B4BEB4ACA42E729CA422832A52994
:100B300084210311A52944196419E2086108073AC0
:100B4000C208A6294521272AEA42A9320B43EA3ADC
:100B50000B438D53AD53CB42CB4A5495CE63082AF9
:100B60008A3A527C527CF9AD39AEF8A539AE59AE0D
:100B70007ABEBCC6BCC69BC67BBE9BBE1DC7BBBEE9
:100B800019A68F639BCEF8B5549DAD63E729483A0B
:100B9000EA52C94A493AAA4A283A8A42283AC62910
:100BA0002411AA42CA4AEB522832AA42CA4A8942AE
:100BB000E629C208C210C2086419A31926324732B6
:100BC00023110319A210E629EA42893A68328932D0
:100BD0004C4B4C4B89326D53B28CAE6330740F6406
:100BE000B6A559BEB7ADD7AD7BBE5AB63AB67BBE39
:100BF0005BBEBDC6DDC65ED71DD79ABE7AB63AAE1D
:100C000039AE1AAE7EE77CBE3ED7138D2832A9429C
:100C1000673A2E7C083A8942C731AA4A483AEB4AD9
:100C2000EB4AAA42893ACA4A4832EA4A4832A521DE
:100C3000C62964216421800001090522E8422A5363
:100C4000E20882088108C629693A893A48322C4B61
:100C50006832EA42AA3A6D5BEF731395AE63AE63F6
:100C6000CF6B769DF8ADD8ADB8A5D9A50F4B547C08
:100C7000D26B30530F4B905BB05B4F530E4B905B7E
:100C8000336C53743795747C1685F7A52A4B6B5BD0
:100C9000CC6BCC6B0A5369420732AA4AA629693A3F
:100CA000AA42693A8942483AE629072AC62185219B
:100CB0008108A52903114319E421E732694BE84271
:100CC00002112419C310C62968320A4B4832A93AC6
:100CD000272A473A2B53507C307CEF73AE6BF06B76
:100CE000CC526B42F68C2B326C3A8C3A2B328D42C2
:100CF000EA31E9292A324A322A2A0A2AC9218821D4
:100D0000C921092AC9292A32C408348DE83AEB5B83
:100D1000EB5B8A53CC5BE84A84218D63CA4AA942C3
:100D2000A942483AA94227322311A5192311431990
:100D300043190211A1080211E421A53227430843F7
:100D4000A42103112419873A4A4B6732883A262A8C
:100D5000473AA84A2B5B0F7C0F746521AF6B7284F6
:100D60000E5BA821EE52D16B9BBE938488212A3260
:100D7000C929C929C9290932882168196719461959
:100D800026190519B48C77A5E410C629662A6C6467
:100D9000894B694BEB5B8A53A421873AE94AA84205
:100DA0000A534A53494B8953284B694B4632C4294D
:100DB0008321A4296321C1088A5BE742C63AA53290
:100DC000873A0211641946326953294B4A53AC637E
:100DD0000D744E7C2F7CEF7BEF7B86292D5B8B4245
:100DE000E929C929CD4A369DBBC6569D2619A82991
:100DF000A8290A3290631374D26BD26BF1738F6B94
:100E0000E939E5189BCEF173093ACA4A0A4B0C64DA
:100E1000694B2843694BA953084B4532E842C74206
:100E2000C742E742084B6853895307436953AA6393
:100E30002C74AB6BCA6B6C7C064B464BC53A853247
:100E4000252A6000C108C319E63AEA5BCA5BAF7C99
:100E50008E7C0C74CC734F8C0F844942F073C41099
:100E6000A829A8298C420A3211748B422A3A6B4273
:100E70006B42A82946192619471906198829C51051
:100E80002619A8312A3A2A3AED52E410CA4A94A502
:100E9000118DAB63CE842B6C4C6C074BCA63AD7C5D
:100EA000CD844F95CC7C0D8DCC7C0D7DAC7C0E8D96
:100EB000AD84EF942B746C7C709D2E8DAC7C0F8573
:100EC0006D74CB630C6CA6322743273B894B484B90
:100ED000CA536C6C6D74ED6BAD73E8390C5B2519FE
:100EE00087210A3A4B42A8298B42093A46216721B9
:100EF0002621261987214719672167212621C93113
:100F0000A41087293284B06B4E5B8F63749DC5310A
:100F10002D7CEE948C7C0A6CA9630E8DCD84C96304
:100F2000AC842A74AB7C6A74C9638853E963E54274
:100F30006D7CCF8CCA636A5B6A5B294B69530B6C0F
:100F4000EA63AD7C2E8D284B684B684B0B5CC95314
:100F50000A5CA94B0A546D6CEC63CD6B8529293A68
:100F60008629ED5293844F5B6F63B06BD1734B4214
:100F700046216F63ED52672187218721E5108C4A56
:100F8000C8312519E831E931C8298521052AAE84FF
:100F9000E96BEC8CEC8CCC848B7C8B744A6CCC7CB9
:100FA0004A7409744A7C8B842F95CA63AD84AD84DE
:100FB0008A5B6E7C2F95EF8CCE84274BE95BEB63CD
:100FC0006E7C2853A963A53206336743473B884BA1
:100FD000E953C94BEA534B5C2B648E74873A473A0A
:100FE0000319041187212619461926196721261984
:100FF000872905196721E931E829A72966212621D2
:101000008308051905190519452123198A5BEF8CF9
:10101000CD84CC84AC7CEC840D85ED7CAC742A6CE6
:101020000E8D6C7CCD8CEC8C8D84EF8C6B7C096C84
:10103000E74A084B4B742B6CAC7CCC7C0C7D685322
:10104000AA63863AC6420733884388430A5C6B64C6
:101050008C642954AC648B5CAC6C2A644C6C495332
:10106000832124192519461946194619462187292D
:10107000C8316F637284117CF594D49436A53AC656
:10108000C83186296208A310A7396421A84A695B80
:10109000AA632C74895B0A6467534B6CA95BCA63AF
:1010A0002F958C7C2A740D8DEE8C719D4E950D8D37
:1010B000AD84AA636B74C95B8753CA7C2B85AB7CF8
:1010C0006B746C7C6C7C483B0A544B5C6C64E953DD
:1010D0002A542A5CCC648B5CAB640C758A6C0D7DE5
:1010E000E6428319651965196519251925192A42DA
:1010F000E9396F6B8F6B4E638F730E636B52AC5A13
:1011000086292521A310A310C739A631A84A295B37
:101110006A63663A095324320C748A5B0B6C0B6C5D
:101120002B74CE840F8D2B74CE8C8E840B74C9637C
:101130006D7C308DCD84ED7C4A6CEB7C8A744A6C7E
:101140006753885B0753694B2B54C94BA94BC94B59
:101150008B6C8B6CE853495C0D75AA640A75C96C7D
:101160008A6CEA5B0101631923110419E418E5187C
:10117000E418E418E518C4180521A3102521E41883
:10118000452945298210C318C639E3200B63E53988
:10119000053A874A6A63A74AC84ACC6BEC6BCB6BAB
:1011A000AA63CB638A63EC73495BAF84D08C1095E0
:1011B000AF7CCD6B6E746D740B6CAD7C6A6C6D8D99
:1011C000AA740D85CE8448438C646C64EA53A84BA2
:1011D000A84B063B674309548B640C75EB748A6C0F
:1011E000864BCC748B6C6D74A73AC208A310A31005
:1011F000A310E4182521252146294629C3180421D6
:101200006529C639A210C3188639E3200C6B8D738B
:101210002B636C6B4B636F844F84B08CAC6B085347
:1012200008536A5B4A5B6A632E7CD09473A56F7C1B
:101230004B5BAD6B2E742D74AF84108DEA63654BE0
:10124000AA6C49646A6C894BE953A843EA53C953B1
:10125000C853053BC853A74BE853295C8B6C874B9D
:101260002643263BE95367436C74052AC110A2103C
:101270008310A310252166318731C739E31844292B
:101280000321E739A210C318E320C318AA5A8952D0
:101290002B630A5B6C6B33A52B6333A532A5AF8C34
:1012A000319DAF8CAB6B8F84319DF19C2D7CED73A8
:1012B0002A53EA52CD73E94ACB6B0D744D7C4B6CCB
:1012C000AB74CB746964A5326743A84B87432A5C2F
:1012D0008B6CE8536A64E8534A642743674B0A649B
:1012E0006532652AA94BE9538C74AC7C8221C2100B
:1012F00004216629E739E741863165298531853141
:1013000024214429894A0F8414A513A57194B19C02
:10131000909412A574AD129DB0946F8C6F8C0D7C5F
:10132000CC73D094F094F09472A552A5AC738C6BEE
:101330008C6B4C6BA952063A2F7CED73CB6BEA6336
:10134000CE840B64A4328532684B894B842A2A648C
:101350002A64674B295C263BA9532A640A64E74246
:10136000AA5B6632494BE5324A64AB74AD7C221904
:10137000E53984296321E639852948424529A6397A
:10138000E741CA5A6C63EE73918C9194719433A5C2
:10139000919474AD32A5109D71A5B2AD14BE8F8C21
:1013A0002A63CC732F84CD730E7CEE7BAD7B0F84D0
:1013B0003084B29CEF83CF7B91940E7C6E84AE849C
:1013C0008F846A5BEC6BA742AA5BCA5BE63A474B29
:1013D000C95B642A474BA9532843CC74474BC74287
:1013E000242AC4210B644B64EC7C4964CC7C4B7490
:1013F000653AAA63E74A0632C5310B63CA5A8E7B47
:101400006D73AE7BAD73AD6BEE73B094D19C0E84F7
:10141000EE7B4F8CD0946D846C84CE8C0F9572A52E
:10142000B094ED7B6C6B8C6B2F842C6B2C6B0F84CE
:10143000B29C72945194318CD39C4C6B2E84EB7380
:101440001195539D6F84663A252AC742863A074B09
:101450000743EB63484B484BA63A26430643663A9C
:10146000042AA7426532874B664B8A6CEC7C096480
:10147000AC7C6B74CD84CB6B2A5B2B638A52EF837D
:10148000EF83EF830B6303194B630D740D7C8C6B3F
:10149000B1942B630D740853CB6B443A6D7C10955B
:1014A0008E8C6E84AF8C2E7CB0940F848D73EF8302
:1014B000308CF3A4D3A4718C518CEB62C952664278
:1014C0004A5BAC6B4F84C84ACC6B873AE842AF7C2E
:1014D0008219A742284B6853474B2964E95B863A37
:1014E000284B0853C7426C6C4E8D6C746C7402228E
:1014F0000A5CC95B6B742C74AC6B4F8C2F8CF3A49F
:10150000EF8391949194EE7BA84AE529884A8C6BED
:101510004B636B6B4B632219A74AAB6B92A592A5E9
:101520002D7C4D7C519DF09452A5D09C33ADAD7B6C
:10153000CE83EF83D39CF39C10846D6B2A63A4311C
:101540008B6B2D7C4E7C2632E94AC84245320743DC
:10155000284B2953A742AF7C074349642A6485324C
:10156000274B074BCB63AE7C4C74CA5BEF84C95BE3
:101570000A5C674BE95B2F8DCF8C6F8C6C738D731E
:101580004C7391949194B19CCE7BC952A531474A3A
:1015900088524742263AE9528B638F84B08CCC73D1
:1015A000D0946E84AE8C509D109DF09C94BD54B52B
:1015B00095BD508C0F8433A5B5B594ADB09490947F
:1015C000AF94D4B5B3AD094B863A69534532E9635C
:1015D000685BE94A0D746E7CC642264BE95BC642E5
:1015E000284B0C6C2532CC6B49536D74274B2E85E0
:1015F0004B6CED842A6CAC7CAD7CCF8C2E848D73CF
:101600006C73AD7BEE83D29CB194B194EE7B0B6393
:10161000274AA53985316429884AB08CB08C0642A6
:10162000E95A8C6B0D7CF094F19C53AD53ADB094A2
:1016300094B512A5D5BDF5B5329DD08C2E7C909475
:10164000CD7B4C6B2F84CB632753E64A4B746C7471
:1016500048538A63885B67532643674B8853A95B6B
:10166000A95B695B495B2A5BE84AEB6B6853AB7427
:1016700009646B744A6C0C850D85EE848E842E840F
:10168000708C8C730E84EE834F8CF29C4F8C0E8486
:101690004C6B0B63A95A64292B5B0E7C0E74442996
:1016A0000742A95A2B632E844F84B094B5B573AD0D
:1016B000B4B552AD94B5D08C6F84CC6B0A636C73A7
:1016C000CE7B508CAE7BCA63C95B8C74E95BE95BF3
:1016D0006B6CCA5B8753096C47536C74C85BAB7CFB
:1016E0008B74C642CB6B8A636A5B4C74CC7CEB7C9C
:1016F000AB74CD84E963496C4D8D4A6C0F8DED7BE5
:101700004F8C0E844F8C909453ADD194B094F1A42F
:10171000EE838D73AA5A684A2B63CA5A4C636529B3
:101720008631484AC639CA5A4B6BCD73908CB5B5D1
:10173000B3B531A5109DF0944E840E7C4B6BEA62DC
:101740002F8C13A591946632484B6D6C6C6C6A6457
:101750006A6C0743A63A48538D7CEA6B6B744A6CFB
:101760004B6C6D7C8A63AA63042A0A648A74486C91
:1017700009644B748C7CE963A753095C2E852C7437
:10178000D0940E84E95A0F84B19C708CF29CF19C29
:1017900074B5EE836C73AA5AC639A531C6392421B3
:1017A0008A5A85318A5A2C6B694A2F84EE7B909431
:1017B000B094D09473A5119573A5D19CEE7B4C7316
:1017C0006C73EE83EE83E942CC5B0943CB5B4E6CDA
:1017D0002E6C2D6C2D744D74119D6E84AE84AE8470
:1017E0004D740D74ED730B6C274BAB74AB74496C7B
:1017F000464BAD7C0B6C8D7CEA636B74E9636B7458
:10180000CE8C2D7C4B6B6C73CE83508C8D738F8CF8
:1018100032A553ADCD7BCA5A8952484AC641863952
:10182000E8496531C639EA5AAD7390842F842F8414
:10183000D194B094D19453A5708C5094EE836C7372
:101840002B6B4C6BCD7BAD63CD63ED6B8C630E6C02
:10185000AD63AD636B5BCD73C9524F848B63708492
:101860008C63C84A8B638F8468530643685306436E
:101870006A74EA636D746D74C9632A6C2A6C0964B6
:10188000CA632C7C0D7C0B6B2C73108C919C6B6B46
:10189000F19C74AD0F84EF83CA5AAA5A895ACB625D
:1018A000AB5ACB62C95A2F8C06426B63AE736D6B19
:1018B000CD734F84AC73129D73AD129D919CB29CFD
:1018C000B19C52A574AD2B5B2B5B4A5B9084AE63DD
:1018D000CE6BAD63EA524C63EF834D6B50840F7C4B
:1018E000B18C0E74E5294F7C4E74084BA542074B12
:1018F000C9630A6C2B6C885BE9630A6CCD84CC7C71
:10190000AC7CCE84E8520F8CCF838E7B0F8CB0944E
:10191000D194B19433A5D2A45194D3A454B50C6BF3
:101920000C6BAE7B0A630A63274AA952484AAA5243
:10193000918C4C6BEE7BB19453A553A5B5B5F29C3D
:1019400073ADF5BD32A5EA52AC6B2B5B4B5B0E74ED
:101950004B5B4F7CEE732C63CE730F7CAE73EA52FD
:101960006B634F7C273A8C632E74AC6B2C74CA6308
:10197000EB6BC963CC7C8B7C2A6C8B744A6C875371
:10198000C85B0E8DEB73E9620C6B108CD2A44F8C8C
:101990006F846F8C13A534AD79D6DBE618CE34B5E1
:1019A0004C730C6B4B6BEA622B630A63484AE73952
:1019B0006C6B8D73CD73D19CD194B194129D4F8C6F
:1019C000F29C129DF29CC952ED73EE732C5B2E7447
:1019D000C8428B636F7C9084B18CAE6B6C634A633E
:1019E000CC6B7084AD6B0F7C6C63D18C4E7C8D7C2A
:1019F000EE8CAD84AB7C6B742D8D2A6C4A6C0964C3
:101A0000AB7C4A740F8D6B6B6952484A308CF29CE8
:101A100033A52F8453ADD3A438CE18CE9ADE59D631
:101A200075BD8D7B0B6B4C73CA62CA6269520742EB
:101A30004C63894A2B5B908C6C6BAD730B63CD73DD
:101A4000CD6B6F7C4E74CA52EB524C638C638B5BD4
:101A50000B6C6953294B2A53CD6B2F7C0A5B0E7C90
:101A60006F847184928C728C0A530E746B5B8E7CC3
:101A70008D7C8D7CCA63AE848D7CAD7C0F8DA95B23
:101A8000C53A67530F8DAF8C0E7CEA5ACE7B708CB3
:101A90002F842F8C0F84F4A459D699D618CE96BDD6
:101AA000F3A4F3A413AD34AD2C6B28522C736952FC
:101AB0004C63273A0632A5298429274AA95A708CF3
:101AC00070842A534B538A4A6D630F742A536A5B9E
:101AD000A53AA63A084BA742AD6B30840F7C5084E0
:101AE000918C928CB394EC5A6D6390846742E84A6F
:101AF0004D74F08CCF8CD08CD08CF194529D0D74A1
:101B0000284B084BCB6392A5D1948C730E7C0A634F
:101B10000B63CD7BEF83F8C518CED7BD54ADD29CF7
:101B2000F3A49194EE7BCA5A0F8C695AEB6A6952FE
:101B3000694AC631063263210742284A0B63284AA4
:101B4000C63143212B5BCB5210746D63273229536E
:101B5000C7428A5B2C6C49536B63CF73B28CF07BAA
:101B600031848E6B6E6B4D6B7084CD6B6A5BCC6316
:101B7000AF840D746B6350844F840F7C7084CD6B85
:101B80006F7C8A5B4C74495B2D7CAC6B8C730E84D0
:101B90004C6BCE7B4C6B6E7BB7BD55ADF4A434ADB6
:101BA00054AD70944C6BAA5A0B6B8A5A895A2952BD
:101BB00069522321CE730642484A895A0C63AE7B90
:101BC0006D73EB62EE7BAB4A2D5BAE6B68420953E3
:101BD0008321CB6BE74A8A5B2632AD6BEB5AAA5264
:101BE000EC5ACB5A8D6B2F7C0E74CC6B6F7CAF8410
:101BF00009532E7CAD73CF7B518CF394CD6B4D7418
:101C0000EE84C95B895B0B6CAE842E7CED7B90947B
:101C10004C736C730B638E7B108414A5D39CF3A45C
:101C2000CE7B0F840F84EF834C734D738A62495AC5
:101C30006952A639C95A0A5BCE7B2C732C6BEF8391
:101C4000508CEF83EE7B2942F07BAA4AAA4A0A53C2
:101C5000A84A8742AB5BA73AA8420532C531284261
:101C60004D6B48426C63AC6B6F7CAC6BAC6B2E7C89
:101C70004E7C4F844C6BAD736D6BCD730D742B6CC0
:101C8000ED84AD7CCA634C74AF8C0C74F094F0940A
:101C9000D19C8D734C6BA95A4C6B508CF29CD6BD69
:101CA000F3A434ADD3A475B5F3A44C73CA6228521F
:101CB000074A274A074264290742AE83EB6269520A
:101CC0000F84EF7BAE7BC731CC52494268424B5BFD
:101CD0000953863A284B6632E842C94AC94A5084B9
:101CE0004C63AD6B8C6BCD6B2E74CC6B4E840D74D2
:101CF0006F842E7C6C6BCA524C6BED73AB6B853A68
:101D00000A6C2F8D519D519DF194CC73D08C119DF7
:101D1000B0940E84B194708CD194908CCE7B4C7323
:101D20007194719458CE38CE919434AD71948D7B6A
:101D3000CA620B6B89528952E741285286390C6B73
:101D40008E7BCB5AEA5A293A69424C632A53AB63D9
:101D5000E842284B863266328B5B4B5B8842E63129
:101D6000A94AE631473A06326B5B0D742E7C9084AB
:101D7000AC6B4F7C6C6B2F84EE7BE952D08C6D7C0E
:101D8000895B0C6CAC6BB08CF39C918C6F842E7C5B
:101D9000CC73CD73ED738C6B0E7C94AD33A5EF8358
:101DA000AE7BEF83B29C38CEF3A454AD34ADEF8359
:101DB000B29CCE7B4C6B65396952084AA741863983
:101DC00045312529E7416D632C5BEA4AC842873AD1
:101DD0008B538A53E84267324B534B5BAC63C94A1F
:101DE000C952EA52E629AD6B0A53CD6B2E7CEE73D5
:101DF0004B638C6BCD73CD73684A0A5BC84A6A5BD0
:101E0000C74A29536A5B8C6BEE7350842F7C8F8496
:101E1000319D4A63AC6BC9522A63EA5A12A5B6BD1A
:101E20000F8CEB622C6BD2A434AD13A5919410846B
:101E30000F84EF830B63CA6249526A528A5A29524D
:101E4000E849A639E74188422B53C942A421873A81
:101E5000294B28432843E8422A532B53E94AE94AAD
:101E6000CC6B6B5BC94A4C63EA4A8C630A53C94A20
:101E7000884AAC73E952ED73C531884A6B634A5B9B
:101E8000CB6BAB63AA5B2D74AE7CF0844E7C0C7480
:101E9000EF8C31958B6B8852484AEB62CA5AEE7BC5
:101EA0002F8CAA5A8A5A308C34ADB29C14A514A532
:101EB00038CEDBDE79D6B6BDCF7BEB6269524952B4
:101EC000EB626A52C741A4212A4B873A0A4B831915
:101ED000C73A452AE742A73AC942EA4AE5294632C3
:101EE000463AE94A8D6B0F7C48424C5BCD6BA84269
:101EF000E952AC738F846B63CD734F84CD736A6387
:101F00006A63AD7CEE7C4B6C0F85CE7CAD7C8D7CAA
:101F10008D7C30958F84074A8A5A084A48522C6B28
:101F2000308C308C2C6BEF83719434AD14A559CE6A
:101F300099D638CE79D699D6FBE67AD618C696B514
:101F4000D39C6D73108C673A0A4B8C5BA521A41946
:101F5000A8426A53C742294B883AA842C5296B5BFD
:101F60006B5B8D634C6B2C6BEA52C94A4B5BA84A86
:101F700009534A634F84ED7BCD732B63684AA84AAB
:101F8000AB6B2B6C0543664B674B26434A6C8C74DA
:101F90008C740F8D8E844C6B2852E849CB62EF8392
:101FA000108CAF7BB29C95B5308CB29C54AD54ADC7
:101FB000F7BD95B595B595B5F8C5F8BD55A555AD21
:101FC00059CE79D6B7BD6319A42167320209252AF3
:101FD0004A53E84AA742ED6B2632473A473A273A36
:101FE000A9428C63473AAD73273AE5290953CC6B74
:101FF000C84AAC734F846C6B0B632B63EA5A674A15
:10200000A74AA6424432E53A264B432A6C6CEE7C42
:102010000F858D7CEB6BB08C8952EB6248524D730F
:10202000B39C518CF3A4AE7B7194D2A4D29C38CED5
:1020300018C635ADF3A434AD34AD55AD75AD18C685
:1020400055ADB6B595B5C1006211052A052AC8423D
:102050004632C94AE94ACC63CC634A5B673A4B5B78
:102060004C5B2B5BC94A0632683AE94A6B5B8A6370
:10207000A74A4A638B6BEA628D736D734C73A95ADE
:10208000884A463A4532A219A63AA63A4D746D746A
:10209000AF7C6D740F8D5095AF84CD7B0A63108C2F
:1020A000F4A418CEB29C55B5508C34ADF3A434AD25
:1020B00035ADD7BD55ADF4A455AD75AD14A592940D
:1020C000B29413A534A5E729C621E729082AE721F8
:1020D00085198A3A8A3AAF5BAF5B2D43D05B8E4B52
:1020E000F05BAF53F05B1064CF635174106C1064FD
:1020F000CF5BEF5BEF5BCF5BAF53536C12647374DA
:10210000316C8F5B927C316CEF63AE5B516C716CA8
:10211000CF5BAE5B0F740B4BEB4A07322B5348324D
:10212000693AAA42EA422B4BA93AA83A0A432F64D9
:102130004C4B0B43C93A47324732272A4732A93A18
:10214000EA426D532A434519851948322832693AC3
:102150008621493ACB4ACB420C4BEC424D4B516C59
:10216000AE5BCF63EF6371746C533495F4846E533C
:102170004D4B8E534D4BAF5BF05B7274F06310644C
:102180005174CF5B1064AE53AE53AE53306CCF5B23
:10219000CF632F6C2B53CA4AAA42AA42AA42693A79
:1021A000A942CA42EB4A2B5347326832262AAC5323
:1021B0000A438C5367328842A621062AC942C93A8B
:1021C0002B430A432A434419072A072A683A693AE3
:1021D000AA3A8A3A4D53CB42CB4A4D532C4BEE632D
:1021E000EA428C5B949DD184CD63D284CF63ED4A67
:1021F0000D4B4E536E536E530C4B927CAF5B4D5355
:102200001064AE53AE538D4B2C434D4B1064CF5BDB
:10221000306C8D5BEB42EA42AA42693A693A483235
:10222000893A893A4C53683A883A6B53883A8B53C7
:102230006A4B8B53262A27324419641947324B4B79
:10224000672A2A43A82AC521683A4B53A9428D5BC5
:10225000CB42AE5B727CEB424B53B07C528D72959D
:10226000CF7C5195929D9295929D11858D5B0C4BE3
:10227000CC420C4B6E5BCC4ACB428E5B6D532C4BED
:102280002C5351740C43EB3AEB3A2C436D534D4BAA
:10229000306C2C4B4C538D5B893A693A072ACA4201
:1022A0006832893A8D5B0B4B0A4BE942C9420D6497
:1022B00029438B53A83A072A4411A621AA42C93AB6
:1022C000672A2622C519C94A4732883AAA420B43CF
:1022D000EB3A8A324D53EB4A907C939DF084F08424
:1022E0005095919D919D9095D2A5D4A57174CF6381
:1022F000106C927C4D5B6D5B0C4BCE632F6C6D5301
:10230000CE63AE5B2C4B0B43CB3A0C436D4B8E53E1
:10231000AE5B2C4BAA3AEB4A8A42CA42493A073290
:10232000693A693A8A42C9424B53E521A83A4A4B75
:1023300087328B534B532732031128324832C93A24
:10234000C93A472A262207322832072A8A3ACB423C
:102350008A322C43AA3AEB422B4B0E6C0D64D3A568
:10236000308D9195B29DD29D14AE4E740B4BEC42C4
:102370004D533395949D907CEF6BD284F7A5EF631A
:102380000A4B6D53EB42CB3AAA32CB420C4BF06373
:102390000C4BCB42EB424832A93A683A48322832D9
:1023A00089420732493A48322B4B0A4BAC5BA83280
:1023B0002A43672A2B4B283224112832E629EA4285
:1023C000262A0A43C5194832683A072AEB4AAA3A2C
:1023D0002B43C93A8832A93AE9422D6C71959195FF
:1023E000AA53508D13A6B29D939D0A4B0B4BF16BD4
:1023F0002D538C5B3395EB4A98A5169532746E5B22
:10240000EF6B6D532D4BEC428A32EC428B3AD38406
:102410008A42AB42CA42693A683A893A0732473A35
:10242000473AA942AA4A0B4B0A43E93A2A43C83A17
:10243000093B0A43EA4289428521C6214832062ADD
:10244000673264198419673AA842E94A2A4B094B52
:10245000A83209436A4B6B4B0C648E7C308D0B6445
:10246000863210851085B395949DAC5BEF63CB42AB
:102470000C532F74D6A577A5537C9FEF97A5B58CE9
:102480003EDF31748F5B6F5B2E536F5B4E534E5B41
:102490000D530C53EB4A6A3A8942072AC7298942ED
:1024A0008942EB4A483AEA4AED6309434A4B4A4BB0
:1024B0006B4B2A4B883AE731C629C629A521C62984
:1024C000E62923114311C5292A4B0D6C0C6CEB63D3
:1024D000AE748E6CAF74CF74EF84EF842F8D508DFB
:1024E000EF7C2D64E942528D8F74949DB5A5928442
:1024F0009284D1842B53A82999A5B48C9484ED524D
:1025000019BE6F632E538F63D48CB06B8F63CD5223
:10251000906B4E638F638F63EC52527CD06B0C5385
:102520004E638A426942893A2A4B2A4B8C530A43AA
:102530000A430A4B4311E629E629652165216519FD
:102540008521A5218521673A0D6CEC63F084AF7C71
:10255000CF74107D0C64EF7C308D50955095929522
:102560008F746C532B4B4C53B1840E6C4F7CF39493
:10257000517C17B6FBD67384D26B99A51AB619B6DF
:10258000B8ADD8B5F9B5D8ADF594B06BAC4A8C42BE
:102590008C4AB06B8C4A4A422A42D8B5FDD62F5B92
:1025A000BCCE1174307C2732683A2B53EA42683231
:1025B000C93A062A231123114419E731E73165216D
:1025C00007322732E2080B4B2C4B6D530F64F17C22
:1025D000D17C0E64ED5BD07C519571957195118D18
:1025E000CA4A6D5B9284D7A5527C769DD7AD75A5FE
:1025F0001CD7BFEFBFEF537CF26B98A5DCD67CC62F
:10260000F694B68CD684F68C779DD8AD97A5337C9E
:10261000159DD7BDB7B5D59C91730E5BD27B4B4A48
:10262000B8B529326E5B7284493A8D63CA4AE62195
:102630002B4B4732EA4A241924198629C62903114B
:10264000E729E6292311682ACA322C43EF5B706C14
:102650000F5CAD538C53CD5B6F74CF8472950E6C51
:10266000693A10746F63D58C369DD8ADB384CB4274
:102670003DD7779D2E534C3A705B789D3BB65CBE40
:10268000BEC67EBE3DB69EBE7DBE3CAED9A5D8A51B
:102690005695B484737C9484179578A599AD38A524
:1026A000D694B06B8A422C530F748D630B534C53EA
:1026B000883A6C536C5BA208C310E418441944199F
:1026C00024112732A521482A2C434C436C4B2B4321
:1026D0006D4B4C4B8D532E6C118D1085D3A54B5BE0
:1026E0006A42CB4A6A426B42569D2E53F16B0D4BA8
:1026F0006B3AC8212A32EA292F4B37953BAE1BAEE5
:102700005CB6DFC65DB67DB63CAE1BA61BA69CBE06
:102710005FCFFBA5FBA51BA63CAEBB9D7A959A9D02
:10272000B78CF2736F6368428842AC6BEA4AE62961
:102730006419893A072AA208C3180419041923192D
:1027400024198942A629A9326C4B4C4B8932CA3ACA
:102750000B43AA3A2B4B11859295929DD3A5883AAB
:10276000693AEB4A6D63F4941174AC422B320A2A35
:10277000CC4288190A2AC929CE4A989D3ED73BAE39
:102780005CB65CB69EBE7CB63CAE5CAE7DB65CB65E
:102790009EB6FC9DFC9DFB9D1C9EBC95FC9D3DA694
:1027A0007A9DBAADB063EA5209538742EB4AEF63B0
:1027B000072A272A4419C210E31845210419A20840
:1027C00065216419C629482A0B43EB4269328D53AF
:1027D000ED5B0D6414A614AE13A6F3A57295A73A8B
:1027E000EA4A78BE507C0C53AB4209326A328B3ACB
:1027F000AC420A32EA3188214C32F78C9FE7FBA5C4
:102800001CB69DB65CB63FCF3CAE9DB67DB61CAE49
:102810003CB6FFC65DB61DAEFCA5FC9D1CA6FCA586
:102820001CAEDBAD5384AA4AAA42EB4AA94A683AD5
:102830008C5BE529C5294419442123192319C208B1
:10284000A62924196521072AAA3A0B4B4D53707407
:10285000AC53EC5B9295CF7C30855195EC63C83AD4
:102860000A4BA942A5218E638B42E829CC42CC4277
:102870006B3A9063B16B6821EA29947CBFEFF784CF
:10288000715B50530F4B136C3BAE3CAE7DB67CB6C8
:102890009DB6BEBE9DB69EB65DAE5DB63DAE3DAECE
:1028A0003CB67DBE579DAB42EB4ACB4AA94A683A3B
:1028B000641988428842C20885212311273A45219C
:1028C0006521C3100419282A4832EB426D532F6C3E
:1028D000AB53AF74F07CEF8471951085F084CB5BC3
:1028E000E942E629073292844A3AC7294D538B3A86
:1028F0004B3A0E532E5388212B32B47C7374957C43
:10290000178D57955795178DDAA5FBA5999D9DBEF7
:10291000788D1364336C346CD67CF78CBDBE178D08
:102920001BAEBEBEB9A5AF6B8A42EB4AC94A26327E
:10293000883A84214419AD63C529842123192419B7
:102940002419C3100419E6214832CA422C4BAD5B4E
:102950000D5CAE6CAE748E74518D1085CF7C6E7430
:10296000CD632832E82993844A3AE8294E5B4E5BCE
:1029700009328C42AC42C9298819B484905B126C2C
:10298000D163905B4F53CD42CE420E3BAC322E43CF
:10299000B05BD163D26BF26B3374789D947CD9A514
:1029A0007CB6FECEBDC69484EC52AE632B53E94A8E
:1029B000A842473A241124114B538421C108E31043
:1029C0000419E310241948324832893AAA3A4C4B88
:1029D0004B430E5CED5BAF743085318D4D746E747E
:1029E000ED63893A8A42B7A5293229324D5BCC4A38
:1029F00009322A32E929E9296B3A3695AC42C921D4
:102A0000EA21EA212B326C3ACD420D4B116CB47C99
:102A1000D0631274937C93842E5373748B3AD57C59
:102A20002E4BAD3A2F4BCC4AAC4A8F6B0A4BE94A3E
:102A30002632A421E208E308C6290732EA528208B6
:102A4000A20882082419CA42CA3ACA3A6D534C43B2
:102A50008C4B4C432F64ED5B8E744E6C2E6C907CD3
:102A60004C5B0C53AF63F06B8A3A69322C4BEC42EF
:102A7000AB3A0D4B8B3A6A3A2A324F5B0E532E53C8
:102A8000B15B9474368D9484537CB48CD49436A505
:102A9000F49419B69BC61CD73DD73DD75AB6BCBED9
:102AA0005BB6D99D989DF16BCC4AAB4AA529842190
:102AB00043114319A200C729E8398208C3102C5BCF
:102AC000652144210311CA3AAD53AD538932682AB6
:102AD000CA322B43CE5BA832C842EC63D084329515
:102AE0006C5BEB4A4D538A42EC424D530C4BAA3A75
:102AF0006932292A082A092A2A3288210E4B905B3A
:102B00007374D47C368D779D3AB69BC6DFF71ED79B
:102B10009FE7FED6DDCEFAB5779D737C5BB65CB6DB
:102B20001BA6FAA57CB6DDC6DCC639B6B6AD55A582
:102B3000B6AD349530847EE7DFF7DFF7B7ADC3106D
:102B4000894AE73145216832CA422B438932EA3A41
:102B5000EA3AAD53CA42E6212E745295F084B0840D
:102B6000CA4A8A428A42CB42AB3A8A3AAA3A4932A4
:102B70000B430B434D4BCF5B4D536A32B05BAF5BA6
:102B8000AF53F063F06311646F534E4B1585368D70
:102B9000989DDAA5799D999D1AAE5895A929715BE2
:102BA0005474546C7574547433745474F9AD17A51B
:102BB000D58C3685389D379D589DFDCEDCCE7AC6A6
:102BC0006A42AE6B6108072AA94288324832CA3A83
:102BD0002B43AA3AEB4A2B536F844E840E74B08475
:102BE0006C63AE6BCF6BAE63CF5BAE638E5B0C4B37
:102BF0004D4B2C43EB3A8A32292A8A32292AE82182
:102C0000292A292AAB3AEC42C821C9196F53D15B52
:102C1000F26B747C915B126CF26B547C4F5B68219D
:102C2000F78CD67C5474F263F36BD36B9163B26B05
:102C3000B2639153D3633574D7845CB6999D747C29
:102C40009CC63DDF8629A52188422732E942893A80
:102C5000AA3A483AAA424C63CE7BAD7B708CEE73A5
:102C6000A9420B53AA42A93AAA426A3A29326A3ABD
:102C7000493A2932282A4932082A292A08226A325E
:102C8000AB3AAA3AEC4AA721E829C821ED426C32B6
:102C90001695B4842E53A82188214B3AE929A40023
:102CA0006F5B2B32E929E9210A2A6A3A8C3A8C3A7D
:102CB0006C328D3A8D3A6D3A304BD25BF36354747B
:102CC000957C3695D48C8421A94288428842072A73
:102CD000683AC629AE6BEF7BEF83AE7B8D734C6396
:102CE000483A4C530B4BEB4AAA42CB4A693A28323A
:102CF0004832693AE729082AE829C8212D53B37CCC
:102D0000158DF9AD3AB6F16B8721E8214A324B3285
:102D10008C426C42127CBBCEF8BD05190A3AA40065
:102D20002E53C921092A0932E9312932A829E93962
:102D30002A3AA931E939E93188294F5B2A3A061143
:102D400067118B42B7AD473A683A473A0632A52138
:102D5000473A0B5B4C63AE7BAE7BCE7B2B634D6304
:102D60008942B284F7ADEF63CA4AAA428942483227
:102D700027320B53AA4AC721493AE829D06B937CE2
:102D8000169599A5547CB9A52A32C8218A322932D0
:102D90002B4288297BC69BCEBBCEAC522A3A061169
:102DA0000A32A821E929A8212A32AB42E931E931C6
:102DB000093AC931A831672147212A3A77A55ABE75
:102DC000E41026111174A8420A530A538B634B5B1B
:102DD0006F840E7CAE73EE7BEE83308C8D735184EA
:102DE000073286218E634C53CA4AEB4AA9424832C5
:102DF0006732B07C2B53E629493A041182088200DD
:102E0000830007116D42337CEE4AC921AB4287290A
:102E1000D07BA839BBD63DE7D9B5AC4AE93187218B
:102E2000E931872108328721C929E931579D369533
:102E3000158D789D799D799D599D589D9584DCD6F9
:102E4000051167190C4B0522494B8A53AE7CD08C77
:102E50002D74CD6B6F84708C0F848D73EF83518CC8
:102E600024216629493ACB52AA42CA42893A4732BA
:102E700067326F74ED63E62907320411C310E41062
:102E8000E410C2082619D26B4E4BA7118B32662173
:102E90004A6BAA4A317C5EE798A529328721A308AC
:102EA0008721E931AC4AED52EE52137C8B42051179
:102EB000E5100511C510E610E610E51867299AC659
:102EC000A8294842F29C652AA632E732A632284B4E
:102ED0002C64CF7C0D74CD732F84AE7B6D73CF8348
:102EE000C3188631E8398B4A2C5B693AA9424832CB
:102EF0002732A83A4732683AA6294419E41004193F
:102F0000C310C20863089163EE428711CC42A72127
:102F10004A424B3A0B322B3A0A32537C2E5BEC522C
:102F2000CC4A4B3A4721E5100A32E931A308872100
:102F30000932C729A8296621872945196200C829AD
:102F40004A3AE741AD7BC732283B483B69432843B7
:102F500048438A4BCB63ED732E846C6B2B63074223
:102F600065298A52E83909422D5B493AE73128320E
:102F70000732072AE729283A85214419E3106521F9
:102F800004194519A208AD4A305BA819CB4266194D
:102F90008E4A6C426C3AEA318C420A326721E51063
:102FA0008721E5100619CD4AC92905116621862118
:102FB0006A3AA72986212519252145196200E83199
:102FC0006A3AE731A629251A283BC62AE72A483B50
:102FD0002733273B694B08534E7CEC732A5B432114
:102FE000C6310B63A73109420C5B4D638A42AA4A82
:102FF0000C5B8942E7292411852124190419EB521D
:10300000CB52C8310319093ACF4AD0635595727C27
:10301000AB4AF073117490634C424F5BCD4AC9299F
:10302000C9296721AC4A6721E9314B3A4519E8299A
:1030300066192519662126196A42A73142082A42D3
:10304000537C527C327CE73268438943A94B4A5C0B
:10305000C94B0A5CA953A95B8953284B8A5BC429D5
:10306000E63107420842863125216629A310A631A0
:1030700086292D5B0D5B8E6B8629E318CB520C5B8A
:103080004D636A42C73146214A42AF6B7BC6948C7E
:1030900022008729327CF273B16BB26BB16BF27391
:1030A000F2735484AC4AC4101174117C0D53A829D6
:1030B0008829C8310519C4100D5B2E5B8D4A0B3A67
:1030C000337C137CF273E63A0A5CE953A84BC8538D
:1030D000C9530A5CCA53E953C853C8534B64E74207
:1030E000E631274208428731452925216208EF7BD6
:1030F000662966298308051924198208EC522D5B7C
:103100002D5BCC52293A8729C310C41046212621B1
:1031100005192521E518C418C41005110519C41096
:10312000E4100619261945190511461925192619FD
:10313000C410C410E410C410C510C510C510C410CC
:103140000519E310E210073BC9534743A84B0A5C3B
:103150004B64C953A84B6B6429546A646A648753EF
:103160006A5BA94A073AA6314521E418C418C73951
:10317000E41886298631821062084100293A6E6B74
:103180008A4AAB524942A729E41883082621E41051
:10319000C410C3108210A310C31025190519E41020
:1031A0000411E418251926194619E4106621CC5299
:1031B0004A426B42E93967298408E518C310863111
:1031C000E639C742A95B48434B64E953884B274320
:1031D000A5324743C84B4A5C495C6A648B6C674BB9
:1031E000AA638A636A63473A0211E310E318E4189A
:1031F000252104212421A2106529E418AB4A2D5B66
:10320000294229422942E8316621A31025210421BF
:103210004208620862088210E41826212521E41879
:10322000252104216B42AE4A11740D532D5B0E53C0
:10323000906B70635384159DE8394621C41826218C
:10324000EA4AAE7CCD7C48436743EA53E953C95B05
:10325000E53A674B874B463BE84B8B646743842AD0
:10326000E6426853484B0B64421964212C63A73132
:1032700009428631E318484A8D6BC6294F634E5B7D
:10328000083A293A4942E831E831A31004212521BE
:10329000C3186208C418A310A310A3108631C31862
:1032A0006529C3104F63515BB9ADD8AD5695D8AD04
:1032B00098A53ABEB9B556A5B073094245298631DD
:1032C0008742096C6974A532063B4743095C29644F
:1032D000C85BE95BE95BA74BE42A4643A953432259
:1032E000242A0743063BE85BAA5B0532E6396629D8
:1032F000252983106A4A09422842A529F26BB06346
:10330000C731AB52E831E8314942A3100421E41837
:10331000A731C41825210521E418A3104529A63199
:10332000AA52AB4A4621F373B48C117C317CF07302
:10333000327C8F636F636F6BAB528631863186311F
:10334000C84AEA6B496C442AA953A532C85387532B
:103350008753C85B47434743674B2B64232208438B
:10336000252AE742632AA64B88532853C00803192D
:10337000E3188210C318A418A3188208347C747C44
:10338000A62929426A4AE8316A42A310252104216C
:10339000E4186629252146290521C418A731073AD2
:1033A000E739E731083A6729C8318729A7298629EB
:1033B000662987292521E418C3180421C739A631B5
:1033C000A84A032A2753E742AA5B0743E532884B02
:1033D0006532274B064326436B6C68538532E429DC
:1033E0006319AA5BEA634964095C0A64A64280081F
:1033F000232143218110A310A3188208B484F68CE2
:10340000A63108420942E8396A4A04210421E31836
:103410004529C318E420C418262966292421031944
:10342000E3104429A6316629C7398B528A4A662996
:10343000A308E41862082521831025296631A731E5
:10344000884AEC730D74A31965328532C63AC53AC1
:103450008953074B684B8432E63A8532453262190C
:10346000E529653A2753C43A874B6A742B74495B44
:10347000295BC852E110E210E3186208B484789D19
:103480002521C7390842A7314A4A24218210E3186E
:10349000C3188210C318C318A318A210A210C3180F
:1034A000C210031924212421A63165298A52494AD0
:1034B0006108C3180421E418E4186529452904218A
:1034C0004B63CE73AE732A4BC83A462A4D6C8319B0
:1034D000663AC7426953C63AA95B885B453AE84AEF
:1034E000A642864289632B74A9532C6CC219495396
:1034F000E84A285B253AA42964210411327CF8B5F6
:10350000A31086318631C7394A4AA3106108821058
:10351000611082108210C318C21803210321C3183E
:103520000419031964216529032145298631494A73
:103530004108C318E318C218E31844296429E218A3
:103540002B638D732B63683A0A4B6732A73A094B9A
:10355000AB6325322C6CC53A4B6C2B6C4432285330
:10356000A6424853CE84AA634C6C6E74E7426953FA
:10357000853A8542695BA74A263A64212D5BD7B517
:10358000E41086314529C7316A4AC318A210A21037
:1035900081108110A210A110E2188429E73924219A
:1035A00004194521842926428429A531442907424A
:1035B000A210A210C218C218E220642902196429BC
:1035C0008C732B638D7305320A538742CB5BE742C2
:1035D000C7422D744D746853C53A475365326532FE
:1035E000EB63A63A6953495BAA5B084BAE7C8953EF
:1035F000474B4753685B8A638642C5316842D39420
:10360000051966298631252108428110C318A210A8
:10361000A2108210A21024216529A5310319E731D7
:1036200085296521C5296642053AC5398531C639DE
:10363000C2184429A6312321E639C6390321AA52EA
:103640008D730F84CE7B463A663A0B6C0A64895BB5
:10365000AA5B4953284B2743064348534753AA5B69
:10366000495329530953A7422C6C074B6B6CC85B19
:103670006B74885BC863A963485B2532473AA94AE3
:1036800045214529452925210742C218C318E420B0
:10369000C318A318A318A21845290742C318242148
:1036A0000419242106324642674A884A8429684A16
:1036B000E639684A8D738852484A0742474A0742AA
:1036C000A531AA522C63E74A8C742A6CC85B8C74AF
:1036D000EA63484B8953474B2B64E9632B6C8D7C21
:1036E000863AA95BAA5B6A53EA636C74AB7C4A6C4A
:1036F0002B6CA95B2B746B7CCA632853463AC52993
:1037000044212521E4182421A63165296529E318DF
:103710000421E420C318C3104521C731E320C31896
:10372000E32044294421273A073AEA5AEA5A894AC7
:10373000A94A0A5BEA52484A694AC639E739EA5A4D
:103740000B63484A2C63A7422D6C2C6C2C6C4C6C80
:10375000284B453289530A64C963096C0A6CEB6BC8
:10376000EC6B69536953084388530964E75B496C00
:103770006C74A9634853EA63074B8D7CC74A4219AE
:1037800022192321E31823216429C6398529A6316A
:10379000452945210419E318E31886292429E32043
:1037A000042104218631E739073A684A4C636D6B7E
:1037B000CA52C952E952E952EA5A2742E639CA5A6C
:1037C0004C6B2B63CA5A0A4BA83A0D6CCC634D74F0
:1037D000AE7C0C6C2D74EF8C8E84CE8C8E844D7CE4
:1037E0002D742C74A95BC63A6A6CCB74AB74054318
:1037F0002A6C2B74AA63E64AC9634C740B6CCF8C99
:103800008429E218C21803218531C639E639894A6C
:10381000073A45210319E310E310E318C3184529BB
:10382000042165296529A631AA5A2842CA5AEA5AAA
:10383000CA528D6B8C6B8C6BEA5ACA5AC639684A6D
:103840008952C9520A634A53CC63CC63EC6BCB6395
:10385000ED6BC94A4E7C2A5B4F7CCC6B4F7CCD73A1
:10386000E84A8A5B4D74AA5B464BC75326430964FA
:103870000A6CEB6B0B6CCA63EA63264B8853AA6332
:10388000E85284298429C5390642E6392742EA529A
:1038900048426529652103192421031924210421A3
:1038A000242124210842E7418A52695289522C631B
:1038B000EA5A0A5BED732B632B63CA5AA95A064274
:1038C000EA5A8852C95288426B5B7084CD6B8C6314
:1038D000CD6B0A530A53AD6BCE7370842F7C2F844B
:1038E000AC6B263AED734D748853C43AE6420A6CC9
:1038F000E963A95B6853EA638853CB746A6C895B9C
:10390000295B674A474AA539E639684A47422B5B33
:10391000EB5ACA52694A6529242945298631A631BC
:103920008631A631A6390421E739484AAA52694AA4
:10393000CA5AA94ACD6B4F844F844C6BAD73AC739C
:103940008F946F8C4A634D630C5B4C5BEE736C5BC6
:10395000707CCD6B4B63CE73CF73EE73EA52CE7334
:103960000F7C27424B636F842953AA636853C96352
:1039700087538C74E95B0543E95B8A74E85B0964EF
:103980008C7C8742A952C639EA5ACA5A694AEB5A0C
:10399000CB520C630C63AA5A4D73CB62E6394429AF
:1039A0002742E63986316531A639A53165294C6B48
:1039B000684AE952AC6B6F844F8490948C73AF94D7
:1039C000119D8E846E844D63317C8D6BAD63E94AAD
:1039D0006B5B6F7CB08CF2948E738D6BEA52AE731E
:1039E000518C2C638D6B6C63B08C6E7C6D7C6C74B5
:1039F0006B74AB746A74EC7C2964E963464B496C64
:103A0000AB7C4D7C263AE639E639CA5A2C630C6306
:103A1000AA52AE7B2C6BF0835194EF838D730742D7
:103A200027420742E7390842284AE74144214842F1
:103A30004742A94ACD6BCD73AD734F842B63ED73B1
:103A40008F842D74AF8C083A2C5B8D636C5BEC6BB0
:103A50006B5B4A5BE952AD730F7C2B5BEE73318479
:103A6000318414A591944C63ED73EC6BAF842C748A
:103A7000EF8CEA638C74CD848C7C8D7C0A64054366
:103A8000674B8E7C6B632742E6390B63308C4D6B42
:103A90004D6B10846D73318C108C518C508CEE7B7F
:103AA0008952C95ACB62A639E741C7412421EA525B
:103AB000C629483A8C63C9524B63CA524B634B6365
:103AC000CD73ED73D08CCC52317C4D632A53873A41
:103AD000873A084BA7428C6B3084EF7B308431846B
:103AE000318431844D6B0B5B90848742A742D08C2C
:103AF0006E7C4E74D08C6F7CB0848F7CCB638532AF
:103B0000284B4D74F08CCD73EA5A2C63694AEB62F2
:103B10004D6B4D6B7194D3A4B29C51948D736D73A6
:103B2000AE73AE7B8E7B495286394952A63127420D
:103B300085298529442165318531694A6D730E7C5B
:103B4000884A2A5B90844E63AF6B493AEB4AC8427D
:103B5000CA5B6D746A5BED6BCE7351847184317C8A
:103B60008E7310848E730F7C0E74294BEC636F7C04
:103B70008F8CAC73AD733084EF7314954E744E74A8
:103B8000C842EB6B2C742D7CC9522B630A63AA5A72
:103B9000EA62AA5A0F84508C7094EF836D736E732F
:103BA000AE7BEC62E849CB62A6390742C639653183
:103BB0002421C63924212842284AEB6208422421C4
:103BC0008529C9522B5BAB4AAF736A422C53A4219F
:103BD0000C64E73AAA5BE5310F7C6D63CB520C5B5A
:103BE000EB5A6D6BEE7BAD73AC634E740D742A5B58
:103BF0000D7C8C730E849294F39CEE73EB6B8D7C36
:103C00008953A95B685B0C74AC6B2B636C6B274AA4
:103C10006C6BA95289522F8C919CEE83EF83B29CDE
:103C20006E73AA5ACB626952084AC741A639A639AF
:103C3000E3204D6B074207428952AB5A8E7B8D734E
:103C40002B63AD738C6B4E63CB528B4A0B53A842E4
:103C5000C73AEB5BC742A842483A073A49424C632D
:103C6000AA526D6B6C6B2E7C0D6C0D74ED73AC6B8E
:103C70002E84AC738C6B8C730E7C2D748C7C8C7C42
:103C80002B6C68534C744D7C4E84AC739094AC7325
:103C9000674A684AEA62EA62EE7B5094518C0C6390
:103CA0003084EF838E7B6952CB62284AE741E7413B
:103CB0002529284208426D732C6B4D6B8E7B0F8437
:103CC000AD73AD73A952494249428A422B532A4BE4
:103CD000C73A694B8632A842483AAA4AEF7BCE736C
:103CE0000B638C6B8C6B4E7CED6B0D6C0E74D18CFE
:103CF0004E846B6B095B4B630D7C8A5BC5424B6CDE
:103D0000AE7CAE84CF8C4D7CEC738F8C8F8C6F8CA3
:103D10008C730E84A9522B636C6B6C6BF3A492941E
:103D2000718CF3A4D29C71948A5A8A5A084A8639B3
:103D3000084AE7410421C6414C73084A49520F849E
:103D4000AD73CE7B684AC531AC6B2A536A5BE842DF
:103D5000294BA63A873A6B638D636942694AAA5236
:103D60002842CA52473ACC63AC6B2F7C0E7CCD7391
:103D70002E842A630E842E848B6B8F848A5BEB6384
:103D8000CF84AF8432953295AB6B4E7C908C4F8450
:103D90004F8CCD738F84D08412956B630B5B8D6BCE
:103DA000308495AD13A5308CD3A40F8CAD736952BC
:103DB00069526952494A074A07428631CB5A2C6BED
:103DC0006952CB5A8A5A4842E94AE94AE742694B62
:103DD000AA53084B46324A5B6C63AD6B884AC952A2
:103DE000EA4AC529CC6BC8424F7CEE734F846C63A2
:103DF000CD736B63AC73E95A874A4B5B6E7CA74209
:103E0000AC630953AC6B2F7C6F7C2E7C908CCC7395
:103E10000A5B8C63C84ACD6BB084329D9194AE73BB
:103E20002C63518475B5B194919C508CCD7BCE7B25
:103E30008D73695285396952284AC73965294531D8
:103E40002529084AAA5AC629C94AE529A73A494B49
:103E50004953E842E94A4A5BC94A0A53C94AAD6B29
:103E60004B5B88426B5B2B532B5BAD6B0A5B2B5B15
:103E70008C6B6B6BAD734329884A2A5BC84ACC6B49
:103E80002953EC6B8B5B2E74B0842E748B6372A5FC
:103E9000CC730A53884A684A2B63909434AD0C6300
:103EA000494ACB5A0F84F29CF39C7194508C108435
:103EB000CE7BEB626952284AAA5A6952E741084A06
:103EC0004431E74169526842683AC842A319C83A86
:103ED000252AE94AE94A09530953463A8842684281
:103EE0004A5BCC6BEE6BAA4AEE730A5BA84A884A1F
:103EF0002E84ED7B6C6B2B630E7C8C6BAC6B8B63BD
:103F00004D744C746C742F85EE844D7C2D744D7CF7
:103F10001195ED73684A6852484A484A4D73F083D8
:103F20004D730C63308C13A5D39C7194F39C59CEC4
:103F3000DBDE59D695BDEF838952484A2842AB5AF9
:103F40006A5208422C6BA84A6B5BC4216319C842B1
:103F50004953E842C842673AC84AE5296B5B4B5B64
:103F60004B5B2B5BAE6BAA4A0A53CC6BA84AA84AA0
:103F70008C6BEE7B2F840E840F840A63095BAB6B22
:103F80004C7C2B6C6C6C4B6CC95B4C746D7C2C74D6
:103F9000CF8C2E7C8852274A285208520C6B318CC9
:103FA0008E7B4D6BAE7B4D6BB29C9294F7BD9AD6D7
:103FB000B7BDF8C518CE59D639CE96BD75B5718C3A
:103FC0006C6B718C8D73431926320211E5296B5B82
:103FD000094BC742EC63052AA842473A673A884230
:103FE0008D6B8A4ACF7348422632E94AAC634B5BF9
:103FF000CD6B708C2B63CA5A484AC95A464AA7529D
:10400000CA6B242A07432743C53A4D744D74AF7CCD
:104010008E7C0C74AC732642274ACB62F083929458
:10402000CF7BB29491940F84518C75AD14A5D7BDFC
:1040300055AD96B514ADB7BD55B534AD96B517C6EB
:1040400037C695ADB6B50211063205326742263243
:10405000E8424A53CC636B5B094B46322A534B5BB5
:104060000B5BAA52083A6942A9422A534A53E94AC9
:104070008C63AD734C6B4C6B2C6B0B63EA5AA85280
:10408000253A042A242A484B8532EC638E7CAF847F
:104090004D746D7C10956A632B6349526D73D39C8C
:1040A000718C9294508CB294F39CF4A4F8BDF8BD3A
:1040B00014A5D39C55B514A555AD14A575AD54AD37
:1040C00095AD33A5B194F2CF0EF0F29EF76AE00FF2
:1040D000F66E400EF7220900F5500EBEF28E120069
:1040E000000000000000005F000000030003001457
:1040F0003E143E14242A7F2A12433308666136494F
:104100005522500005030000001C224100004122FE
:104110001C0014083E081408083E0808005030002F
:104120000008080808080060600000201008040269
:104130003E5149453E0004027F00426151494622FA
:10414000414949361814127F1027454545393E49E3
:104150004949320101710907364949493626494919
:10416000493E003636000000563600000814224151
:1041700000141414141400412214080201510906F9
:104180003E4159555E7E0909097E7F494949363EBF
:10419000414141227F4141413E7F494949417F0997
:1041A0000909013E4141493A7F0808087F00417FE3
:1041B0004100304040403F7F081422417F40404052
:1041C000407F020C027F7F0204087F3E4141413E56
:1041D0007F090909061E2121215E7F090909760050
:1041E000F2CF0EF0F29EF76AFA0FF66E410EF7224A
:1041F0000900F5500EBEF28E1200264949493201DF
:10420000017F01013F4040403F1F2040201F7F2091
:1042100010207F41221C2241070870080761514984
:104220004543007F41000002040810200000417F48
:10423000000402010204404040404000010204002A
:1042400020545454787F44444438384444444438D7
:104250004444447F385454541804047E05050854DB
:1042600054543C7F0804047800447D4000204044BE
:104270003D007F1028440000417F40007C0478040A
:10428000787C0804047838444444387C14141408B6
:10429000081414147C007C0804044854545420046A
:1042A000043F44443C4040207C1C2040201C3C40B7
:1042B00030403C44281028440C5050503C44645436
:1042C0004C44000836414100007F0000414136085F
:1042D0000002010204020DAE03D0F2CF0EF0F29EF6
:1042E000F60FF66E420EF7220900F5500DAE02D021
:1042F0000EBEF28E12000000000000000000000060
:1043000000000000000000003EFFFF3E0000000033
:10431000000D0D000000000B0700000B070000005F
:10432000000000000000A0E0FEBEE0FEBEA0000F06
:104330000F000F0F00001C3E726767E2CE8E07076A
:10434000040E0E0407038CD2526C60A0B010000063
:104350000000030404030070F88848300080060F52
:10436000090B060F09080000000B07000000000001
:104370000000000000000000F8FC0F030000000037
:1043800001030F0C000000000307FCF80000000010
:104390000C0E070100006060E0FCFCE060600607B6
:1043A000030101030706606060FCFC6060600000C0
:1043B00000030300000000000000000000000000F7
:1043C000000B0700000060606060606060600000DB
:1043D00000000000000000000000000000000000DD
:1043E000000C0C0000000000C0E0381E07010C07A4
:1043F000030000000000F8FE87C3331FFEF801072A
:104400000F0C0C0E070100000606FFFF0000000065
:1044100000000F0F0000040687C3E3773E1C0E0F59
:104420000F0D0C0C0C0C0406076363F7DE8C020600
:104430000E0C0C0E0703E0FFDFC0C0FEFEC0000044
:104440000000000F0F003F3F33333373E3C3020616
:104450000E0C0C0E0703FCFEC76363E7C68403075C
:104460000E0C0C0E0703000303E3F31B0F07000001
:10447000000F0F0000008CDEF76363F7DE8C03078C
:104480000E0C0C0E07031C3E77636337FEFC02061E
:104490000E0C0C0E07030000008C8C0000000000C6
:1044A00000010100000000000018180000000000DA
:1044B000000B0700000040E0B0B0181C0C06000024
:1044C00001010306060CD8D8D8D8D8D8D8D800000F
:1044D000000000000000060C1C18B0B0E0400C0604
:1044E000060301010000383C0606C6C6FC78000041
:1044F000000C0D0D0000F8FE0371898BFF7801039D
:10450000060C0C080400F8FC86838386FCF80F0F69
:10451000010101010F0FFFFF63636363FE9C0F0F37
:104520000C0C0C0C0703FCFE07030307060403072F
:104530000E0C0C0E0602FFFF03030307FEFC0F0F19
:104540000C0C0C0E0703FFFF6363636303030F0F81
:104550000C0C0C0C0C0CFFFF6363636303030F0F65
:10456000000000000000FCFE0703C3C7C6C4030729
:104570000E0C0C060F0FFFFF60606060FFFF0F0F57
:10458000000000000F0F000303FFFF030300000CF7
:104590000C0F0F0C0C00000000000000FFFF0206D3
:1045A0000E0C0C0E0703FFFFF8DC8E0703000F0F45
:1045B000000103070E0CFFFF0000000000000F0FBA
:1045C0000C0C0C0C0C0CFFFF3CF0F03CFFFF0F0F31
:1045D000000000000F0FFFFF1E78E080FFFF0F0FAD
:1045E000000001070F0FFCFE07030307FEFC030793
:1045F0000E0C0C0E0703FFFFC3C3C3E77E3C0F0F77
:10460000000000000000FCFE07030307FEFC030798
:104610000E0C0F070F0FFFFFC3C3C3E77E3C0F0F46
:10462000000000010F0E0C1E3F3363C78604020614
:104630000E0C0C0F0703030303FFFF03030300002B
:10464000000F0F000000FFFF00000000FFFF030746
:104650000E0C0C0E0703FFFF00000000FFFF01031C
:10466000060C0C060301FFFF00F0F000FFFF070F30
:104670000C07070C0F07030F9CF0F09C0F030C0FA7
:10468000030000030F0C1F3F60C0C0603F1F00000D
:10469000000F0F0000000383C3E3733B1F0F0F0FD6
:1046A0000D0C0C0C0C0C0000FFFF030300000000BD
:1046B0000F0F0C0C000001071E38E0C000000000C6
:1046C00000000003070C00000303FFFF00000000D0
:1046D0000C0C0F0F000010180E03030E1810000032
:1046E00000000000000000000000000000000C0CB2
:1046F0000C0C0C0C0C0C000000070B000000000060
:1047000000000000000080D8D8D8D8D8F0E0070F0B
:104710000C0C0C0C0F0FFFFF30181838F0E00F0FC7
:10472000060C0C0E0703E0F0381818383020030789
:104730000E0C0C0E0602E0F038181830FFFF0307CD
:104740000E0C0C060F0FE0F0B89898B8F0E00307D5
:104750000F0D0D0D05013030FEFF333333330000F4
:104760000F0F00000000387CEEC6C66EFCF8000C8F
:104770000C0C0C0E0703FFFF30181838F0E00F0F79
:10478000000000000F0F001818FBFB000000000CD9
:104790000C0F0F0C0C0000001818FBFB0000000CA5
:1047A0000C0E07030000FFFFC060301808000F0F59
:1047B000010103060C08000303FFFF000000000CCA
:1047C0000C0F0F0C0C00F8F810F8F810F8F00F0FA1
:1047D000000F0F000F0FF8F830181838F0E00F0F27
:1047E000000000000F0FE0F038181838F0E0030761
:1047F0000E0C0C0E0703F8F8B01818B8F0E00F0F05
:10480000010303030100E0F0B81818B0F8F8000144
:10481000030303010F0F00F8F87038181800000F99
:104820000F000000000060F0D8989898B0200206B1
:104830000C0C0C0D07030018FFFF181818000000DF
:10484000070F0C0C0C00F8F800000000F8F8030744
:104850000E0C0C060F0FF8F800000000F8F801032A
:10486000060C0C060301F8F800C0C000F8F8070FAA
:10487000070303070F07183870E0E07038180C0EB4
:10488000070303070E0C78F8C08080C0F8F8000C0E
:104890000D0D0D0C070318181898D87838180C0E41
:1048A0000F0D0C0C0C0C000060FEFF03000000005C
:1048B00000070F0C0000000000FFFF0000000000D8
:1048C000000F0F000000000003FFFE60000000006A
:1048D0000C0F070000000C0E060C181C0C0000004A
:1048E000000000000000F2CF0EF0F29EFE0FF66E08
:1048F000480EF7220900F5500EBEF28E120000E0BD
:10490000F0F8FCFCFCFEFEFEFEFEFEFEFEFEFEFCE3
:10491000FCFCF8F0E000FFFFFFFFFFFFFFFFFFFFE1
:1049200003010103FFFFFFFFFFFFFFFFFFFFFFFF8B
:10493000FFFFFFFFFFFFFFFF00000000FFFFFFFF83
:10494000FFFFFFFFFFFFFFFFFFFFFFFFFFFFFFFF77
:1049500000000000FFFFFFFFFFFFFFFFFFFFFFFF63
:10496000FFFFFFFFFFFFFFFF80000080FFFFFFFF53
:10497000FFFFFFFFFFFF010F1F3F7F7F7FFFFFFF55
:10498000FFFFFFFFFFFFFF7F7F7F3F1F0F01000043
:104990000000000080C0E0F0F8FCFEFEFEFEFEFE1F
:1049A000FEFEFEFEFEFE2070F8FCFEFFFFFFFFFF96
:1049B0007F3F1F0FFFFFFFFFFFFFFFFFFFFF000015
:1049C000000103070703010000000000FFFFFFFFD5
:1049D000FFFFFFFFFFFF00000000000000000000DD
:1049E00000000000FFFFFFFFFFFFFFFFFFFF0000D1
:1049F000000000000000000000000000FFFFFFFFBB
:104A0000FFFFFFFFFFFF00000000000000000000AC
:104A100000000000FFFFFFFFFFFFFFFFFFFF00E0C0
:104A2000F0F8FCFCFCFEFEFEFEFEFEFEFEFEFEFCC2
:104A3000FCFCF8F0E000FFFFFFFFFFFFFFFFFFFFC0
:104A400003010103FFFFFFFFFFFFFFFFFFFF030362
:104A50000303030303030303000080C0FFFFFFFF02
:104A6000FFFFFFFFFFFF00C0E0F0F0F8FCFCFEFEE0
:104A7000FFFFFFFFFF7F7F3F3F1F1F0F0701FFFF6C
:104A8000FFFFFFFFFFFFFF0F070301000000000013
:104A9000000000000000FFFFFFFFFFFFFFFFFFFF20
:104AA000FFFFFFFFFFFFFFFFFFFFFFFFFFFF80E0B4
:104AB000F8F8FCFCFEFEFEFEFEFEFEFEFEFEFEFE26
:104AC000FCFCF8F8F0807F7F7F7F7F7F7F7F7F7F98
:104AD00003010103FFFFFFFFFFFFFFFFFFFF0000D8
:104AE0000000000000E0E0E0E0E0E0F0FFFFFFFF9A
:104AF000FFFFFF7F7F1F000000000000001F1F1F3F
:104B00001F1F1F1F3FFFFFFFFFFFFEFEFEFCFFFFFB
:104B1000FFFFFFFFFFFFFFFF8000000080FFFFFFA0
:104B2000FFFFFFFFFFFF030F3F3F7F7F7FFFFFFF81
:104B3000FFFFFFFFFFFFFFFFFF7F7F3F1F0300001F
:104B40000000000000C0F0FEFEFEFEFEFEFEFEFEC7
:104B5000FEFEFEFEFE0000000000C0F0FEFFFFFFB4
:104B6000FFFF3F0700FFFFFFFFFFFFFFFF0000C049
:104B7000F0FEFFFFFFFFFF3F0700000000FFFFFF09
:104B8000FFFFFFFFFF00FEFFFFFFFFFFFFEFE1E082
:104B9000E0E0E0E0E0FFFFFFFFFFFFFFFFE01F1F9F
:104BA0001F1F1F1F1F1F1F1F1F1F1F1F1FFFFFFF75
:104BB000FFFFFFFFFF1F00000000000000000000DB
:104BC0000000000000FFFFFFFFFFFFFFFF00FEFEF1
:104BD000FEFEFEFEFEFEFEFEFEFEFEFEFEFEFEFEF5
:104BE000FEFEFEFE0000FFFFFFFFFFFFFFFFFFFFD7
:104BF0000101010101010101010101010000FFFFAB
:104C0000FFFFFFFFFFFFFFFFF8FCFEFFFFFFFFFFBF
:104C1000FFFFFEFEFCE00707070707070707070778
:104C200001000001FFFFFFFFFFFFFFFFFFFFFCFC94
:104C3000FCFCFCFCFCFCFCFC80000080FFFFFFFF98
:104C4000FFFFFFFFFFFF031F3F7F7F7FFFFFFFFF90
:104C5000FFFFFFFFFFFFFFFF7F7F7F3F1F03C0F0CE
:104C6000F8FCFCFCFEFEFEFEFEFEFEFEFEFEFEFC72
:104C7000FCFCF8F0E000FFFFFFFFFFFFFFFFFFFF7E
:104C80000301030F0F0F0F0F0F0F0F0F0F00FFFF89
:104C9000FFFFFFFFFFFFFFFFF0FCFEFEFEFEFEFE3C
:104CA000FEFCFCF8F0C0FFFFFFFFFFFFFFFFFFFF70
:104CB00003010103FFFFFFFFFFFFFFFFFFFFFFFFF8
:104CC000FFFFFFFFFFFFFFFF80000080FFFFFFFFF0
:104CD000FFFFFFFFFFFF010F1F3F7F7F7FFFFFFFF2
:104CE000FFFFFFFFFFFFFF7F7F7F3F1F0F01FEFEE4
:104CF000FEFEFEFEFEFEFEFEFEFEFEFEFEFEFEFED4
:104D0000FEFEFEFEFEFE01010101010101010101A5
:104D1000010101F9FFFFFFFFFFFFFFFFFF07000099
:104D2000000000000000000000E0FFFFFFFFFFFFA9
:104D3000FFFFFF1F0000000000000000000000C097
:104D4000FCFFFFFFFFFFFFFFFF3F0300000000002D
:104D5000000000000000F8FFFFFFFFFFFFFFFFFF64
:104D6000070000000000000000000000E0FFFFFF5F
:104D7000FFFFFFFFFFFF1F0000000000000000001A
:104D8000E0F0F8FCFCFCFEFEFEFEFEFEFEFEFCFC7F
:104D9000FCF8F0E0000000FFFFFFFFFFFFFFFFFF58
:104DA00003010103FFFFFFFFFFFFFFFFFF00000FF5
:104DB0003F7FFFFFFFFFFFFFF0E0E0F0FFFFFFFF9F
:104DC000FFFF7F3F0F00E0F8FCFEFEFFFFFFFF3F0D
:104DD0001F1F1F1F3FFFFFFFFFFEFEFCF8E0FFFF4E
:104DE000FFFFFFFFFFFFFF800000000080FFFFFFCD
:104DF000FFFFFFFFFFFF010F1F3F7F7F7FFFFFFFD1
:104E0000FFFFFFFFFFFFFF7F7F7F3F1F0F0100E0DE
:104E1000F8FCFCFCFEFEFEFEFEFEFEFEFEFEFEFCC0
:104E2000FCFCF8F0E000FFFFFFFFFFFFFFFFFF03C8
:104E300001010103FFFFFFFFFFFFFFFFFFFFFFFF78
:104E4000FFFFFFFFFFFFFFE0C0C0C0E0FFFFFFFF6D
:104E5000FFFFFFFFFFFF01071F1F3F3F3F3F3F3F98
:104E60003F1F1F07FFFFFFFFFFFFFFFFFFFFFCFCD0
:104E7000FCFCFCFCFCFCFC8000000080FFFFFFFF52
:104E8000FFFFFFFFFFFF071F7F7F7FFFFFFFFFFF8A
:104E9000FFFFFFFFFFFFFF7F7F7F3F3F1F03F2CF3B
:104EA0000EF0F29EB60FF66E4E0EF7220900F55088
:104EB0000EBEF28E120000000000000000008030E4
:104EC000209241ABA2B3C3BBE3BBE3BBE3BBE3BBF9
:104ED000C2B381B3418A80180000000000000000C6
:104EE00000000000406901FD66FE2EFFB2FFB3FF27
:104EF000B3FFD3FFB2FF6EFFC7FE81FD4272000019
:104F000000000000000000008018229B40C3C9FE82
:104F1000D4FFFBFFFDFFFDFFFCFFFBFFF6FF2AFFB9
:104F2000E3ECC089C0AAE1280000000000006593FE
:104F300045FE45FEC0D36FFFF6FFF9FFF9FFF8FF0E
:104F4000F6FF8FFF48FEA2AAC0D3E2FD229B00001D
:104F500000002108A7C46DFFB2FF48FE209266FE44
:104F60008AFE8AFEC9FE48FEC5FDA2AAA3C32CFF85
:104F70002AFFA7C4000000006010EAE5F5FFFAFF71
:104F80002FFFE0798061806180618061806140599C
:104F9000C0898BFEF6FFF1FFA8BC000000000000F6
:104FA0000000000000000000000000000000000001
:104FB00000000000000000000000000000000000F1
:104FC00000000000000000000000000000000000E1
:104FD00000000000000000000000000000000000D1
:104FE00000000000000000000000000000000000C1
:104FF00000000000000000000000000000000000B1
:10500000000000000000C089C0AAE12800000000E4
:105010000000200800000000000000000000000068
:1050200000000000000000000000A2AAC0D3E2FDC2
:10503000229B000000000008400840100000000013
:105040000000000000000000000000000000A2AA14
:10505000A3C32CFF2AFFA7C40000000020084010B3
:1050600040100000000000000000000000000000F0
:1050700000004059C0898BFEF6FFF1FFA8BC00007C
:105080000000000000008030209241ABA2B3C3BBFF
:10509000E3BBE3BBE3BBE3BBC2B381B3418A80188C
:1050A000000000000000000000000000406901FD59
:1050B00066FE2EFFB2FFB3FFB3FFD3FFB2FF6EFF5A
:1050C000C7FE81FD427200000000000000000000E9
:1050D0000000202000BBC9FED4FFFBFFFDFFFDFF49
:1050E000FCFFFBFFF6FF2AFFE3ECC089C0AAE12822
:1050F000000000000000200800088048C4E46FFFA2
:10510000F6FFF9FFF9FFF8FFF6FF8FFF48FEA2AAAE
:10511000C0D3E2FD229B00000000000840084010C0
:105120000010C058E3EC66FE8AFE8AFEC9FE48FE07
:10513000C5FDA2AAA3C32CFF2AFFA7C4000000003C
:1051400020084010401040104018C040806180612D
:105150008061806180614059C0898BFEF6FFF1FF5C
:10516000A8BC0000000000000000000000000000DB
:10517000000000000000000000000000000000002F
:10518000000000000000000000000000000000001F
:10519000000000000000000000000000000000000F
:1051A00000000000000000000000000000000000FF
:1051B000000000008018229B40C300000000000097
:1051C0000000000000000000000000000000C08996
:1051D000C0AAE128000000000000659345FE45FEDE
:1051E000C0D300000000000000000000000000002C
:1051F0000000A2AAC0D3E2FD229B0000000021080B
:10520000A7C46DFFB2FF48FE20920000000000001E
:10521000000000000000A2AAA3C32CFF2AFFA7C41D
:10522000000000006010EAE5F5FFFAFF2FFFE079CB
:10523000000000000000000000000000C0898BFE9C
:10524000F6FFF1FFA8BC0000000000000000803065
:10525000209241ABA2B3C3BBE3BBE3BBE3BBE3BB65
:10526000C2B381B3418A8018000000000000000032
:1052700000000000406901FD66FE2EFFB2FFB3FF93
:10528000B3FFD3FFB2FF6EFFC7FE81FD4272000085
:1052900000000000000000008018229B40C3C9FEEF
:1052A000D4FFFBFFFDFFFDFFFCFFFBFFF6FF2AFF26
:1052B000E3ECC089000000000000000000006593DE
:1052C00045FE45FEC0D36FFFF6FFF9FFF9FFF8FF7B
:1052D000F6FF8FFF48FEA2AA0000000000000000B9
:1052E00000002108A7C46DFFB2FF48FE209266FEB1
:1052F0008AFE8AFEC9FE48FEC5FDA2AA0000000083
:1053000000000000000000006010EAE5F5FFFAFF71
:105310002FFFE07980618061806180618061405908
:105320000000000000000000000000000000C12894
:105330008DEEF9FFFDFF11FF8071000000000000FD
:1053400000000000000862ABB3FFFBFFF4FF26B4CF
:10535000000000006239EEFEFAFFFCFFF0FE205173
:1053600000000000000000000000001824C4F6FF48
:10537000FCFFF3FFC79B00000000035A70FFFBFF18
:10538000FBFF6DF6A04000000000000000000000E0
:10539000202027DDF9FFFCFFF3FFE582000000007D
:1053A000646AB2FFFBFFFBFFC9ED40300000000064
:1053B0000000000000004030C9EDFBFFFBFFB2FF22
:1053C000646A0000000826B4F4FFFBFFB3FF62AB81
:1053D000000800000000000000000000807111FFC4
:1053E000FDFFF9FF8DEEC12800000008A8BCF1FF09
:1053F000F6FF8BFEC0898020000000000000000046
:105400000000E0792FFFFAFFF5FFEAE560100000E9
:105410000000A7C42AFF2CFF83BBA1AA60200008BC
:105420000000000000000000008A48FEB2FF6DFF8F
:10543000A7C4210800000000229BE2FDA0D3A0AA7F
:105440002000000000000000000000000000200814
:10545000C0D345FE45FE6593000000000000E12832
:10546000C0AAA0A220000000000000000000000070
:105470000000A1100000000040C3229B8018000023
:1054800000000000000000000000200040080000B4
:1054900000000000000000000000000862ABB3FF45
:1054A000FBFFF4FF26B40000000000000000000035
:1054B00000000000000000000000000000000000EC
:1054C000001824C4F6FFFCFFF3FFC79B0000000098
:1054D00000000000000000000000000000000000CC
:1054E000000000000000202027DDF9FFFCFFF3FF93
:1054F000E582000000000000000000000000000045
:105500000000000000000000000000004030C9ED75
:10551000FBFFFBFFB2FF646A000000000000000018
:10552000000000000000000000000000000000007B
:105530000000A0406DF6FBFFFBFF70FF035A000068
:105540000000000000000000000000000008000053
:105550000000000000000000E0792FFFFAFFF5FFD7
:10556000EAE56010000000000000000000000000FC
:105570000000000000000000201000008030209299
:1055800048FEB2FF6DFFA7C4210800000000000024
:1055900000000000000000002008000000002000C3
:1055A0000000A018801840BB45FE45FE6593000032
:1055B00000000000000000000000000000002000CB
:1055C0000000000000000000811061310031C0A225
:1055D000229B80180000000000004008401040108E
:1055E0004010400800000000000000000000000023
:1055F000000862ABB3FFFBFFF4FF26B4000000001D
:10560000200840104010401020080000000000005A
:10561000000000000000001824C4F6FFFCFFF3FFA8
:10562000C79B0000000040084010401040082000C8
:10563000000000000000000000000000202027DD26
:10564000F9FFFCFFF3FFE582000000004008401076
:105650004010400820000000000000000000000092
:1056600000004030C9EDFBFFFBFFB2FF646A0000A1
:105670000008201040104010201020000000000002
:105680000000000000000000807111FFFDFFF9FF25
:105690008DEEC1280000000820104010401020109E
:1056A0000008000000000000000000000000E07999
:1056B0002FFFFAFFF5FFEAE5601000000000200868
:1056C0004010401880382051205120512051205145
:1056D0002051E048209248FEB2FF6DFFA7C4210888
:1056E00000000000200820100051C4E48BFECDFE15
:1056F000EEFEF0FEEEFECDFE89FE44D4C0D345FEA4
:1057000045FE659300000000000000080059C4E455
:1057100071FFFAFFFCFFFDFFFDFFFDFFFBFFF5FF43
:10572000E9FEE2CB40C3229B80180000000000008D
:10573000C1288DEEF9FFFDFF11FF80710000000010
:10574000000000000000000862ABB3FFFBFFF4FFA5
:1057500026B4000000006239EEFEFAFFFCFFF0FE06
:10576000205100000000000000000000001824C4C8
:10577000F6FFFCFFF3FFC79B00000000035A70FF19
:10578000FBFFFBFF6DF6A0400000000000000000E2
:105790000000202027DDF9FFFCFFF3FFE582000079
:1057A0000000646AB2FFFBFFFBFFC9ED4030000060
:1057B00000000000000000004030C9EDFBFFFBFFCF
:1057C000B2FF646A0000000826B4F4FFFBFFB3FFD9
:1057D00062AB0008000000000000000000008071C3
:1057E00011FFFDFFF9FF8DEEC12800000008A8BCE5
:1057F000F1FFF6FF8BFEC089405900000000000059
:1058000000000000E0792FFFFAFFF5FFEAE56010E5
:1058100000000000A7C42AFF2CFF83BBA1AA2051CF
:105820002051205120512051E048209248FEB2FFE3
:105830006DFFA7C4210800000000229BE2FDA0D359
:10584000C0AA88EDCDFEEEFEF0FEEEFECDFE89FE96
:1058500044D4C0D345FE45FE65930000000000001F
:10586000E128C0AAA0A2AEF6FAFFFCFFFDFFFDFFF3
:10587000FDFFFBFFF5FFE9FEE2CB40C3229B801852
:10588000000000000000C1288DEEF9FFFDFF11FFB0
:105890008071000000000000000000000000000017
:1058A0000000000000000000000000006239EEFE71
:1058B000FAFFFCFFF0FE2051000000000000000095
:1058C00000000000000000000000000000000000D8
:1058D0000000035A70FFFBFFFBFF6DF6A0400000C5
:1058E00000000000000000000000000000000000B8
:1058F0000000000000000000C79BF3FFFCFFF6FF64
:1059000024C4001800000000000000000000000097
:10591000000000000000000000000000000826B4A5
:10592000F4FFFBFFB3FF62AB0008000000000000C3
:105930000000000000000000000000000000000067
:1059400000000008A8BCF1FFF6FF8BFEC08940599B
:105950000000000000000000000000000000000047
:1059600000000000000000000000A7C42AFF2CFF78
:1059700083BBA1AA20512051205120512051E04841
:1059800020510000000000000000000000000000A6
:10599000229BE2FDA0D3C0AA88EDCDFEEEFEF0FE74
:1059A000EEFECDFE89FE44D4C0D30000000000000E
:1059B000000000000000E128C0AAA0A2AEF6FAFF95
:1059C000FCFFFDFFFDFFFDFFFBFFF5FFE9FEE2CB66
:1059D00040C3229B801800000000001060400000BF
:1059E00000000000000000000000000000000000B7
:1059F00000000000000081C380710000000000086A
:105A0000807162E460CB0000000000000000000034
:105A10000000000000000000000044D445FEC0D398
:105A200020000000202802D4E8FE89FEE2CB00001E
:105A30000000000000000000000000000000E2CBB9
:105A40006EFF8FFF66ED20000000A04066EDF4FFC2
:105A5000F3FF89FEE079000000000000000040280C
:105A60006028229B2AFFF7FFF9FFC9ED20080000FC
:105A700000516DF6FCFFFAFF6EFF42724008000015
:105A8000000000000000000026B4F1FFFCFFFBFF57
:105A900048DD20080000406911FFFEFFFCFF6FFF9A
:105AA0004272200800000000000000000000A7C4AF
:105AB000F5FFFEFFFBFFA7C420080000E07973FF9D
:105AC000FEFFFBFFEEFEC159400800000000000091
:105AD0000000000048DDF8FFFEFFFAFF26B42008B2
:105AE000000064ABF8FFFEFFF9FFEAE5C0282000E4
:105AF00000000000000000000000EEFEFBFFFEFFC3
:105B000095FF418A2000000026B4FAFFFEFFF8FF4F
:105B100048DDC02820080000000000000000000050
:105B2000EEFEFBFFFEFF73FFE07920000000A7C43C
:105B3000FBFFFEFFF5FFA7C4A028400800000000FF
:105B40000000000000006FFFFCFFFEFF11FF406936
:105B50002000000048DDFBFFFCFFF1FF26B48020A1
:105B60002008000000000000000020086EFFFAFF7F
:105B7000FCFF6DF6005100000000000000106040C6
:105B800000BB66FEB7FFFFFFFFFFFFFFFFFFFFFF4A
:105B9000FEFFFAFF2AFF24ED81C3807100000000A0
:105BA0000008807162E460CB62E42FFFF8FFFAFF27
:105BB000FAFFFBFFFAFFF8FFD2FF48FE44D445FE90
:105BC000C0D320000000202802D4E8FE89FEE2CBEA
:105BD000E2CB27DD27DD48DD48DD48DD27DDC5D404
:105BE000E2CB6EFF8FFF66ED20000000A04066ED67
:105BF000F4FFF3FF89FEE0798030602840284028D8
:105C000040286028229B2AFFF7FFF9FFC9ED2008F2
:105C1000000000516DF6FCFFFAFF6EFF4272400873
:105C20000000000000000000000026B4F1FFFCFFAF
:105C3000FBFF48DD20080000406911FFFEFFFCFF6C
:105C40006FFF42722008000000000000000000000A
:105C5000A7C4F5FFFEFFFBFFA7C420080000E07902
:105C600073FFFEFFFBFFEEFEC1594008000000007D
:105C700000000000000048DDF8FFFEFFFAFF26B438
:105C80002008000064ABF8FFFEFFF9FFEAE5C0283A
:105C9000200000000000000000000000EEFEFBFFFE
:105CA000FEFF95FF418A2000000026B4FAFFFEFFA8
:105CB000F8FF48DDC02820080000000000000000B8
:105CC0000000EEFEFBFFFEFF73FFE0792000000006
:105CD000A7C4FBFFFEFFF5FFA7C4A02840080000F3
:105CE00000000000000000006FFFFCFFFEFF11FF3E
:105CF00040692000000048DDFBFFFCFFF1FF26B4F7
:105D000080202008000000000000000020086EFF36
:105D1000FAFFFCFF6DF600510000000000000000DB
:105D20000000000000000000000000000000000073
:105D30000000000000000000000081C3807100002E
:105D40000000000000000000000000000000000053
:105D5000000000000000000000000000000044D42B
:105D600045FEC0D32000000000000000000000003D
:105D70000000000000000000000000000000000023
:105D80000000E2CB6EFF8FFF66ED200000000000F8
:105D90000000000000000000000000000000000003
:105DA000000000006028229B2AFFF7FFF9FFC9EDE1
:105DB00020080000000000000000000000000000BB
:105DC00000000000000000000000000026B4F1FF09
:105DD000FCFFFBFF48DD2008000000000000000081
:105DE00000000000000000000000000000000000B3
:105DF0000000A7C4F5FFFEFFFBFFA7C420080000BA
:105E0000000000000000000000000000400800004A
:105E1000000000000000000048DDF8FFFEFFFAFF70
:105E200026B4200800000000000000000000000070
:105E30000000200000000000000000000000EEFE56
:105E4000FBFFFEFF95FF418A2000000000000000DC
:105E5000000000000000000020080000000000001A
:105E600000000000EEFEFBFFFEFF73FFE079200064
:105E700000000000000000000000000000004008DA
:105E8000000000000000000000006FFFFCFFFEFFAC
:105E900011FF406920000000000000000000000029
:105EA00000000000200800000000000000002008A2
:105EB0006EFFFAFFFCFF6DF60051000000000000CD
:105EC0000000604000BB66FEB7FFFFFFFFFFFFFF63
:105ED000FFFFFFFFFEFFFAFF2AFF24ED81C3807161
:105EE0000000000000000000000060CB62E42FFF13
:105EF000F8FFFAFFFAFFFBFFFAFFF8FFD2FF48FEB8
:105F000044D445FEC0D32000000000000000000083
:105F10000000E2CBE2CB27DD27DD48DD48DD48DDB0
:105F200027DDC5D4E2CB6EFF8FFF66ED20000000B9
:105F30000000000000000000000000008030602829
:105F40004028402840286028229B2AFFF7FFF9FFBD
:105F5000C9ED200800000000000000000000000063
:105F6000000040080000000000000000000026B40F
:105F7000F1FFFCFFFBFF48DD2008000000000000EF
:105F800000000000000000002008000000000000E9
:105F900000000000A7C4F5FFFEFFFBFFA7C4200818
:105FA00000000000000000000000000000004008A9
:105FB0000000000000000000000048DDF8FFFEFFC8
:105FC000FAFF26B4200800000000000000000000D6
:105FD0000000000040080000000000000000000079
:105FE000EAE5F9FFFEFFF8FF64AB200800000000BF
:105FF0000000000000000000000020080000000079
:10600000000000000000EEFEFBFFFEFF73FFE079E2
:106010002000000000000000000000000000000060
:106020004008000000000000000000006FFFFCFFBF
:10603000FEFF11FF4069200000000000000000008A
:106040000000000000002008000000000000000028
:1060500020086EFFFAFFFCFF6DF600510000000003
:1060600000000010604000BB66FEB7FFFFFFFFFFAF
:10607000FFFFFFFFFFFFFEFFFAFF2AFF24ED81C3B2
:106080008071000000000008807162E460CB62E46F
:106090002FFFF8FFFAFFFAFFFBFFFAFFF8FFD2FF2E
:1060A00048FE44D40000000020000000202802D454
:1060B000E8FE89FEE2CBE2CB27DD27DD48DD48DDC7
:1060C00048DD27DDC5D4E2CB000000000000200041
:1060D0000000A04066EDF4FFF3FF89FEE079803018
:1060E0006028402840284028602800000000000068
:1060F000000000002008000000516DF6FCFFFAFFD0
:106100006EFF427240080000000000000000000026
:1061100000000000000000000000200800004069AE
:1061200011FFFEFFFCFF6FFF42722008000000001D
:10613000000000000000000000000000000000005F
:1061400020080000E07973FFFEFFFBFFEEFEC1595F
:1061500040080000000000000000000000000000F7
:1061600000000000000020080000418A95FFFEFFAB
:10617000FBFFEEFE4141400800000000000000006F
:1061800000000000000000000000000020080000E7
:1061900026B4FAFFFEFFF8FF48DDC0282008000003
:1061A00000000000000000000000000000000000EF
:1061B000000020000000A7C4FBFFFEFFF5FFA7C4FE
:1061C000A0284008000000000000000000000000BF
:1061D00000000000000000002000000048DDFBFF80
:1061E000FCFFF1FF26B48020200800000000000022
:1061F0000000200800000000000000000000000077
:106200000000C9EDF9FFF7FF2AFF229BC040C04004
:10621000A038A038A038A038A03889FEF3FFF4FFDA
:1062200066EDA0400000000066ED8FFF6EFFE2CB40
:1062300081C3A7EDEAE50BEE0BEE0BEEC9ED66EDC3
:10624000E2CB89FEE8FE02D4202800000000C0D383
:1062500045FE44D481C3ECFEF5FFF9FFFBFFFBFFD5
:10626000FAFFF7FFD0FF89FE60CB62E4807100087F
:1062700000000000807181C3C0AAE6FDB2FFFAFFF2
:10628000FDFFFEFFFEFFFDFFFCFFF7FF6DFF24EDAE
:106290000039000000000000000000086038C0D392
:1062A00004FEEBFE70FFB2FFB3FFD4FFD3FFB2FFDB
:1062B0006FFFE8FE81FDE5820000000000000000A5
:1062C000000000080051809241AB62ABA3B3A3B3BE
:1062D000A3B3A3ABA3AB62AB229BA18AC1280000EE
:1062E00000000000000000000000000000000000AE
:1062F000000000000000000000000000A03889FE3F
:10630000F3FFF4FF66EDA040000000000000000075
:10631000000000000000000000000000000000007D
:1063200000000000E2CB89FEE8FE02D42028000035
:10633000000000000000000000000000000000005D
:1063400000000000000000000000000060CB62E4DC
:106350008071000800000000000000000000000044
:10636000000000000000000000000000000000002D
:10637000000000000000000000000000000000001D
:10638000000000000000000000000000000000000D
:1063900000000000000000000000000000000000FD
:1063A00000000000000000000000000000000000ED
:1063B00000000000000000000000000000000000DD
:1063C00000000000000000000000000000000000CD
:1063D00000000000C040C040A038A038A038A0385D
:1063E000A03889FEF3FFF4FF66EDA0400000000036
:1063F000000000000000000081C3A7EDEAE50BEEFD
:106400000BEE0BEEC9ED66EDE2CB89FEE8FE02D4A1
:1064100020280000000000000000000081C3ECFE06
:10642000F5FFF9FFFBFFFBFFFAFFF7FFD0FF89FE47
:1064300060CB62E4807100080000000000000000F2
:10644000C0AAE6FDB2FFFAFFFDFFFEFFFEFFFDFF63
:10645000FCFFF7FF6DFF24ED003900000000000095
:10646000000000006038C0D304FEEBFE70FFB2FFF6
:10647000B3FFD4FFD3FFB2FF6FFFE8FE81FDE582DB
:1064800000000000000000000000000800518092A1
:1064900041AB62ABA3B3A3B3A3B3A3ABA3AB62AB58
:1064A000229BA18AC1280000000000000000C9ED65
:1064B000F9FFF7FF2AFF229BC040C040A038A03858
:1064C000A038A038A0380000000000000000000044
:1064D0000000000066ED8FFF6EFFE2CB81C3A7EDE9
:1064E000EAE50BEE0BEE0BEEC9ED66ED62AB0000DC
:1064F00000000000000000000000C0D345FE44D4AE
:1065000081C3ECFEF5FFF9FFFBFFFBFFFAFFF7FF8E
:10651000D0FF89FE62AB0000000000080000000010
:10652000807181C3C0AAE6FDB2FFFAFFFDFFFEFF46
:10653000FEFFFDFFFCFFF7FF6DFF24ED62AB0000E7
:1065400000000000000000086038C0D304FEEBFE2D
:1065500070FFB2FFB3FFD4FFD3FFB2FF6FFFE8FEBF
:1065600081FDE5820000000000000000000000083E
:106570000051809241AB62ABA3B3A3B3A3B3A3AB6F
:10658000A3AB62AB229BA18AC128000000000000DF
:106590000000000000000000A03800000000000023
:1065A000C0AA226A0000000041BBECFEC0D3226AF0
:1065B000C0AAE6FDB2FFB2FFC0AAC0D3B2FFF7FF88
:1065C000F7FFC0D3C0AAECFEB2FFB2FFC0AA000022
:1065D00041BBECFE41BB226A00000000C0AA226A57
:1065E0000000000000000000A0380000F2CF0EF014
:1065F000F29E040FF66E660EF7220900F5500EBEED
:10660000F28E120000008010E0204031004A00525B
:10661000E049E0490052004A0052004A005200524C
:1066200000520052E049E02040080000400840D5F8
:1066300000EE40F640F620F620F660F620FE40F62A
:1066400060F640F620F620F620F620F640F601F639
:1066500060DDA0182000202920F660FE40FE60FECC
:1066600041FE61FE40FE60FE60FE61FE61FE60F67E
:1066700060FE60FE60FE20FE00EEC01800F84008DC
:10668000202940F660FE40FE80FE40FE80FE40FE77
:1066900040FE60FE40FE40FE60FE60FE41FE20F6D1
:1066A0002029200800F800F82008803900F620FE94
:1066B00040FE80FE40FE40FE60FE40FE40FE61FE69
:1066C00040FE20FE00F68039200000F800F800F8B7
:1066D00000F84008005220F660FE40FE40FE60FEDA
:1066E00080FE60F660FE40FE60FE20F60052200054
:1066F00000F800F800F800F800F800F800F8205260
:1067000040F620FE60FE40FE60FE40FE40FE80FE41
:1067100020EE0052400800F800F800F800F800F8F9
:1067200000F800F800F88010E0C4E0EDE0EDE1EDE5
:1067300000EEE0EDC0EDE0EDE049400800F800F8C3
:1067400000F800F800F800F800F800F800F800F889
:106750000000200820002000200020004008200029
:10676000000000F800F800F800F800F8F2CF0EF092
:10677000F29E840FF66E670EF7220900F5500EBEEA
:10678000F28E120000F800F800002008200000F847
:1067900000F800F800F800F800F800F8400880DD84
:1067A0000029400800F800F800F800F800F80000A0
:1067B000E02800F620EE8018200800F800F800F825
:1067C00000F8000000C540FE40FEE0E5A0184008CB
:1067D00000F800F800F8000080DD40FE60FE21FEB9
:1067E000C0DD8010202800F800F82000E0E540FE21
:1067F00040FE61FE41F6A0E56010801000F86008E0
:10680000E0ED60FE60F620FE60FE20FE00CDA018E8
:1068100000F88010E0F560FE60FE40FE40FE80FE65
:10682000E1ED801000F8C02001F640FE60FE60FE41
:1068300040FE40FE20CD400800F8E02820F660FE33
:1068400060FE40FE60FE60FE20CD200800F860394A
:1068500021FE60FE40FE40FE60FE60FE00C50000BE
:1068600000F8005200F660FE60FE60FE40FE40FE52
:106870000052000000F800C540FE40FE40FE60FEF1
:1068800060FE40FE8039000000F8A0DD60FE60FE82
:1068900040FE60FE60FE20FE60390000200880DDC2
:1068A00020FE60FE60FE40FE40FE20F60029000053
:1068B0006008A0E540FE60FE40FE40FE60FE40F63F
:1068C000E0280000801000F640FE40FE40FE60FE22
:1068D00060FEA0E580100000C02000F660FE40FED3
:1068E00061FE40FE40FEC0E560100000E02820F69A
:1068F00060FE41FE40FE40FE40FE80E54008000094
:10690000603920F640FE61FE60FE40FE40FEA0DDE4
:1069100020000000005240FE61FE40FE60FE40FE8E
:1069200041FEE0C400000000E0C440F640FE60FE0E
:1069300060FE60F680DD8010000000F8202900F67F
:1069400060FE41FE00F6808BE02000F800F800F8C1
:106950002008A0DD20F600EEC049A01800F800F8DD
:1069600000F800F800008010E0C42039E02000F8B2
:1069700000F800F800F800F8000000004008E028E7
:1069800000F800F800F800F800F800F8F2CF0EF078
:10699000F29EA40FF66E690EF7220900F5500EBEA6
:1069A000F28E120000F800F800F800F800F800F885
:1069B0002008C0208039000000F800F800F800F836
:1069C00000F820000029E0ED00EE202900F800F892
:1069D00000F800F82000E02000F660FE60FE80DD98
:1069E00000F800F800F84008801020EE60FE40FE3D
:1069F00020FE20F600F800F84008400880DD41FE47
:106A000060FE40FE60FE00F600F80000200840DD59
:106A100021FE60FE60FE40FE20FEC0E500F80000A2
:106A2000801801EE40FE80FE60FE61FE40FE80DDCB
:106A300000000000002920F660FE40FE60FE20FEFF
:106A400040FE60DD00000000803960F640FE60FE20
:106A500060FE40FE60FE00CD00000000205240FEBF
:106A600060FE61FE60FE40FE40F600520000000045
:106A700000CD60FE60FE40FE40FE40FE40F6202954
:106A80000000400880E540FE60FE40FE60FE60FEC3
:106A900020F6C02000008010A0E540FE60F640FE19
:106AA00060FE60F6E0F580180000A01800F660FEB9
:106AB00040FE60FE40FE60FE00F660100000E02830
:106AC00040F660FE60FE60FE40FE40FE00EE2008E4
:106AD0000000202920FE40FE60FE60FE40FE60FEB9
:106AE000A0E500000000005220FE40FE61FE80FE96
:106AF00040FE40FE00CD0000000000CD40FE20FE24
:106B000061FE60FE40FE40F600520000400820CDCD
:106B100040FE20FE60FE60F640FE20F620290000C8
:106B20006010E0ED60FE20FE60FE60FE40FE20F69C
:106B3000E02800008010E0E560FE40FE60FE80FE80
:106B400040FE20F6801000008018803900F660FEBC
:106B500060FE40FE60FE00EE6008000000F8E028E5
:106B6000803900EE40FE60FE00F6E049000000F8CB
:106B700000F800F8C0208039E0ED00EE80392000F8
:106B800000F800F800F800F800F860108018A0186D
:106B90000000000000F800F8F2CF0EF0F29EB00FF7
:106BA000F66E6B0EF7220900F5500EBEF28E120043
:106BB00000F800F800F800F8E0202031E028E02894
:106BC0002029E028E028E028E028E028E0208018BC
:106BD00000F800F800F800F800F800F800F8A01835
:106BE00020CD00EE20EE20F620F620EE21F620F655
:106BF00020F620EE20EE00CDE02800F800F800F8A6
:106C000000F800F8E02080DD40F620FE60FE40FE47
:106C100040FE61FE60FE40FE60FE60FE60FE40FEE3
:106C200020CDC02000F800F800F8E028A0DD40F6F4
:106C300040FE60F620FE40FE60FE40FE40FE60FE2C
:106C400060FE40FE80FE20FE40FE80E56010801861
:106C50000000606200F661FE60FE60FE40FE61FEC4
:106C600040FE60FE40FE60FE40FE61FE61F660FE9A
:106C700020FEE0ED8010000000F8A01880DD20F676
:106C800020FE60FE80FE60F660FE40FE60FE40FE7C
:106C900060FE60FE40FE60FE00EE0029400800F845
:106CA00000F800F8C02000CD20F660FE20FE60FE57
:106CB00040FE60FE20FE80FE20FE20FE20FEE0ED75
:106CC000C020200800F800F800F800F800F8401094
:106CD0002029A0E580E580E580E5A0E5C0DD80E530
:106CE000C0DDA0E500C50029200800F800F800F884
:106CF00000F800F800F800F86010400820082008AC
:106D000020082008200820084008200820008010C3
:106D100000F800F800F800F8F2CF0EF0F29E300F05
:106D2000F66E6D0EF7220900F5500EBEF28E1200BF
:106D300000F8000000000000E0208010A01800F81B
:106D400000F800F800F80000400880D520EEE0E5EB
:106D50008039C02000F800F800F80000603920F603
:106D600040FE40FE01EEC049401000F800F820004F
:106D7000205240F640FE40FE60FE20EE20316010C2
:106D800000F8200020CD60FE40FE60FE60FE40FE68
:106D9000E0EDC02000F84008C0DD60FE40FE60FE6F
:106DA00060FE40FE20F6E02800F8600800EE60FE7D
:106DB00040FE60FE60FE60FE00F6C02000F8600845
:106DC00000F640FE40FE40FE40FE40FE20F68010F1
:106DD00000F8801020F640FE61FE60FE40FE60FE7E
:106DE00000EE600800F8C02000F660FE61FE60FE64
:106DF00040FE60FEE0ED600800F8002920F640FE4D
:106E000040FE60FE40FE60FEC0DD400800F88039B4
:106E100020F640FE60FE40FE40FE40FE20CD2000F9
:106E200000F8205240FE40FE60FE40FE40FE20FE84
:106E30002052000000F860DD40FE40FE60FE60FE73
:106E400020FE40FE804100002008C0DD60FE40FEC4
:106E500060FE40FE40FE20F620290000200800EEE3
:106E600040FE40FE60FE40FE40FE20F6002900008D
:106E7000601000F660FE60FE60FE40FE60FE00F600
:106E8000C02000008018E0F540FE40FE60FE40FE9D
:106E900060FE20EE80100000E020E0F560FE60FE65
:106EA00060FE40FE40FE20F680100000202920F603
:106EB00060FE60FE61FE40FE60F6C0DD600800001E
:106EC000005260FE60FE40FE60FE61FE40FE00C5B6
:106ED0002008000060D540FE40FE80FE60F620FEE7
:106EE000E0ED8010400800F8E0ED40FE40FE60FE5E
:106EF00020FEE1EDA018200800F800F840D520FEA3
:106F000061FE20FE00EE8018401000F800F800F846
:106F1000E02000F640FE00EE0029400800F800F8EE
:106F200000F800F84008C0E500EE0029200800F84D
:106F300000F800F800F800F80000A018E020200891
:106F400000F800F800F800F800F800F8F2CF0EF0B2
:106F5000F29E640FF66E6F0EF7220900F5500EBE1A
:106F6000F28E120000F800F800F800F800F840086F
:106F70008010E02040080000000000F800F800F851
:106F800000F82008202900EE20EEA0DD801000008F
:106F900000F800F800F82008A04100F620FE60FE8E
:106FA00020FEC0EDA01800F800F88010E0C421F623
:106FB00040FE60FE60F661FE20F6801000F80000E2
:106FC000C02001EE60FE40FE40FE60FE61FE00F665
:106FD000600800F80000202940F660FE40FE60FED8
:106FE00060FE61FE00EE400800F80000A04120F6BF
:106FF00060FE40FE60FE40FE40FE00EE200000F815
:107000002000205A41FE40FE40FE40FE60FE60FE31
:10701000A0DD000000F8200020CD40FE60FE60FEF4
:1070200040FE40FE20FE205A000000F8400880DDAF
:1070300060FE80FE40FE40FE40FE21FE80390000E2
:1070400000F86008E0ED60FE60FE40FE60FE40FE7D
:1070500000F62029000000F8801020F640FE40FED7
:1070600061FE60FE60FE20F6C020000000F8A0185F
:1070700020EE40FE40FE61FE60FE60FE01F68018DC
:10708000000000F8C02020F660FE60FE40FE40FEDA
:1070900060FE00EE601000000000202920F640FE97
:1070A00060FE40FE40FE60FE00EE600800F800005A
:1070B000A04140FE60FE60FE40FE40FE40FEC0DD9E
:1070C000400800F80000405A40FE40FE60FE40FECE
:1070D00040FE60FE20CD200000F8000060DD60FE74
:1070E00040FE60FE40FE40FE40FE205A000000F8D8
:1070F0002000E1E540FE40FE60FE40FE40FE21FE35
:10710000A041000000F82008E0ED40FE60FE61F6BE
:1071100040FE60FE40F62029000000F8801000EEDE
:1071200060FE40FE61FE60FE40FE40F6C0200000B2
:1071300000F82000803900F660FE40FE60FE40FE50
:1071400040F6A018000000F800F82008205220F6B1
:1071500040FE80FE60FE20F68010000000F800F87F
:107160006008601000C520F640FE40FEC0ED6010D3
:1071700000F800F800F800F8A018801000C540F6EC
:1071800020FE00CD200800F800F800F800F800F814
:10719000601020082052E0E58018000000F800F898
:1071A00000F800F800F800F8400820006010000027
:1071B00000F800F800F800F800F800F800F800F80F
:1071C0000000000000F800F800F800F8F2CF0EF020
:1071D000F29EE40FF66E710EF7220900F5500EBE16
:1071E000F28E120000F800F800F800F800F84008ED
:1071F00040086010400840084008400840086010FF
:107200002008200000F800F800F800F800F800F866
:1072100000F800F800F820086031A0DDC0E580E546
:1072200080E5A0E5C0DD80E580E500C5A018200868
:1072300000F800F800F800F800F800F800F8401036
:10724000603920EE40FE20FE60FE41FE40FE20FE42
:1072500020FE60FE40FE00CD6008601000F800F8DF
:1072600000F800F800F84008603940F660FE40FE83
:1072700060FE60F640FE60FE60FE60FE60FE40FE66
:1072800020FE00CDA018801000F800F800F82008BB
:10729000002900EE60F640FE61FE60FE60FE40FEEA
:1072A00040FE40FE61F661FE61F620FE00FE00C574
:1072B0006010200800F82008002900EE41FE60FE62
:1072C00060FE61FE40FE60FE60FE40FE40FE40FE4D
:1072D00060FE80FE60FE20FE20F6806A40082000EE
:1072E000002900EE20FE60FE60FE40FE60FE40FED3
:1072F00060FE40FE60FE40FE40FE60FE60FE40FE1E
:1073000040FE40FE01EE80390000A01880D500EE5E
:10731000E0EDE0EDE0EDE0EDC0EDE0EDE0EDC0ED45
:10732000E0EDE0ED00E620EE00E6E0ED00EE80D5D9
:10733000E020000000002008400840084008400805
:1073400040084008400840084008400840084008FD
:107350004008400840084008200800000000F2CF24
:107360000EF0F29EF76A780FF66E730EF7220900A0
:10737000F5500EBEF28E12000008000800088010C2
:1073800040318039C0200000000800080031A06AA8
:10739000C0ED00EE20EEA0DD002900080008C04985
:1073A000C0E500F620FE60FE20FEA0E5007B200880
:1073B000E04920F640FE60FE60F661FE20F6806245
:1073C000C02001EE60FE40FE40FE60FE61FE00F661
:1073D0006062202940F660FE40FE60FE60FE61FEB5
:1073E00000EE6072A04120F660FE40FE60FE40FEAE
:1073F00040FE00EE2062205AA0E540FE40FE40FE26
:1074000060FE60FEA0DD00628039E07260FE60FE1A
:1074100040FE40FE20FE205A2031200820526062AB
:10742000208360B440AC00A4A0410008F2CF0EF06D
:10743000F29EF76A460FF66E740EF7220900F550B9
:107440000EBEF28E12004A616E00F2CF0EF0F29E76
:10745000F76A640FF66E740EF7220900F5500EBE3F
:10746000F28E120046657600F2CF0EF0F29EF76AB9
:10747000820FF66E740EF7220900F5500EBEF28EE2
:1074800012004D617200F2CF0EF0F29EF76AA00F6B
:10749000F66E740EF7220900F5500EBEF28E120041
:1074A00041767200F2CF0EF0F29EF76ABE0FF66ED2
:1074B000740EF7220900F5500EBEF28E12004D61D7
:1074C0006900F2CF0EF0F29EF76ADC0FF66E740ED2
:1074D000F7220900F5500EBEF28E12004A756E00BA
:1074E000F2CF0EF0F29EF76AFA0FF66E740EF722E4
:1074F0000900F5500EBEF28E12004A756900F2CFF7
:107500000EF0F29EF76A180FF66E750EF72209005C
:10751000F5500EBEF28E1200416F7500F2CF0EF0E4
:10752000F29EF76A360FF66E750EF7220900F550D7
:107530000EBEF28E120053657000F2CF0EF0F29E76
:10754000F76A540FF66E750EF7220900F5500EBE5D
:10755000F28E12004F637400F2CF0EF0F29EF76AC3
:10756000720FF66E750EF7220900F5500EBEF28E00
:1075700012004E6F7600F2CF0EF0F29EF76A900F77
:10758000F66E750EF7220900F5500EBEF28E12004F
:1075900044656300CE50216ECFCF22F03480F29448
:1075A00032EF00F00101C86BC851030829E3C8514C
:1075B000C325C96FC40EC825016E010E036ED8B075
:1075C000032A01C0E9FF03C0EAFFEFCFCAF1AA6AAC
:1075D000C9C1A9FFCAC1A8FFA69CA69EA684F2CFD6
:1075E00000F0F29E0F01550EA76EAA0EA76EA6829E
:1075F000A6B2FED7A6940050F2120101C82BD4D730
:107600000001000C0101E051E203F3CF01F0F4CFDF
:1076100000F0E303F3500026E151E203F3500020B1
:10762000026E0001000C929089900101E7BF02D028
:10763000899201D0898292929290898092908990C9
:10764000E7BD02D0899201D089829292929089807E
:1076500092908990E7BB02D0899201D08982929260
:107660009290898092908990E7B902D0899201D056
:10767000898292929290898092908990E7B702D005
:10768000899201D089829292929089809290899079
:10769000E7B502D0899201D0898292929290898036
:1076A00092908990E7B302D0899201D08982929218
:1076B0009290898092908990E7B102D0899201D00E
:1076C00089829292929089800001000C8990929018
:1076D000899492948992929289809290E6C1E7F17E
:1076E000A2DF8990929089849294000C8990929064
:1076F000899492948982929289809290E6C1E7F16E
:1077000092DF8990929089849294000C2A0E010154
:10771000E66F0001DBDFE2C1E6F1E8DFE3C1E6F19D
:10772000E5DF2B0E0101E66F0001D0DFE4C1E6F1D9
:10773000DDDFE5C1E6F1DADF000CDEC1E2F1DEC13A
:10774000E3F1DFC1E4F1DFC1E5F1E0DF2C0E01017F
:10775000E66F0001BBDFE1C1E2F10101E36BE1C1D2
:10776000E6F10001C3DFE0C1E6F1C0DF000CC6C1F5
:1077700003F00101C5C1E9FFC6C1EAFFEF52D8B469
:1077800000D1C6C103F0C5C1E9FFC6C1EAFFEF5091
:107790007E0837E3C6C103F0C5C1E9FFC6C1EAFFF1
:1077A000200EEF5CDF6FE16BE06FE36B100EE26FBA
:1077B000000128DF02C0E1F1010101C0E0F1010E8A
:1077C000EA6ECD0EE96E02C0E5F101C0E4F1F2CF40
:1077D000E2F1F29E026A100E016E022AE5C1F7FF85
:1077E000E45100016BEC21F00A000900EF6AF5CFCB
:1077F000EEFF012EFAD7022EF8D70101E2BFF28E7A
:107800001CD0010EEA6ECD0EE96EF2CFDDF1F29ED4
:10781000026A100E016E022AF76A000E00016BEC7C
:1078200021F00A000900EF6AF5CFEEFF012EFAD72A
:10783000022EF8D70101DDBFF28EC6C103F0C5C12B
:10784000E9FFC6C1EAFFEF500A0A000103E0070A98
:1078500006E008D00D0E0101C4278DD00001010102
:10786000C36B89D0080E0101C325830803E2C36BF3
:107870000D0EC427CB6BCB510708D8A07BD0CC6BA7
:10788000CC51070836E3036ACB51CD0FE96E010EE8
:107890000320EA6EEFCFDDF1DDC100F0CC51016EC7
:1078A00004E0D8900032012EFCD700A00ED0CC51BD
:1078B000C425DD6FC3C1DEF1DF6FC8C1E1F1C7C10F
:1078C000E0F100013ADF12D00101C95303E1CA51CE
:1078D00002080DE0CC51C425DD6FC3C1DEF1DF6FBE
:1078E000CAC1E1F1C9C1E0F1000127DF0101CC2BE0
:1078F000C7D7CC6BCC51030839E3080ECB25036AFC
:10790000CD0FE96E010E0320EA6EEFCFDEF1DEC18E
:1079100000F0CC51016E04E0D8900032012EFCD76B
:1079200000A00FD0080ECC25C425DD6FC3C1DEF149
:10793000DF6FC8C1E1F1C7C1E0F10001FEDE13D085
:107940000101C95303E1CA5102080EE0080ECC251B
:10795000C425DD6FC3C1DEF1DF6FCAC1E1F1C9C16A
:10796000E0F10001EADE0101CC2BC4D7CB51CB2BD7
:10797000C32B81D7C32BC52BD8B4C62B0001F7D698
:1079800001010001000C010EEA6EC30EE96EEF501A
:107990000DE00A0E016E006A002EFED7012EFBD705
:1079A0005F0E006E002EFED7EF2EF3D7000C220ED6
:1079B0000101E66F00018ADE280E0101E66F000179
:1079C00085DE020E0101E66F000180DE100E01016E
:1079D000E66F00017BDE000CA094060E0101C36F70
:1079E00045C0C7F144C0C6F143C0C5F142C0C4F1AF
:1079F0000001D8DD0A0E0101C36F49C0C7F148C0BC
:107A0000C6F147C0C5F146C0C4F10001CBDD030E8D
:107A10000101C36F010EC46FC66B990EC56FF80EDE
:107A2000C86FC76BCA6BC96B0001A1DE3486140E28
:107A30000101C26FC25308E00A0EC36F0001A3DF49
:107A400004000101C207F6D70001B1DF640E010195
:107A5000C26FC25308E0140EC36F000194DF04002C
:107A60000101C207F6D7A194000132EF00F0080E21
:107A7000016E00D08B96949600D0000001019037E3
:107A80008B98D8B09488D8A09498948682A6FED774
:107A9000012E01D002D00001ECD700D08B96949635
:107AA0000000948800D0000000D00000948682A6D8
:107AB000FED7016A00D0000082B801808B969496B0
:107AC0008B9894980001000C948800D0948600D084
:107AD00000008B98949800D08B969496D00E01015C
:107AE000906F0001C4DF89C190F1C1DF8AC190F1BC
:107AF000BEDF94980000948682A6FED700D000D006
:107B00000000948800D0000C070E0101896F400E20
:107B10008A6F0001D9DF080E0101896FAA0E8A6FF2
:107B20000001D2DFF6EF76F00D0E01019C6F949C00
:107B30008B9C949E8B9E93908A9093928A929D6B3D
:107B40009D51030844E304009D5302E1949C8B8CF7
:107B50009D2D02D0949E8B8E9D51020802E1939040
:107B60008A809D51030802E193928A82938881A8BA
:107B70000AD09D51030DF350010F9C6F938881A88B
:107B800002D00400FBD7938681A60AD09D51030D35
:107B9000F350020F9C6F938681A602D00400FBD79E
:107BA000938481A40AD09D51030DF350030F9C6F61
:107BB000938481A402D00400FBD7949C8B9C949E58
:107BC0008B9E93908A9093928A929D2BB9D79C51C9
:107BD0000B08D8B49C6B9CC101F00001000C0101A2
:107BE0009F6B9F51010829E39F519C25A06F9D0E1B
:107BF0009F25016E010E036ED8B0032A01C0E9FF74
:107C000003C0EAFFEFCFA1F1AA6AA0C1A9FFA1C1F9
:107C1000A8FFA69CA69EA684F2CF00F0F29E0F01BC
:107C2000550EA76EAA0EA76EA682A6B2FED7A69480
:107C30000050F21201019F2BD4D70001000C89944F
:107C40009294186AF2BE188EF29E250E0101E66F1C
:107C500000013CDD18BEF28E186AF2BE188EF29E4C
:107C60006FC1E6F143DD18BEF28E89849294000C58
:107C7000186AF2BE188EF29E280E0101E66F00010E
:107C800025DD18BEF28E420E0101566F860E556F2D
:107C9000186AF2BE188EF29E010EE26F830EE36F39
:107CA000010EE46F820EE56F000130DD18BEF28E2A
:107CB000186AF2BE188EF29E2C0E0101E66F0001CA
:107CC00005DD18BEF28E56C154F155C153F10101C4
:107CD000535302E154531CE052C157F1586B186AD8
:107CE000F2BE188EF29E52C1E6F10001FFDC18BE12
:107CF000F28E186AF2BE188EF29E51C1E6F1F6DCE1
:107D000018BEF28E01015351D8B454075307E0D77F
:107D1000186AF2BE188EF29E290EE66F0001D6DCBC
:107D200018BEF28E000C186AF2BE188EF29E410E3A
:107D30000101C36F000127DE18BEF28E8994929470
:107D400089969296186AF2BE188EF29E0A0E01016A
:107D5000C36F000118DE18BEF28E89869296898064
:107D600092908982929289849294186AF2BE188EB7
:107D7000F29E010E0101E66F0001A8DC18BEF28E32
:107D8000186AF2BE188EF29E110E0101E66F000114
:107D90009DDC18BEF28E186AF2BE188EF29E030E9B
:107DA0000101E66F000192DC18BEF28E186AF2BE85
:107DB000188EF29E3A0E0101E66F000187DC18BEB4
:107DC000F28E186AF2BE188EF29E050E0101E66F61
:107DD00000018CDC18BEF28E186AF2BE188EF29E7C
:107DE000360E0101E66F000171DC18BEF28E186AD2
:107DF000F2BE188EF29E0101E66B000177DC18BE20
:107E0000F28EE3C06FF11BDF0101526B516B000179
:107E10002FDF186AF2BE188EF29E290E0101E66F5E
:107E2000000154DC18BEF28E000CE96B400EE86FC6
:107E3000EB6BEA6F010EE85DF46F000EE959F56F28
:107E4000E351F425F66F000EF521F76F010EEA5DA0
:107E5000F86F000EEB59F96FE451F825FA6F000E38
:107E6000F921FB6F186AF2BE188EF29EE3C0E2F1B0
:107E7000F6C0E3F1E4C0E4F1FAC0E5F147DC18BE76
:107E8000F28E186AF2BE188EF29EE9C0E1F1E8C0E7
:107E9000E0F1EBC0E3F1EAC0E2F102EC3BF018BE26
:107EA000F28E02C0F3F001C0F2F0186AF2BE188E32
:107EB000F29E2C0E0101E66F000108DC18BEF28E66
:107EC000EF6BEE6BEF53D8A4AAD0E551EE5DD8B0BE
:107ED000A6D0ED6B020EEC6F020EF225016E000EC5
:107EE000F321036EED51035CD8A07DD003E1015076
:107EF000EC5D79E2186AF2BE188EF29EEFC0E1F1F5
:107F0000EEC0E0F1F3C0E3F1F2C0E2F102EC3BF0CD
:107F100018BEF28E02C0F5F001C0F4F0EC5101245D
:107F2000F66FED510220F76FD890F635026EF735F7
:107F3000036E0250F2CFF8F0F29E03C0F7FF55EC4B
:107F400000F00900F5CF03F0F8BFF28EF96F03C01F
:107F5000FAF003C0FBF0FC6B186AF2BE188EF29EBA
:107F600003C0E6F176EC3BF018BEF28E186AF2BE62
:107F7000188EF29EEFC0E1F1EEC0E0F1F3C0E3F144
:107F8000F2C0E2F102EC3BF018BEF28E02C0F5F056
:107F900001C0F4F0EC510124F66FED510220F76FAF
:107FA000D890F635026EF735036E0250F2CFF8F036
:107FB000F29E03C0F7FF55EC00F00900F5CF03F087
:107FC000F8BFF28EF96F03C0FAF0186AF2BE188E8D
:107FD000F29EE8CFE6F176EC3BF018BEF28EEC2B89
:107FE000D8B4ED2B79D7E7C0F1F0E6C0F0F0F0534C
:107FF00002E1F15310E0186AF2BE188EF29E010EF3
:108000000101C36F0001BFDC18BEF28EF051D8B47D
:10801000F107F007ECD7EE2BD8B4EF2B53D7000CB9
:10802000186AF2BE188EF29E99C1E2F19BC1E3F18B
:108030009AC1E4F19CC1E5F186EC3BF018BEF28EEA
:10804000010199519B5DA86BA76FA8C103F0A751CF
:10805000A8AF08D0000ED880A755006E000EA85516
:10806000036E0050A86F010EA8259F6F000E03201D
:10807000A06F9A519C5DA86BA76FA8C103F0A75190
:10808000A8AF08D0000ED880A755006E000EA855E6
:10809000036E0050A86F010EA825A16F000E0320EB
:1080A000A26F186AF2BE188EF29EA0C1E1F19FC1C4
:1080B000E0F1A2C1E3F1A1C1E2F1000102EC3BF069
:1080C00018BEF28E02C0A6F101C0A5F1186AF2BE78
:1080D000188EF29E2C0E0101E66F000166EC3BF05B
:1080E00018BEF28EA6C1A4F1A5C1A3F10101A3534C
:1080F00002E1A4531EE09EC1A7F1A86B186AF2BE6C
:10810000188EF29E9EC1E6F1000176EC3BF018BE9F
:10811000F28E186AF2BE188EF29E9DC1E6F176ECE0
:108120003BF018BEF28E0101A351D8B4A407A307F7
:10813000DED70001000C010199519B5DB06FB05179
:10814000B0AF03D0000ED880B055036AE8BE030676
:10815000A76F03C0A8F19A519C5DB06FB051B0AF4A
:1081600003D0000ED880B055036AE8BE0306A96F9D
:1081700003C0AAF199C1A0F19AC1A1F1A71DB06FE6
:10818000A81DB16FB02BD8B4B12B186AF2BE188EEF
:10819000F29EB1C1E1F1B0C1E0F1E36B99C1E2F14E
:1081A000000102EC3BF018BEF28E02C0B2F101C039
:1081B000B1F1186AF2BE188EF29EAAC1E1F1A9C10E
:1081C000E0F10101E36B9AC1E2F1000102EC3BF046
:1081D00018BEF28E01500101B15DAB6F0250B25971
:1081E000AC6FA71DB06FA81DB16FB02BD8B4B12B69
:1081F000186AF2BE188EF29EB1C1E1F1B0C1E0F191
:10820000E36B9BC1E2F1000102EC3BF018BEF28E81
:1082100002C0B2F101C0B1F1186AF2BE188EF29E2E
:10822000AAC1E1F1A9C1E0F10101E36B9CC1E2F156
:10823000000102EC3BF018BEF28E01500101B15D6D
:10824000AD6F0250B259AE6F99519B5D69E2FF0E5E
:10825000A26FA71DB06FA81DB16FB02BD8B4B12B02
:10826000186AF2BE188EF29EB1C1E1F1B0C1E0F120
:10827000E36B9BC1E2F1000102EC3BF018BEF28E11
:1082800002C0B2F101C0B1F1186AF2BE188EF29EBE
:10829000AAC1E1F1A9C1E0F10101E36B9CC1E2F1E6
:1082A000000102EC3BF018BEF28E01500101B15DFD
:1082B000AB6F0250B259AC6FA71DB06FA81DB16F64
:1082C000B02BD8B4B12B186AF2BE188EF29EB1C191
:1082D000E1F1B0C1E0F1E36B99C1E2F1000102EC20
:1082E0003BF018BEF28E02C0B2F101C0B1F1186AC3
:1082F000F2BE188EF29EAAC1E1F1A9C1E0F101011E
:10830000E36B9AC1E2F1000102EC3BF018BEF28E81
:1083100001500101B15DAD6F0250B259AE6F02D094
:10832000010EA26F9A519C5D69E2FF0EA36FA71D1B
:10833000B06FA81DB16FB02BD8B4B12B186AF2BEC4
:10834000188EF29EB1C1E1F1B0C1E0F1E36B9BC1C7
:10835000E2F1000102EC3BF018BEF28E02C0B2F175
:1083600001C0B1F1186AF2BE188EF29EAAC1E1F105
:10837000A9C1E0F10101E36B9CC1E2F1000102EC53
:108380003BF018BEF28E01500101B15DAB6F02509F
:10839000B259AC6FA71DB06FA81DB16FB02BD8B488
:1083A000B12B186AF2BE188EF29EB1C1E1F1B0C1D4
:1083B000E0F1E36B99C1E2F1000102EC3BF018BE81
:1083C000F28E02C0B2F101C0B1F1186AF2BE188E8D
:1083D000F29EAAC1E1F1A9C1E0F10101E36B9AC1EA
:1083E000E2F1000102EC3BF018BEF28E01500101F7
:1083F000B15DAD6F0250B259AE6F02D0010EA36FE6
:10840000AAAF03D0A8AF0CD002D0A8BF3AD1AA51CE
:10841000A85DD8A036D104E1A951A75DD8A031D17B
:10842000186AF2BE188EF29EE16B020EE06FAAC1CE
:10843000E3F1A9C1E2F1000102EC3BF018BEF28EBB
:108440000101A751015CA56FA8510258A66FAF6B3F
:10845000AFAF03D0A8AF09D002D0A8BF11D1A853A5
:1084600004E1AF51A75DD8A00BD1D8909D31FF0A90
:10847000010FA46FD8909D31B06F9D51010BB025B5
:10848000A4BF03D0A45DD8B0AAD0036AA051006EE7
:10849000E8BE0306B06F03C0B1F1186AF2BE188ED1
:1084A000F29EA8C1E1F1A7C1E0F103C0E3F1E26FE0
:1084B000000102EC3BF018BEF28E02C0B2F101C026
:1084C000B1F10101A451A125036A006EE8BE0306C3
:1084D000B36F03C0B4F1186AF2BE188EF29EAAC13F
:1084E000E1F1A9C1E0F103C0E3F1E26F000102ECA8
:1084F0003BF018BEF28E02C003F001500101B1251D
:10850000B46F0250B221B56FAB51B425B66FAC5108
:10851000B521B76FE8BE61D000D0036AA051006EEC
:10852000E8BE0306B86F03C0B9F1186AF2BE188E30
:10853000F29EA8C1E1F1A7C1E0F103C0E3F1E26F4F
:10854000000102EC3BF018BEF28E02C0BAF101C08D
:10855000B9F10101A451A125036A006EE8BE03062A
:10856000BB6F03C0BCF1186AF2BE188EF29EAAC19E
:10857000E1F1A9C1E0F103C0E3F1E26F000102EC17
:108580003BF018BEF28E02C003F001500101B92584
:10859000BC6F0250BA21BD6FAD51BC25BE6FAE514C
:1085A000BD21BF6FE8BE05D0BF5317E1BE51000823
:1085B00014E3A451A125B06F186AF2BE188EF29E82
:1085C000A0C1DEF1DF6F9FC1E1F19EC1E0F10001CA
:1085D0009DEC3BF018BEF28E0101A42B4BD7A6BF39
:1085E00001D018D0186AF2BE188EF29EE16B020E0E
:1085F000E06FAAC1E3F1A9C1E2F1000102EC3BF096
:1086000018BEF28E01500101A5270250A623A251E7
:10861000A02734D0186AF2BE188EF29EE16B020ECB
:10862000E06FAAC1E3F1A9C1E2F1000102EC3BF065
:1086300018BEF28E02C0B1F101C0B0F1186AF2BEEC
:10864000188EF29E0101E16B020EE06FA8C1E3F10A
:10865000A7C1E2F1000102EC3BF018BEF28E01501E
:108660000101B05D006E0250B159036E0050A527A4
:108670000350A623A251A027A351A127AF2BE8D6D0
:1086800030D1186AF2BE188EF29EE16B020EE06FD6
:10869000A8C1E3F1A7C1E2F1000102EC3BF018BE72
:1086A000F28E0101A951015CA56FAA510258A66F73
:1086B000AF6BAFAF03D0AAAF09D002D0AABF11D120
:1086C000AA5304E1AF51A95DD8A00BD1A6BF01D038
:1086D00018D0186AF2BE188EF29EE16B020EE06F9F
:1086E000A8C1E3F1A7C1E2F1000102EC3BF018BE22
:1086F000F28E01500101A5270250A623A351A12704
:1087000034D0186AF2BE188EF29EE16B020EE06F52
:10871000A8C1E3F1A7C1E2F1000102EC3BF018BEF1
:10872000F28E02C0B1F101C0B0F1186AF2BE188E2B
:10873000F29E0101E16B020EE06FAAC1E3F1A9C153
:10874000E2F1000102EC3BF018BEF28E0150010193
:10875000B05D006E0250B159036E0050A527035062
:10876000A623A251A027A351A127D8909D31FF0A8B
:10877000010FA46FD8909D31B06F9D51010BB025B2
:10878000A4BF03D0A45DD8B0AAD0036AA051006EE4
:10879000E8BE0306B06F03C0B1F1186AF2BE188ECE
:1087A000F29EA8C1E1F1A7C1E0F103C0E3F1E26FDD
:1087B000000102EC3BF018BEF28E02C0B2F101C023
:1087C000B1F10101A451A125036A006EE8BE0306C0
:1087D000B36F03C0B4F1186AF2BE188EF29EAAC13C
:1087E000E1F1A9C1E0F103C0E3F1E26F000102ECA5
:1087F0003BF018BEF28E02C003F001500101B1251A
:10880000B46F0250B221B56FAB51B425B66FAC5105
:10881000B521B76FE8BE61D000D0036AA051006EE9
:10882000E8BE0306B86F03C0B9F1186AF2BE188E2D
:10883000F29EA8C1E1F1A7C1E0F103C0E3F1E26F4C
:10884000000102EC3BF018BEF28E02C0BAF101C08A
:10885000B9F10101A451A125036A006EE8BE030627
:10886000BB6F03C0BCF1186AF2BE188EF29EAAC19B
:10887000E1F1A9C1E0F103C0E3F1E26F000102EC14
:108880003BF018BEF28E02C003F001500101B92581
:10889000BC6F0250BA21BD6FAD51BC25BE6FAE5149
:1088A000BD21BF6FE8BE05D0BF5317E1BE51000820
:1088B00014E3A451A025B06F186AF2BE188EF29E80
:1088C000DE6FA1C1DFF19FC1E1F19EC1E0F10001C6
:1088D0009DEC3BF018BEF28E0101A42B4BD7AF2BC1
:1088E000E8D60001000C010199519B5DB06BAF6FA0
:1088F000B0C103F0AF51B0AF08D0000ED880AF5573
:10890000006E000EB055036E0050A76F03C0A8F1B3
:108910009A519C5DB06BAF6FB0C103F0AF51B0AF77
:1089200008D0000ED880AF55006E000EB055036E13
:108930000050A96F03C0AAF1036A99C19FF103C057
:10894000A0F1036A9AC1A1F103C0A2F199519B5D04
:1089500004E2FF0EA46FA36F03D0A46B010EA36FFC
:108960009A519C5D04E2FF0EA66FA56F03D0A66B23
:10897000010EA56FAAAF03D0A8AF0CD002D0A8BF3C
:108980009CD0AA51A85DD8A098D004E1A951A75DB8
:10899000D8A093D0186AF2BE188EF29EE16B020E38
:1089A000E06FAAC1E3F1A9C1E2F1000102EC3BF0E2
:1089B00018BEF28E0101A751015CAB6FA85102589D
:1089C000AC6FAE6BAD6BAEAF03D0A8AF0AD002D028
:1089D000A8BF72D0AE51A85D6FE303E1AD51A75DB2
:1089E0006BE3186AF2BE188EF29E9FC1DEF1A1C140
:1089F000DFF19EC1E1F19DC1E0F100019DEC3BF092
:108A000018BEF28E0101ACBF01D01AD0186AF2BEB6
:108A1000188EF29EE16B020EE06FAAC1E3F1A9C1CC
:108A2000E2F1000102EC3BF018BEF28E01500101B0
:108A3000AB270250AC23A3519F27A451A02338D0C9
:108A4000186AF2BE188EF29EE16B020EE06FAAC1A8
:108A5000E3F1A9C1E2F1000102EC3BF018BEF28E95
:108A600002C0B0F101C0AFF1186AF2BE188EF29EDA
:108A70000101E16B020EE06FA8C1E3F1A7C1E2F1D1
:108A8000000102EC3BF018BEF28E01500101AF5D17
:108A9000006E0250B059036E0050AB270350AC2358
:108AA000A3519F27A451A023A551A127A651A223DA
:108AB000AD2BD8B4AE2B87D792D0186AF2BE188EE1
:108AC000F29EE16B020EE06FA8C1E3F1A7C1E2F1F3
:108AD000000102EC3BF018BEF28E0101A951015CCD
:108AE000AB6FAA510258AC6FAE6BAD6BAEAF03D09B
:108AF000AAAF0AD002D0AABF72D0AE51AA5D6FE36E
:108B000003E1AD51A95D6BE3186AF2BE188EF29EC7
:108B10009FC1DEF1A1C1DFF19EC1E1F19DC1E0F194
:108B200000019DEC3BF018BEF28E0101ACBF01D0FC
:108B30001AD0186AF2BE188EF29EE16B020EE06F38
:108B4000A8C1E3F1A7C1E2F1000102EC3BF018BEBD
:108B5000F28E01500101AB270250AC23A551A12791
:108B6000A651A22338D0186AF2BE188EF29EE16B8D
:108B7000020EE06FA8C1E3F1A7C1E2F1000102EC2F
:108B80003BF018BEF28E02C0B0F101C0AFF1186A1E
:108B9000F2BE188EF29E0101E16B020EE06FAAC1D7
:108BA000E3F1A9C1E2F1000102EC3BF018BEF28E44
:108BB00001500101AF5D006E0250B059036E0050CC
:108BC000AB270350AC23A3519F27A451A023A55149
:108BD000A127A651A223AD2BD8B4AE2B87D7000175
:108BE000000C010194531DE09251905D05E290C18B
:108BF00097F192C198F104D092C197F190C198F188
:108C00008FC199F197C19AF191C19BF198C19CF1E3
:108C100096C19EF195C19DF1000110EC40F07BD012
:108C20000101935343E08FC199F190C19AF191C131
:108C30009BF190C19CF193C19DF196C19FF195C1AB
:108C40009EF100019BEC40F08FC199F192C19AF125
:108C500091C19BF192C19CF193C19DF196C19FF18D
:108C600095C19EF19BEC40F08FC199F190C19AF1B2
:108C70008FC19BF192C19CF193C19DF196C19FF16F
:108C800095C19EF19BEC40F091C199F190C19AF190
:108C900091C19BF192C19CF193C19DF196C19FF14D
:108CA00095C19EF19BEC40F036D001018FC199F146
:108CB00090C19AF191C19BF190C19CF196C19EF136
:108CC00095C19DF100010FDE8FC199F192C19AF11A
:108CD00091C19BF192C19CF196C19EF195C19DF10C
:108CE00002DE8FC199F190C19AF18FC19BF192C1BF
:108CF0009CF196C19EF195C19DF1F5DD91C199F16F
:108D000090C19AF191C19BF192C19CF196C19EF1E3
:108D100095C19DF1E8DD000CFF0EE46FE36FE4C048
:108D200003F0E351D8B4E407E307031006E0D2AA46
:108D300003D0010E016E03D0F2D7000E016EA3EF37
:108D400078F0E46BE451010818E3E50EE425036ACA
:108D5000D8B0032AE96E03C0EAFFE451E325F2CF5D
:108D6000EAF0F29EAA6AA96EA69CA69EA680A850CA
:108D7000EABFF28EEF6EE42BE5D7E5C001F0E6C066
:108D800002F0ACEF78F0E46BE451030818E3E50E71
:108D9000E425036AD8B0032AE96E03C0EAFFE45170
:108DA000E325F2CFECF0F29EAA6AA96EA69CA69EDD
:108DB000A680A850ECBFF28EEF6EE42BE5D7E5C09D
:108DC00000F0E6C001F0E7C002F0E8C003F0000CDC
:108DD000E3532EE0FF0E776E766E796A786A6F6ADB
:108DE0006E6A716A706A736A726A756A746A020E70
:108DF0007B6EE00E7A6E010E856FE00E846FA50E1D
:108E00007F6E100E7E6E7F0E7D6EEF0E7C6E070EF7
:108E1000816FE00E806F7F0E836FEF0E826FFF0E0B
:108E2000876FE00E866F7F0E896FEF0E886F35D0EB
:108E3000776A766AFF0E796E786ED30E6F6EC00E0B
:108E40006E6EFF0E716EE00E706E070E736EE00EAA
:108E5000726E070E756EFF0E746E020E7B6EE00E64
:108E60007A6E010E856FE00E846FA50E7F6E100E78
:108E70007E6E7F0E7D6EEF0E7C6E070E816FE00EB4
:108E8000806F7F0E836FEF0E826FFF0E876FE00E95
:108E9000866F7F0E896FEF0E886F000C01019B6B50
:108EA0009C6B010E9D6FDA6AD96AA06F930E9F6F5B
:108EB000010EEA6E970EE96EA0C1E2FF9FC1E1FFCD
:108EC0009DC19EF1D890E550EE02F3509B23F450E3
:108ED0009C239E2FF7D79BC1DEFF9CC19BF19C6B0F
:108EE000D8B09C2B9F2BD8B4A02B9D2B9D5105084F
:108EF000DFE10001000CCE501B6ECFCF1CF01C50E8
:108F00001E5C14E303E11D501B5C10E2FF0ED880D1
:108F10001D5401018B6F000E1E548C6F1B508B254E
:108F20001F6E1C508C21206E08D000011D501B5C50
:108F30001F6E1E501C58206E01011CC01EF01BC06D
:108F40001DF01F502126205022228E6B8D6B20C0D9
:108F50008CF11FC08BF162C000F063C001F0026AA7
:108F6000036A03C092F102C091F163C090F162C044
:108F70008FF18EC196F18DC195F120C094F11FC083
:108F800093F103C09AF102C099F163C098F162C0F5
:108F900097F1000183DF03C038F002C037F001C051
:108FA00036F000C035F035C000F036C001F037C0F3
:108FB00002F038C003F0000C01018A5142268B51A7
:108FC00043228C5144228D5145224550040812E21F
:108FD000FF0A08E14450F4080DE2FF0A03E14350A0
:108FE000E00808E2FF0E425EE00E435AF50E445AD6
:108FF000050E455A0001000C01018B5146268C518B
:1090000047228D5148228E51492249520DE1485044
:10901000970812E2FF0A08E1475095080DE2FF0A9F
:1090200003E146507F0808E27F0E465E960E475ADF
:10903000980E485A000E495A0001000CB60E006EF8
:10904000036A026A016AF551F611F711F81102E19B
:10905000006A0DD0D89001BE09D0F537F637F73742
:10906000F837033602360136002EF4D7019E26EF7C
:109070004DF001010D51D8B471D0006E1151D8B42A
:109080006DD0002604E3810E002668E204D07F0E36
:10909000005E64E363E00EC115F11251151B0E8FE3
:1090A000128F10511403F4CF17F10F511303F4CFA3
:1090B00003F0F3CF16F11403F3501727F4501623DF
:1090C000000E032210511303F3501727F4501623F8
:1090D000000E026A032202220E511403F3501627D7
:1090E000F4500322000E02220E511303F350032604
:1090F000F4500222000E016A012210511203F350B3
:109100001627F4500322000E022201220F511203EF
:10911000F3500326F4500222000E01220E511203D6
:10912000F3500226F4500122002A01BE05D0163762
:109130000336023601360006000E16AF0AD0032AA7
:1091400002220122015005E1025003E1035001E136
:10915000002A15BF018E15AF019E04D0006A016A76
:10916000026A036A0001000C01010951D8B4A5D0BC
:10917000156F0D51D8B4A1D0155F05E37F0E1527EB
:10918000D8B09BD006D0810E155FD8A096D0D8B4A9
:1091900094D015C100F0016A026A036A146B0AC117
:1091A00013F1138F0BC112F10CC111F1190E156FD0
:1091B0001051115F0DE2010E125F0AE2135F08E227
:1091C000145F06E2142B132B122B1051112728D0F9
:1091D0000F51125F12E2010E135F0FE2145F0DE2F6
:1091E000142B132B0F5112271051112719E3122B97
:1091F00017E1132B15E1142B13D00E518009135FC7
:109200000EE2010E145F0BE2142B0E51800913279E
:109210000F511227E9E3132BE7E1142BE5D7038065
:10922000152F01D00BD0D8901137123713371437C0
:10923000D8900336023601361637BAD716A106D0B3
:10924000D890013202320332163302D0000635E0E4
:1092500016BF1ED0D890113712371337143710515C
:10926000115F07E2010E125F04E2135F02E2145F76
:109270001AE30F51125F05E2010E135F02E2145F61
:1092800012E30E518009135F03E2010E145F0BE33A
:10929000032A09E1022A07E1012A05E1002A0DE07B
:1092A0000132023203320AC115F10E51151B15AFFE
:1092B00002D0018E06D0019E04D0006A016A026AC3
:1092C000036A0001000C0AC111F101010E51111BCA
:1092D00011AF05D0D894D8900ABFD8802FD00AC13A
:1092E00011F10DC112F10951125F06E011AF26D044
:1092F000D850010AD86E22D00EC112F10A51125F65
:1093000006E011AF1BD0D850010AD86E17D00FC19C
:1093100012F10B51125F06E011AF10D0D850010AC4
:10932000D86E0CD010C112F10C51125F06E011AFD3
:1093300005D0D850010AD86E01D0D8900001000C99
:109340008E0E006E01010951005E0AC102F00BC1D0
:1093500001F0028E005209E0D890025202E101525F
:1093600004E002320132002EF7D70AAF05D0011E09
:10937000021E012AD8B4022A0001000C8E0E006ED3
:109380000EC101F00DC102F0036A015209E102C0F1
:1093900001F0026A080E005E015202E1006A08D084
:1093A000D89001BE04D0023601360006F9D7019EDE
:1093B000000C800ED8A202D00101121B0101176B14
:1093C000186B0EC116F11251161B0D51D8B4DFD017
:1093D000156F006E1151D8B4E3D0155FD8B483D0A7
:1093E0003EE312C11BF11B8F13C11AF114C119F115
:1093F000186BD8901B331A3319331833152FF8D73D
:1094000016AF03D01781E0D0179115911789010E7F
:10941000EA6E100EE96EEBD0179916BF0AD015A1AF
:1094200013D01B331A3319331833002AD8B4C7D0DA
:109430000BD01BBF0CD0D890183719371A371B37F1
:109440000006D8B4BCD0F5D7178D6DD0179D0EC1CE
:1094500016F10EAF02D01B8FABD01B9FA9D011C14C
:1094600015F111C100F00D51155F0EC11BF11B8FDD
:109470000FC11AF110C119F1186BD8901B331A33B0
:1094800019331833152FF8D716AF03D017839CD094
:1094900017931591178B010EEA6E140EE96EA7D083
:1094A000179B16BF0AD015A113D01B331A331933DB
:1094B0001833002AD8B483D00BD01BBF0CD0D8905F
:1094C000183719371A371B370006D8B478D0F5D7B4
:1094D000178F29D0179F12C116F112AF02D01B8F20
:1094E00067D01B9F65D012C11BF11B8F13C11AF1EE
:1094F00014C119F116AF04D01B9F178565D01795BD
:10950000186B1591010EEA6E100EE96E70D016BF41
:109510001CD00EC116F115A106D01B331A33193316
:109520001833002A4CE018AF0BD0192B09E11A2B85
:1095300007E11B2B05E11B331A331933002A3FE0E7
:1095400017BD84D717BFC6D71CD0800E1B1B1BAFFF
:1095500004D03AD012C116F10AD00EC116F11B5335
:1095600006E11A5304E1195302E1006A21D01BBF3E
:1095700008D0D890183719371A371B37002EF7D76D
:109580001ED016AF02D01B8F13D01B9F11D011C15C
:1095900000F012C11BF113C11AF114C119F108D066
:1095A0000DC100F00EC11BF10FC11AF110C119F16C
:1095B0001BC101F01AC102F019C103F034D0006AD6
:1095C000016A026A036A2FD0186B191F1A1F1B1F2A
:1095D000181F182B05E1192B03E11A2B01E11B2B96
:1095E00017B112D717B354D717B589D7B3D7EF50E0
:1095F000192705E31A2B03E11B2BD8B41581ED5273
:10960000EF501A2703E31B2BD8B41581ED52EF500E
:10961000EFBE01D0800A1B27D8B0158117B9FCD640
:1096200017BB3ED774D70001000C01010891FCC0A4
:1096300001F1FBC000F1FAC0FFF0F9C0FEF0FCC080
:109640000CF1FBC00BF1FAC00AF1F9C009F1106B83
:109650000F6B0E6B0D6B000136DE05E30101088117
:10966000800E0001FF1B01C10CF100C10BF1FFC016
:109670000AF1FEC009F10101106B0F6B0E6B8E0E2B
:109680000D6F000120DE01E217E101C10CF100C104
:109690000BF1FFC00AF1FEC009F152DE02C00EF16B
:1096A00001C00DF16BDE03C005F102C004F101C081
:1096B00003F100C002F1C7D001C10CF100C10BF1F0
:1096C000FFC00AF1FEC009F1800E0101106F960E75
:1096D0000F6F180E0E6F960E0D6F0001F4DDD8A0FF
:1096E000AAD001C10CF100C10BF1FFC00AF1FEC00C
:1096F00009F10101106B0F6B0E6B8E0E0D6F0001E7
:1097000033DD03C00CF102C00BF101C00AF100C04F
:1097100009F116DE02C007F101C006F101C10CF12A
:1097200000C10BF1FFC00AF1FEC009F10101106B8D
:109730000F6B0E6B8E0E0D6F000116DD00C009F170
:1097400001C00AF102C00BF103C00CF107C10EF118
:1097500006C10DF113DED8820CC110F10BC10FF15F
:109760000AC10EF109C10DF103C014F102C013F1D9
:1097700001C012F100C011F11CDE0101106B0F6B72
:109780000E6B8E0E0D6F03C014F102C013F101C0F9
:1097900012F100C011F100016CDC03C001F102C044
:1097A00000F101C0FFF000C0FEF007C10EF106C1DC
:1097B0000DF1E4DD0101106B0F6B0E6B8E0E0D6F62
:1097C00003C014F102C013F101C012F100C011F185
:1097D00000014FDC03C005F102C004F101C003F138
:1097E00000C002F101C10CF100C10BF1FFC00AF190
:1097F000FEC009F1A5DD02C00EF101C00DF1BEDD14
:10980000D89205C110F104C10FF103C10EF102C1DC
:109810000DF103C014F102C013F101C012F100C038
:1098200011F1C7DD03C005F102C004F101C003F16D
:1098300000C002F108D001C105F100C104F1FFC070
:1098400003F1FEC002F101C10CF100C10BF1FFC038
:109850000AF1FEC009F174DD02C00EF101C00DF184
:109860008DDDD88201C110F100C10FF1FFC00EF1F2
:10987000FEC00DF103C014F102C013F101C012F1DA
:1098800000C011F196DD03C001F102C000F101C07A
:10989000FFF000C0FEF0010108A102D0800E031B02
:1098A00001C10CF100C10BF1FFC00AF1FEC009F1CA
:1098B000106B0F6B0E6B0D6B000105DD44E00101B9
:1098C00008A120D00001FD53D8B402D001011AD064
:1098D000D88205C110F104C10FF103C10EF102C11C
:1098E0000DF10101146B136B126B7F0E116F0001F0
:1098F00060DD03C005F102C004F101C003F100C046
:1099000002F1010108B120D00001FD2D01D002D0EB
:1099100001011AD0D89205C110F104C10FF103C1A1
:109920000EF102C10DF10101146B136B126B7F0E6E
:10993000116F00013EDD03C005F102C004F101C05A
:1099400003F100C002F10101FCC00CF1FBC00BF1FE
:10995000FAC00AF1F9C009F1106B0F6B0E6B0D6BB9
:109960000001B1DC06E10101056B046B036B026BC6
:10997000000102C100F003C101F004C102F005C101
:1099800003F0CDEF4CF0F8C0FCF0F7C0FBF0F6C0F0
:10999000FAF0F5C0F9F0FD6B48D6000C2250245CBB
:1099A00012E303E12350215C0EE2FF0ED880235422
:1099B000F56F000E2454F66F2150F525256E2250C8
:1099C000F621266E06D02350215C256E24502258A5
:1099D000266E22C024F021C023F03490F86BF76B80
:1099E00026C0F6F025C0F5F062C000F063C001F0BB
:1099F000026A036A03C0FCF002C0FBF063C0FAF025
:109A000062C0F9F0F8C096F1F7C095F126C094F164
:109A100025C093F103C09AF102C099F163C098F197
:109A200062C097F14EEC47F003C0E8F002C0E7F0E7
:109A300001C0E6F000C0E5F0E8C0F8F0E7C0F7F0DC
:109A4000E6C0F6F0E5C0F5F01EEF48F000C0F5F016
:109A500001C0F6F002C0F7F003C0F8F003C010F147
:109A600002C00FF101C00EF100C00DF10101146B35
:109A7000136B100E126F840E116F000139EC48F059
:109A800003C0ECF002C0EBF001C0EAF000C0E9F066
:109A9000ECC00CF1EBC00BF1EAC00AF1E9C009F12E
:109AA0000101106B0F6B480E0E6F860E0D6F0001DB
:109AB000B4EC48F003C0ECF002C0EBF001C0EAF0F7
:109AC00000C0E9F0ECC0F8F0EBC0F7F0EAC0F6F047
:109AD000E9C0F5F058DF03C0F0F002C0EFF001C0BC
:109AE000EEF000C0EDF0F0C00CF1EFC00BF1EEC0F5
:109AF0000AF1EDC009F10101106B0F6B200E0E6F22
:109B0000820E0D6F0001B4EC48F003C0F0F002C00B
:109B1000EFF001C0EEF000C0EDF0F0C0F8F0EFC0E3
:109B2000F7F0EEC0F6F0EDC0F5F02DDF03C0F4F075
:109B300002C0F3F001C0F2F000C0F1F0D882F0C032
:109B400010F1EFC00FF1EEC00EF1EDC00DF1F4C059
:109B500014F1F3C013F1F2C012F1F1C011F129DCDC
:109B600000C0F5F001C0F6F002C0F7F003C0F8F055
:109B700003C00CF102C00BF101C00AF100C009F1F1
:109B80000101106B0F6B0E6B7E0E0D6F000163EC0D
:109B900049F009E3F4C0F0F0F3C0EFF0F2C0EEF0EA
:109BA000F1C0EDF01AD0D892F4C010F1F3C00FF16B
:109BB000F2C00EF1F1C00DF10101146B136B126BC9
:109BC0007F0E116F0001D9EC49F003C0F0F002C024
:109BD000EFF001C0EEF000C0EDF0F0C00CF1EFC00E
:109BE0000BF1EEC00AF1EDC009F1A0EC49F0015013
:109BF0003BEF79F0016A026A006A036A01019F5132
:109C000002E19E5118E0100EA06FD8909C379D374E
:109C1000003603369F51035C02E19E51005C07E36E
:109C20009E51005ED8A003069F51035ED880013686
:109C30000236A02FEAD70001000C006A016A026A0E
:109C4000036A0101936B946B956B966B9251911122
:109C500090118F112CE0200E976FD8908B378C3796
:109C60008D378E3793379437953796379251965D67
:109C700008E19151955D05E19051945D02E18F51AC
:109C8000935D0FE38F51935F9051D8A0903D945F07
:109C90009151D8A0913D955F9251D8A0923D965F89
:109CA000D8800036013602360336972FD6D7010EFC
:109CB000EA6E930EE96E0001000C186AF2BE188E6F
:109CC000F29E360E0101E66F000166EC3BF018BE15
:109CD000F28E186AF2BE188EF29E200E0101E66F17
:109CE000000176EC3BF018BEF28E2F0E01019E258E
:109CF000A66F170E9D25A76F186AF2BE188EF29EEA
:109D00009EC1E2F1A6C1E3F19DC1E4F1E56F00015E
:109D100086EC3BF018BEF28E186AF2BE188EF29EE8
:109D20002C0E0101E66F000166EC3BF018BEF28ECE
:109D30000101A46BA4511708D8A083D2A56BA5512B
:109D4000070866E3186AF2BE188EF29EE16B9FC1A7
:109D5000E0F1E36B900EE26F000102EC3BF018BE05
:109D6000F28E02C0A7F101C0A6F10101A4510124A5
:109D7000016E000E0220036E0150F2CFA8F1F29E98
:109D800003C0F7FF000173EC24F00101A8BFF28EBD
:109D9000A96F006EA551016E04E0D8900032012E2B
:109DA000FCD700A01AD0A1C1A6F1A76B186AF2BE19
:109DB000188EF29EA1C1E6F1000176EC3BF018BED0
:109DC000F28E186AF2BE188EF29EA0C1E6F176EC11
:109DD0003BF018BEF28E19D00101A3C1A6F1A76B0A
:109DE000186AF2BE188EF29EA3C1E6F1000176EC6D
:109DF0003BF018BEF28E186AF2BE188EF29EA2C117
:109E0000E6F176EC3BF018BEF28E0101A52B97D758
:109E1000A56BA551070867E3186AF2BE188EF29E7B
:109E2000E16B9FC1E0F1E36B900EE26F000102EC89
:109E30003BF018BEF28E02C0A7F101C0A6F1180EC9
:109E40000101A4250124016E000E0220036E0150C1
:109E5000F2CFA9F1F29E03C0F7FF000173EC24F0EA
:109E60000101A9BFF28EAA6F006EA551016E04E038
:109E7000D8900032012EFCD700A01AD0A1C1A6F1C3
:109E8000A76B186AF2BE188EF29EA1C1E6F100011E
:109E900076EC3BF018BEF28E186AF2BE188EF29E77
:109EA000A0C1E6F176EC3BF018BEF28E19D00101AC
:109EB000A3C1A6F1A76B186AF2BE188EF29EA3C1C9
:109EC000E6F1000176EC3BF018BEF28E186AF2BEA5
:109ED000188EF29EA2C1E6F176EC3BF018BEF28E2F
:109EE0000101A52B96D7A56BA551070867E3186A52
:109EF000F2BE188EF29EE16B9FC1E0F1E36B900E13
:109F0000E26F000102EC3BF018BEF28E02C0A7F136
:109F100001C0A6F1300E0101A4250124016E000E3E
:109F20000220036E0150F2CFA9F1F29E03C0F7FFA9
:109F3000000173EC24F00101A9BFF28EAA6F006E3C
:109F4000A551016E04E0D8900032012EFCD700A08C
:109F50001AD0A1C1A6F1A76B186AF2BE188EF29EA4
:109F6000A1C1E6F1000176EC3BF018BEF28E186A52
:109F7000F2BE188EF29EA0C1E6F176EC3BF018BE60
:109F8000F28E19D00101A3C1A6F1A76B186AF2BE27
:109F9000188EF29EA3C1E6F1000176EC3BF018BEEC
:109FA000F28E186AF2BE188EF29EA2C1E6F176EC2D
:109FB0003BF018BEF28E0101A52B96D7A56BA551DB
:109FC000070867E3186AF2BE188EF29EE16B9FC124
:109FD000E0F1E36B900EE26F000102EC3BF018BE83
:109FE000F28E02C0A7F101C0A6F1480E0101A4251E
:109FF0000124016E000E0220036E0150F2CFA9F180
:10A00000F29E03C0F7FF000173EC24F00101A9BF29
:10A01000F28EAA6F006EA551016E04E0D890003256
:10A02000012EFCD700A01AD0A1C1A6F1A76B186A17
:10A03000F2BE188EF29EA1C1E6F1000176EC3BF073
:10A0400018BEF28E186AF2BE188EF29EA0C1E6F11A
:10A0500076EC3BF018BEF28E19D00101A3C1A6F137
:10A06000A76B186AF2BE188EF29EA3C1E6F100013A
:10A0700076EC3BF018BEF28E186AF2BE188EF29E95
:10A08000A2C1E6F176EC3BF018BEF28E0101A52BE1
:10A0900096D7A56BA551070867E3186AF2BE188E1C
:10A0A000F29EE16B9FC1E0F1E36B900EE26F000165
:10A0B00002EC3BF018BEF28E02C0A7F101C0A6F17F
:10A0C000600E0101A4250124016E000E0220036E22
:10A0D0000150F2CFA9F1F29E03C0F7FF000173EC2B
:10A0E00024F00101A9BFF28EAA6F006EA551016E86
:10A0F00004E0D8900032012EFCD700A01AD0A1C1F4
:10A10000A6F1A76B186AF2BE188EF29EA1C1E6F105
:10A11000000176EC3BF018BEF28E186AF2BE188E83
:10A12000F29EA0C1E6F176EC3BF018BEF28E19D09B
:10A130000101A3C1A6F1A76B186AF2BE188EF29EA8
:10A14000A3C1E6F1000176EC3BF018BEF28E186A6E
:10A15000F2BE188EF29EA2C1E6F176EC3BF018BE7C
:10A16000F28E0101A52B96D7A56BA551070867E3D1
:10A17000186AF2BE188EF29EE16B9FC1E0F1E36BAC
:10A18000900EE26F000102EC3BF018BEF28E02C0AE
:10A19000A7F101C0A6F1780E0101A4250124016EEA
:10A1A000000E0220036E0150F2CFA9F1F29E03C00F
:10A1B000F7FF000173EC24F00101A9BFF28EAA6F32
:10A1C000006EA551016E04E0D8900032012EFCD73C
:10A1D00000A01AD0A1C1A6F1A76B186AF2BE188E12
:10A1E000F29EA1C1E6F1000176EC3BF018BEF28EC2
:10A1F000186AF2BE188EF29EA0C1E6F176EC3BF032
:10A2000018BEF28E19D00101A3C1A6F1A76B186A7E
:10A21000F2BE188EF29EA3C1E6F1000176EC3BF08F
:10A2200018BEF28E186AF2BE188EF29EA2C1E6F136
:10A2300076EC3BF018BEF28E0101A52B96D7A42B2D
:10A2400079D5186AF2BE188EF29E360EE66F0001BE
:10A2500066EC3BF018BEF28E186AF2BE188EF29EC3
:10A260000101E66B000176EC3BF018BEF28E000CAB
:10A270000101536B546B556B566B576B040E626F39
:10A28000636B676B686B696B6A6B6B6B6C6B6D6B2D
:10A290006E6B6F6B706B530E726F610E736F690E26
:10A2A000746F730E756F690E766F650E776F200E83
:10A2B000786F640E796F750E7A6F7B6B430E7C6FCF
:10A2C0006F0E7D6F6D0E7E6F700E7F6F740E806FE0
:10A2D000650E816F750E826F720E836F200E846F14
:10A2E000540E856F6F0E866F740E876F610E886FC8
:10A2F0006C0E896F8A6B0D0E636F7181666B656B77
:10A30000586B420E596F45C061F144C060F143C0C3
:10A310005FF142C05EF161C18EF160C18DF15FC13C
:10A320008CF15EC18BF1926B916B030E906FE80E16
:10A330008F6F000182DC03C05DF102C05CF101C0DF
:10A340005BF100C05AF15DC18EF15CC18DF15BC162
:10A350008CF15AC18BF10101926B916B270E906FBA
:10A36000100E8F6F000169DC00C057F15DC18EF1E6
:10A370005CC18DF15BC18CF15AC18BF10101926B13
:10A38000916B270E906F100E8F6F000156DCEFCF90
:10A390005AF1ECCF5BF1ECCF5CF1ECCF5DF15DC13C
:10A3A0008EF15CC18DF15BC18CF15AC18BF1010161
:10A3B000926B916B030E906FE80E8F6F00013DDC86
:10A3C00000C056F15DC18EF15CC18DF15BC18CF1B5
:10A3D0005AC18BF10101926B916B030E906FE80EE5
:10A3E0008F6F00012ADCEFCF5AF1ECCF5BF1ECCF9D
:10A3F0005CF1ECCF5DF15DC18EF15CC18DF15BC1B3
:10A400008CF15AC18BF10101926B916B906B640ED0
:10A410008F6F000112DC00C055F15DC18EF15CC18F
:10A420008DF15BC18CF15AC18BF10101926B916B83
:10A43000906B640E8F6F000100DCEFCF5AF1ECCF10
:10A440005BF1ECCF5CF1ECCF5DF15DC18EF15CC1F5
:10A450008DF15BC18CF15AC18BF10101926B916B53
:10A46000906B0A0E8F6F00011DEC4EF000C054F18E
:10A470005DC18EF15CC18DF15BC18CF15AC18BF174
:10A480000101926B916B906B0A0E8F6F00011DECB6
:10A490004EF0EFCF53F1186AF2BE188EF29E190EED
:10A4A0000101C36F140EC46F010EC66F720EC56F2B
:10A4B0007F0EC86FEF0EC76FCA6BC96B0001B7EC98
:10A4C0003BF018BEF28E186AF2BE188EF29E020E93
:10A4D0000101C36F210EC46F010EC66F7C0EC56FE4
:10A4E0007F0EC86FEF0EC76FCA6BC96B0001B7EC68
:10A4F0003BF018BEF28E010163510C08D8B4D8D0DD
:10A5000000017BEC47F003C055F002C054F001C0DD
:10A5100053F000C052F055C08EF154C08DF153C0BD
:10A520008CF152C08BF1FCEC47F00400010171B1D9
:10A5300004D063510D08D8B4A2D07191646B6451FA
:10A5400004080FE3D8906435036A670FE96E010EC3
:10A550000320EA6E070EEC6EED52E00EEF6E642BF8
:10A56000EED7D8906235036A670FE96E010E0320BB
:10A57000EA6EF80EEC6EED52EF6A680E58258B6F9E
:10A580009D6F59C19EF153C19FF168C1A1F167C18F
:10A59000A0F166C1A3F165C1A2F100015DEC4EF02E
:10A5A0004F0E010158258B6F9D6F59C19EF154C10B
:10A5B0009FF16AC1A1F169C1A0F166C1A3F165C1B2
:10A5C000A2F100015DEC4EF0320E010158258B6FB7
:10A5D0009D6F59C19EF155C19FF16CC1A1F16BC135
:10A5E000A0F166C1A3F165C1A2F100015DEC4EF0DE
:10A5F000190E010158258B6F9D6F59C19EF156C1EF
:10A600009FF16EC1A1F16DC1A0F166C1A3F165C159
:10A61000A2F100015DEC4EF058C19DF159C19EF1CF
:10A6200057C19FF170C1A1F16FC1A0F166C1A3F143
:10A6300065C1A2F15DEC4EF04F0E01015825516F3E
:10A64000260E5925526F040E515D8B6F020E522556
:10A650008C6F020E515D8D6F090E52258E6F8BC16E
:10A660008FF18CC190F18DC191F1926F010E936FBA
:10A67000946FFF0E966F956F0001F1EC45F00001AD
:10A6800094EC3DF001C063F10101635109080FE34F
:10A69000036A6251530FE96E010E0320EA6E63C133
:10A6A000EFFF625302E0620702D0040E626F24D70C
:10A6B0005D6B5C6B5B6B53C15AF18E6B8D6B8C6BFE
:10A6C00054C18BF18EC196F18DC195F18CC194F17D
:10A6D00054C193F19A6B996B986B0A0E976F0001B6
:10A6E0004EEC47F0005001015A2701505B23025005
:10A6F0005C2303505D238E6B8D6B8C6B55C18BF18E
:10A700008EC196F18DC195F18CC194F155C193F133
:10A710009A6B996B986B640E976F00014EEC47F043
:10A72000005001015A2701505B2302505C23035063
:10A730005D238E6B8D6B8C6B56C18BF18EC196F148
:10A740008DC195F18CC194F156C193F19A6B996BBF
:10A75000030E986FE80E976F00014EEC47F0005023
:10A7600001015A2701505B2302505C2303505D23F3
:10A770008E6B8D6B8C6B57C18BF18EC196F18DC139
:10A7800095F18CC194F157C193F19A6B996B270E97
:10A79000986F100E976F00014EEC47F000500101CA
:10A7A0005A2701505B2302505C2303505D235DC197
:10A7B00096F15CC195F15BC194F15AC193F19A6B2A
:10A7C000996B030E986FE80E976F00014EEC47F0FF
:10A7D00003C045F002C044F001C043F000C042F0A5
:10A7E00072EF61F00101536B546B556B566B576BF5
:10A7F0005C6B5D6B5E6B5F6B606B616B626B636B05
:10A80000646B656B040E6E6F6F6B530E726F610E2F
:10A81000736F690E746F730E756F690E766F650EC8
:10A82000776F200E786F640E796F750E7A6F7B6B81
:10A83000430E7C6F6F0E7D6F6D0E7E6F700E7F6F9F
:10A84000740E806F650E816F750E826F720E836F4E
:10A85000200E846F500E856F610E866F720E876FAB
:10A86000740E886F896B0D0E6F6F5B6B5A6B586B34
:10A87000420E596F718149C06DF148C06CF147C0FB
:10A880006BF146C06AF16DC18EF16CC18DF16BC187
:10A890008CF16AC18BF1926B916B906B640E8F6F30
:10A8A00000011DEC4EF003C069F102C068F101C067
:10A8B00067F100C066F169C18EF168C18DF167C1B1
:10A8C0008CF166C18BF10101926B916B270E906F39
:10A8D000100E8F6F00011DEC4EF000C057F169C1E2
:10A8E0008EF168C18DF167C18CF166C18BF10101F8
:10A8F000926B916B270E906F100E8F6F00011DEC05
:10A900004EF0EFCF66F1ECCF67F1ECCF68F1ECCF12
:10A9100069F169C18EF168C18DF167C18CF166C1C1
:10A920008BF10101926B916B030E906FE80E8F6FAC
:10A9300000011DEC4EF000C056F169C18EF168C1F6
:10A940008DF167C18CF166C18BF10101926B916B46
:10A95000030E906FE80E8F6F00011DEC4EF0EFCFED
:10A9600066F1ECCF67F1ECCF68F1ECCF69F169C12A
:10A970008EF168C18DF167C18CF166C18BF1010167
:10A98000926B916B906B640E8F6F00011DEC4EF01B
:10A9900000C055F169C18EF168C18DF167C18CF1BC
:10A9A00066C18BF10101926B916B906B640E8F6F9E
:10A9B00000011DEC4EF0EFCF66F1ECCF67F1ECCF6C
:10A9C00068F1ECCF69F169C18EF168C18DF167C1A1
:10A9D0008CF166C18BF10101926B916B906B0A0E49
:10A9E0008F6F00011DEC4EF000C054F169C18EF173
:10A9F00068C18DF167C18CF166C18BF10101926B69
:10AA0000916B906B0A0E8F6F00011DEC4EF0EFCF33
:10AA100053F1186AF2BE188EF29E190E0101C36F2F
:10AA2000140EC46F010EC66F720EC56F7F0EC86F15
:10AA3000EF0EC76FCA6BC96B0001B7EC3BF018BED5
:10AA4000F28E186AF2BE188EF29E060E0101C36FD6
:10AA5000230EC46F010EC66F7C0EC56F7F0EC86FCC
:10AA6000EF0EC76FCA6BC96B0001B7EC3BF018BEA5
:10AA7000F28E01016F510C08D8B4D8D000017BECE4
:10AA800047F003C055F002C054F001C053F000C0BD
:10AA900052F055C08DF154C08CF153C08BF152C0AF
:10AAA0008AF1DCEC47F00400010171B104D06F5170
:10AAB0000D08D8B4A2D07191706B705104080FE3E7
:10AAC000D8907035036A5C0FE96E010E0320EA6EC0
:10AAD000070EEC6EED52E00EEF6E702BEED7D890B5
:10AAE0006E35036A5C0FE96E010E0320EA6EF80E04
:10AAF000EC6EED52EF6A680E58258A6F9D6F59C152
:10AB00009EF153C19FF15DC1A1F15CC1A0F15BC198
:10AB1000A3F15AC1A2F100015DEC4EF04F0E01010C
:10AB200058258A6F9D6F59C19EF154C19FF15FC135
:10AB3000A1F15EC1A0F15BC1A3F15AC1A2F1000174
:10AB40005DEC4EF0360E010158258A6F9D6F59C19C
:10AB50009EF155C19FF161C1A1F160C1A0F15BC13E
:10AB6000A3F15AC1A2F100015DEC4EF0190E0101F2
:10AB700058258A6F9D6F59C19EF156C19FF163C1DF
:10AB8000A1F162C1A0F15BC1A3F15AC1A2F1000120
:10AB90005DEC4EF058C19DF159C19EF157C19FF136
:10ABA00065C1A1F164C1A0F15BC1A3F15AC1A2F1D9
:10ABB0005DEC4EF0360E01015825516F260E5925D9
:10ABC000526F040E515D8A6F020E52258B6F020E7A
:10ABD000515D8C6F090E52258D6F8AC18FF18BC12B
:10ABE00090F18CC191F1926F010E936F946FFF0EF3
:10ABF000966F956F0001F1EC45F0000194EC3DF08B
:10AC000001C06FF101016F5109080FE3036A6E5132
:10AC1000530FE96E010E0320EA6E6FC1EFFF6E5312
:10AC200002E06E0702D0040E6E6F24D7696B686B6A
:10AC3000676B53C166F18D6B8C6B8B6B54C18AF162
:10AC40008DC196F18CC195F18BC194F154C193F1F2
:10AC50009A6B996B986B0A0E976F00014EEC47F058
:10AC600000500101662701506723025068230350FA
:10AC700069238D6B8C6B8B6B55C18AF18DC196F1FD
:10AC80008CC195F18BC194F155C193F19A6B996B7D
:10AC9000986B640E976F00014EEC47F00050010175
:10ACA00066270150672302506823035069238D6B88
:10ACB0008C6B8B6B56C18AF18DC196F18CC195F16D
:10ACC0008BC194F156C193F19A6B996B030E986FF7
:10ACD000E80E976F00014EEC47F000500101662727
:10ACE0000150672302506823035069238D6B8C6BDE
:10ACF0008B6B57C18AF18DC196F18CC195F18BC1D7
:10AD000094F157C193F19A6B996B270E986F100EBF
:10AD1000976F00014EEC47F000500101662701508B
:10AD20006723025068230350692369C196F168C103
:10AD300095F167C194F166C193F19A6B996B986B29
:10AD4000640E976F00014EEC47F003C049F002C05B
:10AD500048F001C047F000C046F083EF61F0B6C094
:10AD6000EAFFB5C0E9FF0101A5C1EFFFE92AD8B4A8
:10AD7000EA2AEF6A0001B52BD8B4B62B000CEACF53
:10AD8000A4F1E9CFA3F101019D39F0099F6F9F273D
:10AD9000E20FA06F320FA26F9D510F0BA027A027CB
:10ADA000A227E90FA16FA127A1279C390F0BA1278B
:10ADB000A227A137A237A21FA2379C510F0BA227AF
:10ADC0009F37070E9E6F0A0EA107A227FDE3A0077B
:10ADD000A127FDE39F07A027FDE39E079F27FDE333
:10ADE000010EEA6E9E0EE96E070EA315A39DE926DD
:10ADF000A20EE95CD8B4A38DEF50006E08E1A3BDAC
:10AE000006D0A3B915D0A3B702D0200E03D0A387D4
:10AE1000A399300E0026EACF9DF1E9CF9CF100C046
:10AE2000A5F100019CDF9DC1EAFF9CC1E9FF010182
:10AE3000EE50A3ADDDD7000149EF58F00101516B91
:10AE4000526B536B566B576B586B596B5A6B5B6BF2
:10AE5000020E5E6F5F6B450E616F740E626F610E66
:10AE6000636F6C0E646F6F0E656F6E0E666F676F4B
:10AE7000610E686F670E696F650E6A6F6B6B440ECB
:10AE80006C6F690E6D6F730E6E6F740E6F6F610E67
:10AE9000706F6E0E716F630E726F650E736F200EA2
:10AEA000746F650E756F6E0E766F200E776F630E82
:10AEB000786F6D0E796F7A6B700E7B6F610E7C6FA1
:10AEC000720E7D6F200E7E6F690E7F6F6D0E806F2C
:10AED000700E816F750E826F6C0E836F730E846FB0
:10AEE000690E856F6F0E866F6E0E876F886B490EC9
:10AEF000896F6D0E8A6F700E8B6F750E8C6F6C0E76
:10AF00008D6F730E8E6F200E8F6F3A0E906F916B58
:10AF1000996B986B0D0E5F6F5D6B5C6B546B4A0E9B
:10AF2000556F63C09BF162C09AF1186AF2BE188E29
:10AF3000F29E010EC36FC46FC66F890EC56FA50E5A
:10AF4000C86F080EC76FCA6BC96B0001B7EC3BF046
:10AF500018BEF28E186AF2BE188EF29E140E01010F
:10AF6000C36FC46F010EC66F610EC56F7F0EC86FD1
:10AF7000EF0EC76FCA6BC96B0001B7EC3BF018BE90
:10AF8000F28E186AF2BE188EF29E010E0101C36F96
:10AF9000230EC46F010EC66F6C0EC56F7F0EC86F97
:10AFA000EF0EC76FCA6BC96B0001B7EC3BF018BE60
:10AFB000F28E186AF2BE188EF29E050E0101C36F62
:10AFC000320EC46F010EC66F7B0EC56F7F0EC86F49
:10AFD000EF0EC76FCA6BC96B0001B7EC3BF018BE30
:10AFE000F28E9BC19DF19AC19CF101019F6B640E91
:10AFF0009E6F0001FAEC4DF001C053F19BC19DF131
:10B000009AC19CF101019F6B640E9E6F0001FAECE6
:10B010004DF000C09AF1010103C09BF19BC19DF16D
:10B020009AC19CF19F6B0A0E9E6F0001FAEC4DF0E5
:10B0300001C052F19BC19DF19AC19CF101019F6B2E
:10B040000A0E9E6F0001FAEC4DF000C051F10101B3
:10B05000F29ACF6ACE6A1C6A1B6A226A216A5F5121
:10B060000C08D8B4A0D004005F510A0802E1CF6AEE
:10B07000CE6ACE50986FCFCF99F1010E0001B66F16
:10B08000920EB56F080EE96E99C19DF198C19CF1C1
:10B0900076D60101976B186AF2BE188EF29E4B0E9F
:10B0A000C36F010EC46FC66F920EC56FFF0EC86FDF
:10B0B000C76FCA6BC96B0001B7EC3BF018BEF28ECC
:10B0C0000101606B605102080FE3D8906035036A9C
:10B0D000560FE96E010E0320EA6E070EEC6EED527C
:10B0E000E00EEF6E602BEED7D8905E35036A560FF8
:10B0F000E96E010E0320EA6EF80EEC6EED52EF6A77
:10B100004B0E54259C6F9D6F55C19EF151C19FF10F
:10B1100057C1A1F156C1A0F15DC1A3F15CC1A2F17B
:10B1200000015DEC4EF0320E010154259C6F9D6FC5
:10B1300055C19EF152C19FF159C1A1F158C1A0F171
:10B140005DC1A3F15CC1A2F100015DEC4EF0190EEE
:10B15000010154259C6F9D6F55C19EF153C19FF114
:10B160005BC1A1F15AC1A0F15DC1A3F15CC1A2F123
:10B1700000015DEC4EF094EC3DF001C05FF1010187
:10B180005F5109080FE3036A5E51510FE96E010E2A
:10B190000320EA6E5FC1EFFF5E5302E05E0702D05C
:10B1A000020E5E6F5CD7CF6ACE6AF28A636A51C1C3
:10B1B00062F09D6B52C19CF1186AF2BE188EF29E2D
:10B1C0009DC1E1F152C1E0F1E36B0A0EE26F0001B3
:10B1D00002EC3BF018BEF28E015062260250632250
:10B1E00001019D6B53C19CF1186AF2BE188EF29E4C
:10B1F0009DC1E1F153C1E0F1E36B640EE26F000128
:10B2000002EC3BF018BEF28E01506226025063221F
:10B21000120E01019C6F63C09EF162C09DF100019E
:10B22000EFEC3DF094EF61F0080E0101916F00C06A
:10B2300092F1948800D00000948682A6FED782B84E
:10B24000D88082A8D890013600D094968B96912F02
:10B25000F0D7948800D000008B989251D8A494988D
:10B260000000948682A6FED700D08B96949600D0DC
:10B2700000008B989498000166EF59F0948800D0F4
:10B28000948600D000008B98949800D08B9694966A
:10B29000D00E0101906F000137EC3DF08EC190F1AE
:10B2A00037EC3DF0948800D0948600D0000082A650
:10B2B000FED78B98949800D08B969496D10E01016E
:10B2C000906F000137EC3DF0006AAED701C08FF1FE
:10B2D00094980000948682A6FED700D000D000008B
:10B2E000948800D001018FC101F00001000C010120
:10B2F00090BF11D00F0E006E8F3900160A0E005C41
:10B3000003E2300E002602D09051002600C0A5F1C5
:10B31000000125DD01010F0E8F170A0E8F5D02E27D
:10B32000300E02D0909F90518F278FC1A5F1000160
:10B3300016DD000C020E01018E6F00019FDF01C0BF
:10B340008BF1010E01018E6F000198DF01C08CF1BD
:10B3500001018E6B000192DF01C08DF18AC1B6F050
:10B3600089C1B5F08BC18FF1570E0101906F0001BB
:10B37000BEDF3A0E0101A56F0001F1DC8CC18FF137
:10B38000570E0101906F0001B2DF3A0E0101A56F67
:10B390000001E5DC8DC18FF1570E0101906F0001B6
:10B3A000A6DF080E01018925E96E000E8A21EA6EEA
:10B3B000EF6A89C101F000010FEF5CF0040E01019A
:10B3C0008E6F00015BDF01C08BF1050E01018E6FF6
:10B3D000000154DF01501F0B01018D6F060E8E6FAF
:10B3E00000014CDF01C08EF18AC1B6F089C1B5F011
:10B3F0008BC18FF1570E0101906F000178DF2F0E86
:10B400000101A56F0001ABDC8DC18FF1570E010169
:10B41000906F00016CDF2F0E0101A56F00019FDC12
:10B420008EC18FF1570E0101906F000160DF080E91
:10B4300001018925E96E000E8A21EA6EEF6A89C151
:10B4400001F0000116EF5CF00101946B8CC103F078
:10B450008BC1E9FF8CC1EAFFEF52D8B423D18CC174
:10B4600003F08BC1E9FF8CC1EAFFEF507E083EE399
:10B470008CC103F08BC1E9FF8CC1EAFF200EEF5CA9
:10B48000A96F186AF2BE188EF29EE16BE06FE36B53
:10B49000100EE26F000102EC3BF018BEF28E02C00B
:10B4A000ABF1010101C0AAF1010EEA6E950EE96E41
:10B4B00002C0AFF101C0AEF1F2CFACF1F29E026A70
:10B4C000100E016E022AAFC1F7FFAE5100016BEC06
:10B4D00021F00A000900EF6AF5CFEEFF012EFAD73E
:10B4E000022EF8D70101ACBFF28E1CD0010EEA6E1D
:10B4F000950EE96EF2CFA7F1F29E026A100E016E70
:10B50000022AF76A000E00016BEC21F00A00090024
:10B51000EF6AF5CFEEFF012EFAD7022EF8D7010120
:10B52000A7BFF28E8CC103F08BC1E9FF8CC1EAFF8B
:10B53000EF500A0A000103E0070A06E009D00D0EE9
:10B5400001018A27AAD00001010E0101896FA5D04F
:10B55000080E01018925830804E2010E896F0D0E92
:10B560008A27926B92510708D8A096D09151945D8A
:10B5700004E1F80EA66FA56B04D08EC1A6F18DC1B3
:10B58000A5F1936B935107083EE3036A9251950F1F
:10B59000E96E010E0320EA6EEFCFA7F1A7C100F01C
:10B5A0009351016E04E0D8900032012EFCD700A028
:10B5B00015D093518A25A76F186AF2BE188EF29E95
:10B5C00089C1DEF1DF6FA6C1E1F1A5C1E0F10001A3
:10B5D0009DEC3BF018BEF28E13D0010193518A25E9
:10B5E000A76F186AF2BE188EF29E89C1DEF1DF6F76
:10B5F000E16B8FC1E0F100019DEC3BF018BEF28ED3
:10B600000101932BBFD7936B9351030841E3080EBD
:10B610009225036A950FE96E010E0320EA6EEFCFC3
:10B62000A8F1A8C100F09351016E04E0D890003257
:10B63000012EFCD700A016D0080E93258A25A76FEF
:10B64000186AF2BE188EF29E89C1DEF1DF6FA6C1C4
:10B65000E1F1A5C1E0F100019DEC3BF018BEF28ED6
:10B6600014D00101080E93258A25A76F186AF2BE2F
:10B67000188EF29E89C1DEF1DF6FE16B8FC1E0F1C0
:10B6800000019DEC3BF018BEF28E0101932BBCD75C
:10B690009251922B892B66D7892B8B2BD8B48C2B6C
:10B6A000942BD4D60001000C0D0E0101516F530EE6
:10B6B000696F610E6A6F690E6B6F730E6C6F690E46
:10B6C0006D6F650E6E6F200E6F6F640E706F650E7E
:10B6D000716F726B6C0E736F270E746F680E756FDF
:10B6E000650E766F750E776F720E786F650E796FD7
:10B6F000200E7A6F650E7B6F740E7C6F7D6B640E0F
:10B700007E6F650E7F6F200E806F6C0E816F610EF5
:10B71000826F200E836F640E846F610E856F740ECE
:10B72000866F650E876F886B0D0E516F686B676B48
:10B73000536B0A0E546F186AF2BE188EF29E180EE2
:10B74000C36F140EC46F010EC66F690EC56F7F0EF6
:10B75000C86FEF0EC76FCA6BC96B0001B7EC3BF047
:10B7600018BEF28E186AF2BE188EF29E0A0E010101
:10B77000C36F230EC46F010EC66F730EC56F7F0EAD
:10B78000C86FEF0EC76FCA6BC96B0001B7EC3BF017
:10B7900018BEF28E186AF2BE188EF29E1E0E0101BD
:10B7A000C36F320EC46F010EC66F7E0EC56F7F0E63
:10B7B000C86FEF0EC76FCA6BC96B0001B7EC3BF0E7
:10B7C00018BEF28E0101526B51510C08D8B400D250
:10B7D00000017BEC47F003C055F002C054F001C0FB
:10B7E00053F000C052F055C08DF154C08CF153C0DD
:10B7F0008BF152C08AF1DCEC47F055C08EF154C099
:10B800008DF153C08CF152C08BF1FCEC47F0040079
:10B81000010E01018A6F550E896F00018BD5010E53
:10B8200001018A6F5E0E896F0001C8D50101535175
:10B830000A081BE1186AF2BE188EF29E1B0EC36F37
:10B84000460EC46F010EC66F550EC56F070EC86F4A
:10B85000E00EC76F68C1CAF167C1C9F10001B7EC5A
:10B860003BF018BEF28E13D001011B0E896F460EFD
:10B870008A6F010E8C6F550E8B6F070E8E6FE00E68
:10B880008D6F8F6B906B53C191F10001DDDD010174
:10B8900054510A081BE1186AF2BE188EF29E1B0E64
:10B8A000C36F5A0EC46F010EC66F5E0EC56F070ED2
:10B8B000C86FFF0EC76F68C1CAF167C1C9F1000147
:10B8C000B7EC3BF018BEF28E13D001011B0E896F4E
:10B8D0005A0E8A6F010E8C6F5E0E8B6F070E8E6F85
:10B8E000FF0E8D6F8F6B906B54C191F10001ACDD39
:10B8F00094EC3DF001C051F10101525320E151514E
:10B9000002081DE3020E8E6F0001B8DC01503F0BF0
:10B91000666E66500F0B0101896F5151100DF35087
:10B920008925666E522B010E536F0D0E516F020E5C
:10B93000896F66C08AF1000164EC3DF00101522D6F
:10B9400025D05151090822E36650180806E26650D6
:10B9500019081CE25151030819E3020E8E6F000111
:10B960008DDC01503F0B666E6650F00B01015125D6
:10B97000666E522B030E536F0D0E516F020E896FC0
:10B9800066C08AF1000164EC3DF0010152510208E9
:10B9900020E1515105081DE3010E8E6F00016EDCA0
:10B9A00001507F0B676E67500F0B0101896F51517A
:10B9B000100DF3508925676E522B040E536F0D0E38
:10B9C000516F010E896F67C08AF1000164EC3DF090
:10B9D0000101525103081DE1515109081AE3010EFA
:10B9E0008E6F00014BDC01507F0B676E6750F00BD0
:10B9F00001015125676E522B546B0A0E536F0D0EC9
:10BA0000516F010E896F67C08AF1000164EC3DF04F
:10BA1000010104005251040820E1515103081DE3C3
:10BA2000040E8E6F00012ADC01503F0B696E6950D5
:10BA30000F0B0101896F5151100DF3508925696E6B
:10BA4000522B010E546F0D0E516F040E896F69C099
:10BA50008AF1000164EC3DF001015251050826E134
:10BA60005151090823E369502F0806E26950300854
:10BA70001DE2515101081AE3040E8E6F00013EECE5
:10BA800059F001503F0B696E6950F00B01015125CF
:10BA9000696E0D0E516F522B030E546F040E896F99
:10BAA00069C08AF1000164EC3DF0010152510608C1
:10BAB00021E1515101081EE3050E8E6F00013EEC9D
:10BAC00059F001501F0B6A6E6A500F0B0101896F0C
:10BAD0005151100DF35089256A6E522B040E546F8C
:10BAE0000D0E516F050E896F6AC08AF1000164EC7A
:10BAF0003DF001015251070826E15151090823E3A5
:10BB00006A500F0806E26A5010081DE251510208FF
:10BB10001AE3050E8E6F00013EEC59F001501F0B29
:10BB20006A6E6A50F00B010151256A6E0D0E516F5D
:10BB3000522B060E546F050E896F6AC08AF1000100
:10BB400064EC3DF0010104005251080820E151511C
:10BB500009081DE3060E8E6F00013EEC59F001C08E
:10BB60006BF06B500F0B0101896F5151100DF350A9
:10BB700089256B6E522B070E546F0D0E516F060EFA
:10BB8000896F6BC08AF1000164EC3DF001015251F4
:10BB900009081DE1515109081AE3060E8E6F0001D4
:10BBA0003EEC59F001C06BF06B50F00B01015125D8
:10BBB0006B6E0D0E516F526B536B0A0E546F060E67
:10BBC000896F6BC08AF1000164EC3DF00101FCD586
:10BBD0000001A4EF61F001017251016A715D03E29D
:10BBE00071C100F00CD0006A080E736F7137003617
:10BBF0007251005CD8B0006E0136732FF7D7000188
:10BC0000000C01506FC171F1640E0101726F0001EF
:10BC1000E2DF00C06FF10150300E08E1010170A3B6
:10BC200010D070B70ED070B9200E04D001017097FB
:10BC300070997081012601C0A5F10001AFEC56F0AA
:10BC400001016FC171F10A0E726F0001C4DF00C003
:10BC50006FF10150300E08E1010170B70BD070A1F7
:10BC600009D070B9200E0001012601C0A5F1AFEC8A
:10BC700056F00101300E6F276FC1A5F10001AFEC46
:10BC800056F0000C0D0E0101516F010E536F520E54
:10BC9000566F650E576F670E586F6C0E596F610EB9
:10BCA0005A6F670E5B6F650E5C6F200E5D6F640EE2
:10BCB0005E6F750E5F6F606B430E616F6F0E626F2C
:10BCC0006E0E636F740E646F720E656F610E666F39
:10BCD000730E676F740E686F650E696F6A6B556BD4
:10BCE000546B186AF2BE188EF29E140EC36FC46FA6
:10BCF000010EC66F560EC56F7F0EC86FEF0EC76F71
:10BD0000CA6BC96B0001B7EC3BF018BEF28E186A23
:10BD1000F2BE188EF29E190E0101C36F230EC46F7E
:10BD2000010EC66F610EC56F7F0EC86FEF0EC76F35
:10BD3000CA6BC96B0001B7EC3BF018BEF28E010E66
:10BD40000101526F52511F081CE3546B5235556F5D
:10BD500055375537F80E551753C199F1410E9A6F63
:10BD600053C19BF1500E9C6F55C19EF154C19DF182
:10BD7000000173EC44F0040001015251522B532B8B
:10BD8000E1D7556B546B010E526F52513F0824E3BB
:10BD9000706B5235546F7035556F54375537543773
:10BDA00055375437553754375537E00E541753C16C
:10BDB00099F1410E9A6F53C19BF1500E9C6F55C182
:10BDC0009EF154C19DF1000173EC44F004000101A7
:10BDD0005251522B532BD9D7556B546B010E526FC6
:10BDE00052511F0818E3556B52C154F153C199F1D8
:10BDF000410E9A6F53C19BF1500E9C6F55C19EF13D
:10BE000054C19DF1000173EC44F004000101525152
:10BE1000522B532BE5D751510C085EE00400000172
:10BE20007BEC47F003C055F002C054F001C053F062
:10BE300000C052F055C08DF154C08CF153C08BF14D
:10BE400052C08AF1DCEC47F055C08EF154C08DF140
:10BE500053C08CF152C08BF1FCEC47F094EC3DF0F8
:10BE600001C051F1010EB66F6B0EB56F65C06FF179
:10BE7000030E0101706F0001C4DE01016E6B186AD0
:10BE8000F2BE188EF29E320EC36F550EC46F010EB5
:10BE9000C66F6B0EC56FFF0EC86FE00EC76FCA6B23
:10BEA000C96B0001B7EC3BF018BEF28E0101515195
:10BEB000040804E165500108D8A065065151060840
:10BEC00004E165507E08D8B0652A65C06FF10001B5
:10BED0001FEC3EF001019FD7AA6A170EA96E65C03C
:10BEE000A8FFA69CA69EA684F2CF00F0F29E0F01AA
:10BEF000550EA76EAA0EA76EA682A6B2FED7A6946E
:10BF00000050F2120001B3EF61F0080EEB6F840EE7
:10BF1000EC6FE00EED6FFF0EEE6FEF6F070EF06F40
:10BF2000260EF16F9B0EF26FC00EF36FD30EF46FFF
:10BF30001F0EF56FF80EF66F530EF76F610EF86F68
:10BF4000690EF96F730EFA6F690EFB6F650EFC6F69
:10BF5000200EFD6F540EFE6F6F0EFF6F740E010109
:10BF6000006F610E016F6C0E026F200E036F046F85
:10BF7000056B530E066F610E076F690E086F730E27
:10BF8000096F690E0A6F650E0B6F200E0C6F500E55
:10BF90000D6F610E0E6F720E0F6F740E106F690EC3
:10BFA000116F650E126F6C0E136F146B520E156FBE
:10BFB000650E166F670E176F6C0E186F610E196F96
:10BFC000670E1A6F650E1B6F200E1C6F520E1D6FD1
:10BFD0006F0E1E6F750E1F6F650E206F200E216F86
:10BFE000226F236B480E246F650E256F750E266F2A
:10BFF000720E276F650E286F200E296F2D0E2A6F87
:10C00000200E2B6F440E2C6F610E2D6F740E2E6F51
:10C01000650E2F6F200E306F316F326B430E336F12
:10C020006F0E346F6E0E356F740E366F720E376F83
:10C03000610E386F730E396F740E3A6F650E3B6F79
:10C04000200E3C6F3D6F3E6F3F6F406F416B426F04
:10C05000436F446F456F466F476F486F496F520E8D
:10C060004A6F650E4B6F740E4C6F6F0E4D6F750EF1
:10C070004E6F720E4F6F506B0001E681E36BE56B04
:10C08000FF0EE86FE76F0101526B516B000138EC56
:10C090003EF0840EEA6F080EE96FE553D8A46FD125
:10C0A000040094EC3DF001C0E4F07BEC47F003C0E9
:10C0B00055F002C054F001C053F000C052F055C01A
:10C0C0008DF154C08CF153C08BF152C08AF1DCEC7D
:10C0D00047F055C08EF154C08DF153C08CF152C061
:10C0E0008BF1FCEC47F0E451020808E0E451080849
:10C0F00005E0E4510C0802E0E6A140D1E691E451EC
:10C1000002081FE1E3531DE0D890E335036AEB0F0B
:10C11000E96E000E0320EA6EEAC0ECFFED52E9C0C2
:10C12000EFFFE307D890E335036AEB0FE96E000EEB
:10C130000320EA6EECCF03F0ED52EFCFE9F003C03D
:10C14000EAF0E451080820E1E35104081DE3D89027
:10C15000E335036AEB0FE96E000E0320EA6EEAC0D6
:10C16000ECFFED52E9C0EFFFE32BD890E335036A13
:10C17000EB0FE96E000E0320EA6EECCF03F0ED52F8
:10C18000EFCFE9F003C0EAF0D890E335036AEB0F94
:10C19000E96E000E0320EA6EE8C0ECFFED52E7C046
:10C1A000EFFF186AF2BE188EF29E010E0101C36FF6
:10C1B000130EC46FC66BF70EC56FECC0C8F1EBC0B1
:10C1C000C7F1CA6BC96B0001B7EC3BF018BEF28E29
:10C1D000186AF2BE188EF29E010E0101C36F220E84
:10C1E000C46F010EC66F060EC56FEEC0C8F1EDC07C
:10C1F000C7F1CA6BC96B0001B7EC3BF018BEF28EF9
:10C20000186AF2BE188EF29E010E0101C36F310E44
:10C21000C46F010EC66F150EC56FF0C0C8F1EFC038
:10C22000C7F1CA6BC96B0001B7EC3BF018BEF28EC8
:10C23000186AF2BE188EF29E010E0101C36F400E05
:10C24000C46F010EC66F240EC56FF2C0C8F1F1C0F5
:10C25000C7F1CA6BC96B0001B7EC3BF018BEF28E98
:10C26000186AF2BE188EF29E010E0101C36F4F0EC6
:10C27000C46F010EC66F330EC56FF4C0C8F1F3C0B2
:10C28000C7F1CA6BC96B0001B7EC3BF018BEF28E68
:10C29000186AF2BE188EF29E010E0101C36F610E84
:10C2A000C46F010EC66F420EC56FF6C0C8F1F5C06F
:10C2B000C7F1CA6BC96B0001B7EC3BF018BEF28E38
:10C2C0000400E4510C085AE1E351FA0F57E2060F5B
:10C2D000C1EF61F00101526B516B000138EC3EF08F
:10C2E00038EF51F00101526B516B000138EC3EF018
:10C2F000010EE56F43D00101526B516B000138EC28
:10C300003EF0F2EF53F00101526B516B000138EC3B
:10C310003EF0010EE56F32D00101526B516B00010E
:10C3200038EC3EF01EEF57F00101526B516B0001EB
:10C3300038EC3EF0E68122D00101526B516B0001D6
:10C3400038EC3EF054EF5BF00101526B516B000191
:10C3500038EC3EF0E68112D00101526B516B0001C6
:10C3600038EC3EF08FD40101526B516B000138EC78
:10C370003EF0E68103D0010EE56F00D08ED637EF98
:10C380007AF0F2CF0EF0F29EE824A70FF66EC30EFD
:10C39000F76ED8B0F72A0A00F550FA6E0800F5508B
:10C3A0000EBEF28EF96ED4C2F6C218C338C358C39B
:10C3B00076C3F0C0F2F0EFC0F1F0F2C003F0F1C0CC
:10C3C000E9FFF2C0EAFFEF5204E0F12BD8B4F22B00
:10C3D000F4D7EF51F15D006EF051F259036E00C0D9
:10C3E00001F0026E23EF63F0F2C003F0F1C0E9FF49
:10C3F000F2C0EAFFEF52D8B408D1F2C003F0F1C0A6
:10C40000E9FFF2C0EAFFEF50520828E3F2C003F060
:10C41000F1C0E9FFF2C0EAFF200EEF5C050DF3501A
:10C42000036A0101036FEA6AFC0EE96E076B03C140
:10C4300006F1F2CF04F1F29E050E016EF76A035188
:10C44000000163EC20F00A000900F5CFEEFF012E99
:10C45000FBD7010104BFF28E38D00001F2C003F017
:10C46000F1C0E9FFF2C0EAFFEF507E0828E3F2C016
:10C4700003F0F1C0E9FFF2C0EAFF530EEF5C050DD7
:10C48000F350036A0101036FEA6AFC0EE96E076B61
:10C4900003C106F1F2CF04F1F29E050E016EF76AB8
:10C4A00003510001F0EC20F00A000900F5CFEEFF87
:10C4B000012EFBD7010104BFF28E07D00001FC6BF7
:10C4C000FD6BFE6BFF6B0101006BF2C003F000011E
:10C4D000F1C0E9FFF2C0EAFFEF500A0A03E0070AE1
:10C4E00007E008D0F351070DF350010FF02788D073
:10C4F000EF6B86D0F351050DF350EF25830806E26C
:10C50000EF6BF351070DF350010FF027F86BF85163
:10C510000408D8A075D0F96BF9510608D8A06CD0E2
:10C52000036AF851FC0FE96E000E0320EA6EEFCFAC
:10C5300001F101C100F0F951016E04E0D890003220
:10C54000012EFCD700A029D0FA6BF351FA5D24E24A
:10C55000FB6BF351FB5D1EE2FB51EF250101016F07
:10C560000001F951F303F350F025FA250101036F9F
:10C57000186AF2BE188EF29E01C1DEF1DF6FF5C0BF
:10C58000E1F1F4C0E0F100019DEC3BF018BEF28E49
:10C59000FB2BDFD7FA2BD9D72DD0F65303E1F75178
:10C5A000020828E0FA6BF351FA5D24E2FB6BF351C9
:10C5B000FB5D1EE2FB51EF250101016F0001F95106
:10C5C000F303F350F025FA250101036F186AF2BE58
:10C5D000188EF29E01C1DEF1DF6FF7C0E1F1F6C007
:10C5E000E0F100019DEC3BF018BEF28EFB2BDFD793
:10C5F000FA2BD9D7F92B90D7F82BF351EF2787D700
:10C60000F12BD8B4F22BEF2BEFD6000C6B0EE86FAA
:10C610006D0EE96F680EEA6FEB6B670EEC6F5E0EE6
:10C62000ED6F550EEE6FB66BE40EB56FE3C06FF1B4
:10C63000130E0101706F000101EC5EF0E76BF06B0F
:10C64000E40EEF6FB6D602C0F0F001C0EFF0010EBD
:10C65000015CF16F000E0258F26FEC0EF125E96EED
:10C66000000EF221EA6EEFCFF3F0186AF2BE188ED8
:10C67000F29EF3C0C3F1040E0101C46FC66BE40E59
:10C68000C56F83C0C8F182C0C7F17BC0CAF17AC050
:10C69000C9F10001B7EC3BF018BEF28E710EEF6FDE
:10C6A000090EF06FF26BE80EF16F010EF36F81C0AF
:10C6B000F5F080C0F4F07BC0F7F07AC0F6F094DEBD
:10C6C00002EF7BF0120EEF25FC6F1F0EF025FD6FC1
:10C6D000186AF2BE188EF29EEFC0E2F1FCC0E3F1E0
:10C6E000F0C0E4F1E8CFE5F186EC3BF018BEF28E45
:10C6F000186AF2BE188EF29E2C0E0101E66F000140
:10C7000066EC3BF018BEF28EF1510908D8A032D287
:10C71000120EEF25FC6F1F0EF025FD6F186AF2BE9A
:10C72000188EF29EEFC0E2F1FCC0E3F1F0C0E4F13C
:10C73000E8CFE5F186EC3BF018BEF28E186AF2BE47
:10C74000188EF29E2C0E0101E66F000166EC3BF0A4
:10C7500018BEF28EF151F60FD8B0A3D00A0F37EF02
:10C7600066F0F36BF26B020EF56F3A0EF46F050E86
:10C77000F76F910EF66F090EF96FA60EF86F91D054
:10C78000F36B720EF26F020EF56FE50EF46F070E8B
:10C79000F76F330EF66F0A0EF96F180EF86F81D02F
:10C7A000F36BE40EF26F030EF56F900EF46F080E4C
:10C7B000F76FD50EF66F0A0EF96FFC0EF86F71D099
:10C7C000F36BE40EF26F030EF56F900EF46F080E2C
:10C7D000F76F040EF66F0A0EF96F8A0EF86F61D0CC
:10C7E000010EF36F560EF26F040EF56F3B0EF46FF1
:10C7F000080EF76F040EF66F0A0EF96F180EF86F39
:10C8000050D0010EF36FC80EF26F040EF56FE60EF6
:10C81000F46F080EF76F040EF66F0A0EF96F8A0EAA
:10C82000F86F3FD0010EF36FC80EF26F040EF56F74
:10C83000E60EF46F060EF76F620EF66F090EF96FD3
:10C84000A60EF86F2ED0F36BE40EF26F020EF56FAA
:10C85000E50EF46F070EF76F330EF66F0A0EF96FE1
:10C86000180EF86F1ED0F36BF26B040EF56F3B0ED3
:10C87000F46F060EF76F620EF66F090EF96FA60ED3
:10C88000F86F0FD0F36BF26B040EF56F3B0EF46F85
:10C89000080EF76F040EF66F0A0EF96F8A0EF86F26
:10C8A00000D0FB6BFA6BFB5356E1FA51710853E36E
:10C8B000FA51F225FC6FFB51F321FD6FD890FC3546
:10C8C000026EFD35036E0250F2CFFEF0F29E03C001
:10C8D000F7FF4FEC27F00900F5CF03F0FEBFF28E13
:10C8E000FF6F03C000F103C001F10101026B186A80
:10C8F000F2BE188EF29E03C0E6F1000176EC3BF02A
:10C9000018BEF28EFA51F225FC6FFB51F321FD6F38
:10C91000D890FC35026EFD35036E0250F2CFFEF06A
:10C92000F29E03C0F7FF4FEC27F00900F5CF03F0AC
:10C93000FEBFF28EFF6F03C000F1186AF2BE188EC0
:10C94000F29EE8CFE6F176EC3BF018BEF28EFA2BC1
:10C95000D8B4FB2BA8D7FB6BFA6BFB5356E1FA510B
:10C96000AA0853E3FA51F425FC6FFB51F521FD6F42
:10C97000D890FC35026EFD35036E0250F2CFFEF00A
:10C98000F29E03C0F7FF4FEC27F00900F5CF03F04C
:10C99000FEBFF28EFF6F03C000F103C001F1010181
:10C9A000026B186AF2BE188EF29E03C0E6F1000117
:10C9B00076EC3BF018BEF28EFA51F425FC6FFB5179
:10C9C000F521FD6FD890FC35026EFD35036E0250E7
:10C9D000F2CFFEF0F29E03C0F7FF4FEC27F0090004
:10C9E000F5CF03F0FEBFF28EFF6F03C000F1186AAF
:10C9F000F2BE188EF29EE8CFE6F176EC3BF018BE60
:10CA0000F28EFA2BD8B4FB2BA8D7FB6BFA6BFB5337
:10CA100056E1FA51D00853E3FA51F625FC6FFB5169
:10CA2000F721FD6FD890FC35026EFD35036E025084
:10CA3000F2CFFEF0F29E03C0F7FF4FEC27F00900A3
:10CA4000F5CF03F0FEBFF28EFF6F03C000F103C00D
:10CA500001F10101026B186AF2BE188EF29E03C04A
:10CA6000E6F1000176EC3BF018BEF28EFA51F625A5
:10CA7000FC6FFB51F721FD6FD890FC35026EFD3540
:10CA8000036E0250F2CFFEF0F29E03C0F7FF4FECB0
:10CA900027F00900F5CF03F0FEBFF28EFF6F03C051
:10CAA00000F1186AF2BE188EF29EE8CFE6F176EC3D
:10CAB0003BF018BEF28EFA2BD8B4FB2BA8D7FB6B39
:10CAC000FA6BFB5356E1FA51710853E3FA51F8251A
:10CAD000FC6FFB51F921FD6FD890FC35026EFD35DE
:10CAE000036E0250F2CFFEF0F29E03C0F7FF4FEC50
:10CAF00027F00900F5CF03F0FEBFF28EFF6F03C0F1
:10CB000000F103C001F10101026B186AF2BE188E38
:10CB1000F29E03C0E6F1000176EC3BF018BEF28E07
:10CB2000FA51F825FC6FFB51F921FD6FD890FC35C7
:10CB3000026EFD35036E0250F2CFFEF0F29E03C08E
:10CB4000F7FF4FEC27F00900F5CF03F0FEBFF28EA0
:10CB5000FF6F03C000F1186AF2BE188EF29EE8CF94
:10CB6000E6F176EC3BF018BEF28EFA2BD8B4FB2B34
:10CB7000A8D77CD0040EEF25FC6F080EF025FD6FC2
:10CB8000186AF2BE188EF29EEFC0E2F1FCC0E3F12B
:10CB9000F0C0E4F1E8CFE5F186EC3BF018BEF28E90
:10CBA000186AF2BE188EF29E2C0E0101E66F00018B
:10CBB00066EC3BF018BEF28EFB6BFA6BFB5356E152
:10CBC000FA512C0853E36E0EFA25FC6F0B0EFB2175
:10CBD000FD6FD890FC35026EFD35036E0250F2CF2A
:10CBE000FEF0F29E03C0F7FF4FEC27F00900F5CFEF
:10CBF00003F0FEBFF28EFF6F03C000F103C001F12E
:10CC00000101026B186AF2BE188EF29E03C0E6F1B3
:10CC1000000176EC3BF018BEF28E6E0EFA25FC6F2A
:10CC20000B0EFB21FD6FD890FC35026EFD35036EB7
:10CC30000250F2CFFEF0F29E03C0F7FF4FEC27F058
:10CC40000900F5CF03F0FEBFF28EFF6F03C000F1C5
:10CC5000186AF2BE188EF29EE8CFE6F176EC3BF051
:10CC600018BEF28EFA2BD8B4FB2BA8D7000CF2CF4B
:10CC70000EF0F29EE824930FF66ECC0EF76ED8B04D
:10CC8000F72A0A00F550FA6E0800F5500EBEF28E33
:10CC9000F96E62C780C7A0C7C0C7E0C702C824C872
:10CCA00046C866C884C8E56BE66BE76BE86B020EA6
:10CCB00001018E6F00013EEC59F001C0E9F0010E58
:10CCC00001018E6F00013EEC59F001C0EAF0010154
:10CCD0008E6B00013EEC59F001C0EBF0E939006EBB
:10CCE0000F0E00160050030BE86FE9510F0BE76FB2
:10CCF000EA39006E0F0E00160050070BE66FEA517E
:10CD00000F0BE56F0400E551955D02E134AC09D0ED
:10CD1000400EE325EC6FEF6FE4C0F0F0E5C0F1F0FA
:10CD2000D1DCE651965D02E134AC09D02D0EE3254D
:10CD3000EC6FEF6FE4C0F0F0E6C0F1F0C3DCE75158
:10CD4000975D02E134AC09D0130EE325EC6FEF6F71
:10CD5000E4C0F0F0E7C0F1F0B5DCE851985D02E125
:10CD600034AC07D0E3C0EFF0E4C0F0F0E8C0F1F07D
:10CD7000A9DC0400EBA11BD0130EE325140FED6F0B
:10CD8000070EE425EE6FEDC0EFF0F06F0B0EF16FC4
:10CD900099DC130EE325130FED6F120EE425EE6FF1
:10CDA000EDC0EFF0F06F0B0EF16F8CDC1FD0130EA7
:10CDB000E325130FED6F050EE425EE6F130EE3254B
:10CDC000180FF06F190EE425F16FEDC08FF1EEC072
:10CDD00090F1F0C091F1E8CF92F1010E0101936F53
:10CDE000946F966B956B0001F1EC45F0E5C095F002
:10CDF000E6C096F0E7C097F0E8C098F0349C88EF62
:10CE00007BF0EB6BEC6BED6BEE6BEF6B73C0F9F0E3
:10CE100072C0F8F079C0FBF078C0FAF077C0FDF08E
:10CE200076C0FCF075C0FFF074C0FEF0E75309E077
:10CE300051C0F7F050C0F6F04FC0F5F04EC0F4F01E
:10CE400008D049C0F7F048C0F6F047C0F5F046C03A
:10CE5000F4F0F7C051F0F6C050F0F5C04FF0F4C058
:10CE60004EF0F7C08EF1F6C08DF1F5C08CF1F4C034
:10CE70008BF10101926B916B906B640E8F6F0001CF
:10CE80001DEC4EF003C0F3F002C0F2F001C0F1F06F
:10CE900000C0F0F0F3C08EF1F2C08DF1F1C08CF162
:10CEA000F0C08BF10101926B916B270E906F100E09
:10CEB0008F6F00011DEC4EF000C0EFF0F3C08EF15B
:10CEC000F2C08DF1F1C08CF1F0C08BF10101926BD9
:10CED000916B270E906F100E8F6F00011DEC4EF0BE
:10CEE000EFCFF0F0ECCFF1F0ECCFF2F0ECCFF3F0CD
:10CEF000F3C08EF1F2C08DF1F1C08CF1F0C08BF176
:10CF00000101926B916B030E906FE80E8F6F000121
:10CF10001DEC4EF000C0EEF0F3C08EF1F2C08DF1CA
:10CF2000F1C08CF1F0C08BF10101926B916B030E9B
:10CF3000906FE80E8F6F00011DEC4EF0EFCFF0F018
:10CF4000ECCFF1F0ECCFF2F0ECCFF3F0F3C08EF1D8
:10CF5000F2C08DF1F1C08CF1F0C08BF10101926B48
:10CF6000916B906B640E8F6F00011DEC4EF000C052
:10CF7000EDF0F3C08EF1F2C08DF1F1C08CF1F0C094
:10CF80008BF10101926B916B906B640E8F6F0001BE
:10CF90001DEC4EF0EFCFF0F0ECCFF1F0ECCFF2F073
:10CFA000ECCFF3F0F3C08EF1F2C08DF1F1C08CF153
:10CFB000F0C08BF10101926B916B906B0A0E8F6F39
:10CFC00000011DEC4EF000C0ECF0F3C08EF1F2C099
:10CFD0008DF1F1C08CF1F0C08BF10101926B916B7E
:10CFE000906B0A0E8F6F00011DEC4EF0EFCFEBF04F
:10CFF0000400E75313E0E85309E0A50EF96F080EAB
:10D00000F86FA50EFF6F100EFE6F08D0A50EFF6F14
:10D01000080EFE6FA50EF96F100EF86FEB51905DC4
:10D0200004E1E75302E134AA14D0680EE5250101BA
:10D03000006F9D6FE6C09EF1EBC09FF1FFC0A1F1B4
:10D04000FEC0A0F1FDC0A3F1FCC0A2F100015DECA7
:10D050004EF0EC51915D04E1E75302E134AA14D0A3
:10D060004F0EE5250101006F9D6FE6C09EF1ECC0FB
:10D070009FF1FFC0A1F1FEC0A0F1FDC0A3F1FCC073
:10D08000A2F100015DEC4EF0ED51925D04E1E75339
:10D0900002E134AA14D0360EE5250101006F9D6F20
:10D0A000E6C09EF1EDC09FF1FFC0A1F1FEC0A0F16E
:10D0B000FDC0A3F1FCC0A2F100015DEC4EF0EE5109
:10D0C000935D04E1E75302E134AA14D0190EE5257B
:10D0D0000101006F9D6FE6C09EF1EEC09FF1F9C0A7
:10D0E000A1F1F8C0A0F1FDC0A3F1FCC0A2F10001C4
:10D0F0005DEC4EF0EF51945D04E1E75302E134AA98
:10D1000010D0E5C09DF1E6C09EF1EFC09FF1F9C0DF
:10D11000A1F1F8C0A0F1FDC0A3F1FCC0A2F15DEC4B
:10D120004EF0360EE525E96F260EE625EA6F040E71
:10D13000E95D0101006F020E0001EA250101016FA6
:10D14000020E0001E95D0101026F090E0001EA25EE
:10D150000101036F00C18FF101C190F102C191F192
:10D16000926F010E936F946FFBC096F1FAC095F128
:10D170000001F1EC45F0EBC090F0ECC091F0EDC097
:10D1800092F0EEC093F0EEC094F0349A96EF7BF0FC
:10D19000EB6BEC6BED6BEE6BEF6B6FC0F1F06EC099
:10D1A000F0F079C0F3F078C0F2F077C0F5F076C017
:10D1B000F4F071C0F7F070C0F6F0E75309E04DC02D
:10D1C000FFF04CC0FEF04BC0FDF04AC0FCF008D0B0
:10D1D00045C0FFF044C0FEF043C0FDF042C0FCF08B
:10D1E000FFC04DF0FEC04CF0FDC04BF0FCC04AF05B
:10D1F000FFC08EF1FEC08DF1FDC08CF1FCC08BF143
:10D200000101926B916B030E906FE80E8F6F00011E
:10D210001DEC4EF003C0FBF002C0FAF001C0F9F0C3
:10D2200000C0F8F0FBC08EF1FAC08DF1F9C08CF1AE
:10D23000F8C08BF10101926B916B270E906F100E6D
:10D240008F6F00011DEC4EF000C0EFF0FBC08EF1BF
:10D25000FAC08DF1F9C08CF1F8C08BF10101926B2D
:10D26000916B270E906F100E8F6F00011DEC4EF02A
:10D27000EFCFF8F0ECCFF9F0ECCFFAF0ECCFFBF019
:10D28000FBC08EF1FAC08DF1F9C08CF1F8C08BF1C2
:10D290000101926B916B030E906FE80E8F6F00018E
:10D2A0001DEC4EF000C0EEF0FBC08EF1FAC08DF127
:10D2B000F9C08CF1F8C08BF10101926B916B030EF8
:10D2C000906FE80E8F6F00011DEC4EF0EFCFF8F07D
:10D2D000ECCFF9F0ECCFFAF0ECCFFBF0FBC08EF125
:10D2E000FAC08DF1F9C08CF1F8C08BF10101926B9D
:10D2F000916B906B640E8F6F00011DEC4EF000C0BF
:10D30000EDF0FBC08EF1FAC08DF1F9C08CF1F8C0E0
:10D310008BF10101926B916B906B640E8F6F00012A
:10D320001DEC4EF0EFCFF8F0ECCFF9F0ECCFFAF0C7
:10D33000ECCFFBF0FBC08EF1FAC08DF1F9C08CF19F
:10D34000F8C08BF10101926B916B906B0A0E8F6F9D
:10D3500000011DEC4EF000C0ECF0FBC08EF1FAC0F5
:10D360008DF1F9C08CF1F8C08BF10101926B916BDA
:10D37000906B0A0E8F6F00011DEC4EF0EFCFEBF0BB
:10D380000400E75313E0E85309E0A50EF16F080E1F
:10D39000F06FA50EF76F100EF66F08D0A50EF76FA1
:10D3A000080EF66FA50EF16F100EF06FEB518B5D4E
:10D3B00004E1E75302E134A814D0680EE525010129
:10D3C000006F9D6FE6C09EF1EBC09FF1F7C0A1F129
:10D3D000F6C0A0F1F5C0A3F1F4C0A2F100015DEC2C
:10D3E0004EF0EC518C5D04E1E75302E134A814D017
:10D3F0004F0EE5250101006F9D6FE6C09EF1ECC068
:10D400009FF1F7C0A1F1F6C0A0F1F5C0A3F1F4C0FF
:10D41000A2F100015DEC4EF0ED518D5D04E1E753AA
:10D4200002E134A814D0320EE5250101006F9D6F92
:10D43000E6C09EF1EDC09FF1F1C0A1F1F0C0A0F1F6
:10D44000F5C0A3F1F4C0A2F100015DEC4EF0EE5185
:10D450008E5D04E1E75302E134A814D0190EE525EE
:10D460000101006F9D6FE6C09EF1EEC09FF1F1C01B
:10D47000A1F1F0C0A0F1F5C0A3F1F4C0A2F1000148
:10D480005DEC4EF0EF518F5D04E1E75302E134A80B
:10D4900010D0E5C09DF1E6C09EF1EFC09FF1F1C054
:10D4A000A1F1F0C0A0F1F5C0A3F1F4C0A2F15DECD0
:10D4B0004EF04F0EE525E96F260EE625EA6F040EC5
:10D4C000E95D0101006F020E0001EA250101016F13
:10D4D000020E0001E95D0101026F090E0001EA255B
:10D4E0000101036F00C18FF101C190F102C191F1FF
:10D4F000926F010E936F946FF3C096F1F2C095F1A5
:10D500000001F1EC45F0EFC08FF0EEC08EF0EDC001
:10D510008DF0ECC08CF0EBC08BF03498EAEF7BF030
:10D52000186AF2BE188EF29E360E0101E66F0001F7
:10D5300066EC3BF018BEF28E186AF2BE188EF29EB0
:10D54000200E0101E66F000176EC3BF018BEF28E72
:10D550000B0E01010125096F070E00250A6F186ADD
:10D56000F2BE188EF29E01C1E2F109C1E3F100C1E1
:10D57000E4F1E56F000186EC3BF018BEF28E186A0C
:10D58000F2BE188EF29E2C0E0101E66F000166ECD1
:10D590003BF018BEF28E0101076B07510708D8A0B7
:10D5A000D7D0086B0851070866E3186AF2BE188ED8
:10D5B000F29EE16B02C1E0F1E36B100EE26F00013D
:10D5C00002EC3BF018BEF28E02C00AF101C009F174
:10D5D000010107510124016E000E0220036E01506B
:10D5E000F2CF0BF1F29E03C0F7FF00016BEC21F0CC
:10D5F00001010BBFF28E0C6F006E0851016E04E04A
:10D60000D8900032012EFCD700A01AD004C109F135
:10D610000A6B186AF2BE188EF29E04C1E6F1000190
:10D6200076EC3BF018BEF28E186AF2BE188EF29EAF
:10D6300003C1E6F176EC3BF018BEF28E19D0010181
:10D6400006C109F10A6B186AF2BE188EF29E06C175
:10D65000E6F1000176EC3BF018BEF28E186AF2BEDD
:10D66000188EF29E05C1E6F176EC3BF018BEF28E04
:10D670000101082B97D7086B0851030867E3186A64
:10D68000F2BE188EF29EE16B02C1E0F1E36B100E68
:10D69000E26F000102EC3BF018BEF28E02C00AF10C
:10D6A00001C009F1080E010107250124016E000ED9
:10D6B0000220036E0150F2CF0CF1F29E03C0F7FF7F
:10D6C00000016BEC21F001010CBFF28E0D6F006EBA
:10D6D0000851016E04E0D8900032012EFCD700A062
:10D6E0001AD004C109F10A6B186AF2BE188EF29EB4
:10D6F00004C1E6F1000176EC3BF018BEF28E186A28
:10D70000F2BE188EF29E03C1E6F176EC3BF018BE35
:10D71000F28E19D0010106C109F10A6B186AF2BE36
:10D72000188EF29E06C1E6F1000176EC3BF018BEC1
:10D73000F28E186AF2BE188EF29E05C1E6F176EC02
:10D740003BF018BEF28E0101082B96D7072B25D788
:10D75000186AF2BE188EF29E360EE66F000166EC75
:10D760003BF018BEF28E186AF2BE188EF29E0101CE
:10D77000E66B000176EC3BF018BEF28E000CE96B14
:10D78000EA6BEB6BEC6BED6BD30EEF6FC00EEE6FD5
:10D79000FF0EF16FF06FF36BF26BF56FE00EF46F4D
:10D7A0000400E75309E04DC0FDF04CC0FCF04BC055
:10D7B000FBF04AC0FAF008D045C0FDF044C0FCF0D0
:10D7C00043C0FBF042C0FAF0FDC04DF0FCC04CF08D
:10D7D000FBC04BF0FAC04AF0FDC08EF1FCC08DF1E9
:10D7E000FBC08CF1FAC08BF10101926B916B030EBF
:10D7F000906FE80E8F6F00011DEC4EF003C0F9F042
:10D8000002C0F8F001C0F7F000C0F6F0F9C08EF1E8
:10D81000F8C08DF1F7C08CF1F6C08BF10101926B6D
:10D82000916B270E906F100E8F6F00011DEC4EF064
:10D8300000C0EDF0F9C08EF1F8C08DF1F7C08CF1A9
:10D84000F6C08BF10101926B916B270E906F100E59
:10D850008F6F00011DEC4EF0EFCFF6F0ECCFF7F03C
:10D86000ECCFF8F0ECCFF9F0F9C08EF1F8C08DF103
:10D87000F7C08CF1F6C08BF10101926B916B030E36
:10D88000906FE80E8F6F00011DEC4EF000C0ECF0C1
:10D89000F9C08EF1F8C08DF1F7C08CF1F6C08BF1B4
:10D8A0000101926B916B030E906FE80E8F6F000178
:10D8B0001DEC4EF0EFCFF6F0ECCFF7F0ECCFF8F038
:10D8C000ECCFF9F0F9C08EF1F8C08DF1F7C08CF112
:10D8D000F6C08BF10101926B916B906B640E8F6FB0
:10D8E00000011DEC4EF000C0EBF0F9C08EF1F8C065
:10D8F0008DF1F7C08CF1F6C08BF10101926B916B49
:10D90000906B640E8F6F00011DEC4EF0EFCFF6F0C0
:10D91000ECCFF7F0ECCFF8F0ECCFF9F0F9C08EF1E6
:10D92000F8C08DF1F7C08CF1F6C08BF10101926B5C
:10D93000916B906B0A0E8F6F00011DEC4EF000C0D2
:10D94000EAF0F9C08EF1F8C08DF1F7C08CF1F6C0A5
:10D950008BF10101926B916B906B0A0E8F6F00013E
:10D960001DEC4EF0EFCFE9F00400E75313E0E8536D
:10D9700009E0A50EEF6F080EEE6FA50EF56F100E05
:10D98000F46F08D0A50EF56F080EF46FA50EEF6FBB
:10D99000100EEE6FE9518B5D04E1E75302E134A80C
:10D9A00015D0320EE525FE6F100EE925FF6FFEC083
:10D9B00000F1E6C001F1E8CF02F1F5C004F1F4C0D6
:10D9C00003F1F3C006F1F2C005F1AADDEA518C5D66
:10D9D00004E1E75302E134A815D0280EE525FE6FD7
:10D9E000100EEA25FF6FFEC000F1E6C001F1E8CF9E
:10D9F00002F1F5C004F1F4C003F1F3C006F1F2C086
:10DA000005F18EDDEB518D5D04E1E75302E134A8B1
:10DA100015D0140EE525FE6F100EEB25FF6FFEC02E
:10DA200000F1E6C001F1E8CF02F1EFC004F1EEC071
:10DA300003F1F3C006F1F2C005F172DDEC518E5D29
:10DA400004E1E75302E134A815D00A0EE525FE6F84
:10DA5000100EEC25FF6FFEC000F1E6C001F1E8CF2B
:10DA600002F1EFC004F1EEC003F1F3C006F1F2C021
:10DA700005F156DDED518F5D04E1E75302E134A875
:10DA800012D0100EED25FE6FE5C000F1E6C001F1E9
:10DA9000E8CF02F1EFC004F1EEC003F1F3C006F1EC
:10DAA000F2C005F13DDD140EE5250A0FFF6FE8CF4A
:10DAB00000F1E6C001F10C0E0101026FFF0E046FD0
:10DAC000036FF3C006F1F2C005F1000129DDEDC0DE
:10DAD0008FF0ECC08EF0EBC08DF0EAC08CF0E9C0A6
:10DAE0008BF034980400000CE96BEA6BEB6BEC6B89
:10DAF000ED6B070EEF6FE00EEE6FFF0EF16FF06F44
:10DB0000F36BF26B070EF56FFF0EF46F0400E75333
:10DB100009E051C0FDF050C0FCF04FC0FBF04EC01A
:10DB2000FAF008D049C0FDF048C0FCF047C0FBF057
:10DB300046C0FAF0FDC051F0FCC050F0FBC04FF001
:10DB4000FAC04EF0FDC08EF1FCC08DF1FBC08CF12F
:10DB5000FAC08BF10101926B916B906B640E8F6F29
:10DB600000011DEC4EF003C0F9F002C0F8F001C056
:10DB7000F7F000C0F6F0F9C08EF1F8C08DF1F7C0F3
:10DB80008CF1F6C08BF10101926B916B270E906FB7
:10DB9000100E8F6F00011DEC4EF000C0EDF0F9C0CB
:10DBA0008EF1F8C08DF1F7C08CF1F6C08BF1010158
:10DBB000926B916B270E906F100E8F6F00011DEC12
:10DBC0004EF0EFCFF6F0ECCFF7F0ECCFF8F0ECCF73
:10DBD000F9F0F9C08EF1F8C08DF1F7C08CF1F6C004
:10DBE0008BF10101926B916B030E906FE80E8F6FBA
:10DBF00000011DEC4EF000C0ECF0F9C08EF1F8C051
:10DC00008DF1F7C08CF1F6C08BF10101926B916B35
:10DC1000030E906FE80E8F6F00011DEC4EF0EFCFFA
:10DC2000F6F0ECCFF7F0ECCFF8F0ECCFF9F0F9C06C
:10DC30008EF1F8C08DF1F7C08CF1F6C08BF10101C7
:10DC4000926B916B906B640E8F6F00011DEC4EF028
:10DC500000C0EBF0F9C08EF1F8C08DF1F7C08CF187
:10DC6000F6C08BF10101926B916B906B640E8F6F1C
:10DC700000011DEC4EF0EFCFF6F0ECCFF7F0ECCF5B
:10DC8000F8F0ECCFF9F0F9C08EF1F8C08DF1F7C0E3
:10DC90008CF1F6C08BF10101926B916B906B0A0EC7
:10DCA0008F6F00011DEC4EF000C0EAF0F9C08EF15C
:10DCB000F8C08DF1F7C08CF1F6C08BF10101926BC9
:10DCC000916B906B0A0E8F6F00011DEC4EF0EFCF41
:10DCD000E9F00400E75313E0E85309E0A50EEF6F05
:10DCE000080EEE6FA50EF56F100EF46F08D0A50E9E
:10DCF000F56F080EF46FA50EEF6F100EEE6FE95181
:10DD0000905D04E1E75302E134AA16D0320EE52516
:10DD1000FE6F100EE925FF6FFEC000F1E6C001F1B5
:10DD2000E8CF02F1F5C004F1F4C003F1F3C006F14D
:10DD3000F2C005F190EC6AF0EA51915D04E1E7531D
:10DD400002E134AA16D0280EE525FE6F100EEA2552
:10DD5000FF6FFEC000F1E6C001F1E8CF02F1F5C0AF
:10DD600004F1F4C003F1F3C006F1F2C005F190EC48
:10DD70006AF0EB51925D04E1E75302E134AA16D058
:10DD80001E0EE525FE6F100EEB25FF6FFEC000F1A5
:10DD9000E6C001F1E8CF02F1F5C004F1F4C003F1EF
:10DDA000F3C006F1F2C005F190EC6AF0EC51935D1E
:10DDB00004E1E75302E134AA16D00A0EE525FE6F0E
:10DDC000100EEC25FF6FFEC000F1E6C001F1E8CFB8
:10DDD00002F1EFC004F1EEC003F1F3C006F1F2C0AE
:10DDE00005F190EC6AF0ED51945D04E1E75302E136
:10DDF00034AA13D0100EED25FE6FE5C000F1E6C089
:10DE000001F1E8CF02F1EFC004F1EEC003F1F3C07D
:10DE100006F1F2C005F190EC6AF00A0EE5250A0F52
:10DE2000FF6FE8CF00F1E6C001F10C0E0101026FB7
:10DE3000FF0E046F036FF3C006F1F2C005F100019D
:10DE400090EC6AF0E9C090F0EAC091F0EBC092F07B
:10DE5000ECC093F0ECC094F0349A0400000CEE0E89
:10DE6000F76F480EF86FBA0EF96FDA0EFA6F5C0EA4
:10DE7000FB6FD60EFC6FF60EFD6F4A0EFE6FFE0EA8
:10DE8000FF6FDE0E0101006F0001F1510B0866E12A
:10DE9000080EEF250101016F090E0001F0250101B7
:10DEA000026F186AF2BE188EF29EEFC0E2F101C155
:10DEB000E3F1F0C0E4F1E56F000186EC3BF018BE41
:10DEC000F28E186AF2BE188EF29E2C0E0101E66FD9
:10DED000000166EC3BF018BEF28EF26BF25159086D
:10DEE0003CE3D890F235036AF2CF01F1F29EAFEC39
:10DEF00039F00900F5CF03F0010101BFF28E026F86
:10DF000003C003F103C004F1056B186AF2BE188E5A
:10DF1000F29E03C0E6F1000176EC3BF018BEF28EF3
:10DF2000D890F235036AF2CF01F1F29EAFEC39F0EE
:10DF30000900F5CF03F0010101BFF28E026F03C0AB
:10DF400003F1186AF2BE188EF29EE66F000176ECBD
:10DF50003BF018BEF28EF22BC1D7F8D2F36BF3511F
:10DF60003A08D8A0F3D2F46BF4511D08D8A0ECD233
:10DF7000F451060864E2F4511A0861E3F351080809
:10DF80005EE3186AF2BE188EF29E0101E16BF3C0E7
:10DF9000E0F1E36B280EE26F000102EC3BF018BEEB
:10DFA000F28E02C002F101C001F1070EF45D036AB6
:10DFB000026ED89002360336025001010124016E30
:10DFC000025103220150F2CF04F1F29E03C0F7FF89
:10DFD0000001F6EC32F00900F5CF03F0010104BFB7
:10DFE000F28E0001F56F03C0F6F0F55303E1F65130
:10DFF000F80825E0036AF151F70FE96E000E0320DF
:10E00000EA6EEF50020B02E1F66BF56BF451EF256F
:10E010000101016F0001F351F0250101026F186A3F
:10E02000F2BE188EF29E01C1DEF1DF6FF6C0E1F1A3
:10E03000F5C0E0F100019DEC3BF018BEF28EF4510A
:10E04000020869E2F451170866E3F351310863E20C
:10E05000F3513A0860E3320EF35D0101026F186A72
:10E06000F2BE188EF29EE16BE06FE36B2A0EE26F58
:10E07000000102EC3BF018BEF28E02C004F101C0B8
:10E0800003F1030EF45D036A026ED8900236033684
:10E09000025001010124016E045103220150F2CF0C
:10E0A00006F1F29E03C0F7FF0001E6EC38F009002C
:10E0B000F5CF03F0010106BFF28E0001F56F03C03A
:10E0C000F6F0F55303E1F651F80825E0036AF15143
:10E0D000F70FE96E000E0320EA6EEF50800B02E1AD
:10E0E000F66BF56BF451EF250101016F0001F3515F
:10E0F000F0250101026F186AF2BE188EF29E01C16E
:10E10000DEF1DF6FF6C0E1F1F5C0E0F100019DEC5A
:10E110003BF018BEF28EF451130869E2F4511D0869
:10E1200066E3F351020863E2F3511B0860E3030E58
:10E13000F35D0101026F186AF2BE188EF29EE16B68
:10E14000E06FE36B140EE26F000102EC3BF018BECF
:10E15000F28E02C004F101C003F1140EF45D036AF3
:10E16000026ED89002360336025001010124016E7E
:10E17000045103220150F2CF06F1F29E03C0F7FFD3
:10E180000001C6EC34F00900F5CF03F0010106BF31
:10E19000F28E0001F56F03C0F6F0F55303E1F6517E
:10E1A000F80825E0036AF151F70FE96E000E03202D
:10E1B000EA6EEF50080B02E1F66BF56BF451EF25B8
:10E1C0000101016F0001F351F0250101026F186A8E
:10E1D000F2BE188EF29E01C1DEF1DF6FF6C0E1F1F2
:10E1E000F5C0E0F100019DEC3BF018BEF28EF45159
:10E1F000040869E2F451190866E3F351170863E271
:10E20000F351200860E3180EF35D0101026F186AF4
:10E21000F2BE188EF29EE16BE06FE36B280EE26FA8
:10E22000000102EC3BF018BEF28E02C004F101C006
:10E2300003F1050EF45D036A026ED89002360336D0
:10E24000025001010124016E045103220150F2CF5A
:10E2500006F1F29E03C0F7FF0001CCEC35F0090097
:10E26000F5CF03F0010106BFF28E0001F56F03C088
:10E27000F6F0F55303E1F651F80825E0036AF15191
:10E28000F70FE96E000E0320EA6EEF50100B02E16B
:10E29000F66BF56BF451EF250101016F0001F351AD
:10E2A000F0250101026F186AF2BE188EF29E01C1BC
:10E2B000DEF1DF6FF6C0E1F1F5C0E0F100019DECA9
:10E2C0003BF018BEF28EF451090864E3F3511C08C8
:10E2D00061E2F35137085EE31D0EF35D0101026F49
:10E2E000186AF2BE188EF29EE16BE06FE36B140EBB
:10E2F000E26F000102EC3BF018BEF28E02C004F1A6
:10E3000001C003F1D890F435026E036A033602505F
:10E3100001010124016E045103220150F2CF05F1E5
:10E32000F29E03C0F7FF00018CEC36F00900F5CF38
:10E3300003F0010105BFF28E0001F56F03C0F6F096
:10E34000F55303E1F651F80825E0036AF151F70FA0
:10E35000E96E000E0320EA6EEF50200B02E1F66B2F
:10E36000F56BF451EF250101016F0001F351F02528
:10E370000101026F186AF2BE188EF29E01C1DEF131
:10E38000DF6FF6C0E1F1F5C0E0F100019DEC3BF07C
:10E3900018BEF28EF451020869E2F4510C0866E3EB
:10E3A000F351010863E2F3511B0860E3020EF35DD1
:10E3B0000101026F186AF2BE188EF29EE16BE06FE7
:10E3C000E36B140EE26F000102EC3BF018BEF28E1C
:10E3D00002C004F101C003F1030EF45D036A026E92
:10E3E000D89002360336025001010124016E045117
:10E3F00003220150F2CF06F1F29E03C0F7FF0001A5
:10E40000B6EC33F00900F5CF03F0010106BFF28E40
:10E410000001F56F03C0F6F0F55303E1F651F8087B
:10E4200025E0036AF151F70FE96E000E0320EA6E52
:10E43000EF50040B02E1F66BF56BF451EF2501018F
:10E44000016F0001F351F0250101026F186AF2BE5D
:10E45000188EF29E01C1DEF1DF6FF6C0E1F1F5C06A
:10E46000E0F100019DEC3BF018BEF28EF451110872
:10E4700069E2F4511C0866E3F3511C0863E2F351AE
:10E48000380860E31D0EF35D0101026F186AF2BEE9
:10E49000188EF29EE16BE06FE36B160EE26F0001E7
:10E4A00002EC3BF018BEF28E02C004F101C003F191
:10E4B000120EF45D036A026ED890023603360250E3
:10E4C00001010124016E045103220150F2CF06F133
:10E4D000F29E03C0F7FF0001A6EC37F00900F5CF6C
:10E4E00003F0010106BFF28E0001F56F03C0F6F0E4
:10E4F000F55303E1F651F80825E0036AF151F70FEF
:10E50000E96E000E0320EA6EEF50400B02E1F66B5D
:10E51000F56BF451EF250101016F0001F351F02576
:10E520000101026F186AF2BE188EF29E01C1DEF17F
:10E53000DF6FF6C0E1F1F5C0E0F100019DEC3BF0CA
:10E5400018BEF28EF42B10D5F32B09D5000CE56B19
:10E55000E66BE76BE86B020E01018E6F00013EEC8B
:10E5600059F001C0E9F0010E01018E6F00013EEC8F
:10E5700059F001C0EAF001018E6B00013EEC59F048
:10E5800001C0EBF0E939006E0F0E00160050030BCE
:10E59000E86FE9510F0BE76FEA39006E0F0E0016B6
:10E5A0000050070BE66FEA510F0BE56F0400E551D1
:10E5B000955D02E134AC09D0640EE325EC6FEF6F9A
:10E5C000E4C0F0F0E5C0F1F04ADCE651965D02E10E
:10E5D00034AC09D0460EE325EC6FEF6FE4C0F0F0E9
:10E5E000E6C0F1F03CDCE751975D02E134AC09D0C4
:10E5F0001E0EE325EC6FEF6FE4C0F0F0E7C0F1F022
:10E600002EDCE851985D02E134AC07D0E3C0EFF0B6
:10E61000E4C0F0F0E8C0F1F022DC0400EBA11BD074
:10E620001E0EE3251F0FED6F190EE425EE6FEDC0F2
:10E63000EFF0F06F0B0EF16F12DC1E0EE3251D0FD5
:10E64000ED6F280EE425EE6FEDC0EFF0F06F0B0ECE
:10E65000F16F05DC1FD01E0EE3251D0FED6F190EA7
:10E66000E425EE6F1E0EE325270FF06F330EE42531
:10E67000F16FEDC08FF1EEC090F1F0C091F1E8CFF5
:10E6800092F1010E0101936F946F966B956B0001EF
:10E69000F1EC45F0E5C095F0E6C096F0E7C097F0E4
:10E6A000E8C098F0349CEAEF7BF0E56BE66BE76B33
:10E6B000E86B79C0EDF078C0ECF077C0EFF076C091
:10E6C000EEF0020E01018E6F00013EEC59F001C028
:10E6D000E9F0010E01018E6F00013EEC59F001C01E
:10E6E000EAF001018E6B00013EEC59F001C0EBF045
:10E6F000E939006E0F0E00160050030BE86FE95168
:10E700000F0BE76FEA39006E0F0E00160050070B73
:10E71000E66FEA510F0BE56F0400E551955D02E1EC
:10E7200034AC13D0620EE325F06FE8CF9DF1E4C066
:10E730009EF1E5C09FF1EDC0A1F1ECC0A0F1EFC0EA
:10E74000A3F1EEC0A2F15DEC4EF0E651965D02E160
:10E7500034AC13D0460EE325F06FE8CF9DF1E4C052
:10E760009EF1E6C09FF1EDC0A1F1ECC0A0F1EFC0B9
:10E77000A3F1EEC0A2F15DEC4EF0E751975D02E12E
:10E7800034AC13D01E0EE325F06FE8CF9DF1E4C04A
:10E790009EF1E7C09FF1EDC0A1F1ECC0A0F1EFC088
:10E7A000A3F1EEC0A2F15DEC4EF0E851985D02E1FC
:10E7B00034AC13D0020EE325F06FE8CF9DF1E4C036
:10E7C0009EF1E8C09FF1EDC0A1F1ECC0A0F1EFC057
:10E7D000A3F1EEC0A2F15DEC4EF00400EBA141D03C
:10E7E0001E0EE3251D0FF16F140EE425F26F1E0EB1
:10E7F000E325210FF46F180EE425F56FF1C08FF1BA
:10E80000F2C090F1F4C091F1E8CF92F1010E010154
:10E81000936F946FFF0E966F956F0001F1EC45F0CA
:10E820001E0EE3251D0FF16F1E0EE425F26F1E0E66
:10E83000E325210FF46F220EE425F56FF1C08FF16F
:10E84000F2C090F1F4C091F1E8CF92F1010E010114
:10E85000936F946FFF0E966F956F0001F1EC45F08A
:10E860003ED01E0EE3251D0FF16F140EE425F26F4E
:10E870001E0EE325210FF46F180EE425F56FF1C08D
:10E880008FF1F2C090F1F4C091F1E8CF92F1010E56
:10E890000101936F946F966B956B0001F1EC45F05D
:10E8A0001E0EE3251D0FF16F1E0EE425F26F1E0EE6
:10E8B000E325210FF46F220EE425F56FF1C08FF1EF
:10E8C000F2C090F1F4C091F1E8CF92F1010E010194
:10E8D000936F946F966B956B0001F1EC45F0E5C07A
:10E8E00095F0E6C096F0E7C097F0E8C098F0349C49
:10E8F000EAEF7BF04A0EF16F610EF26F6E0EF36F6E
:10E90000F46B050E01018E6F00013EEC59F00150D1
:10E910001F0BF06FF02D10D0B66BF10EB56FF56BCD
:10E92000F55116EC3AF0000907E0F52B0101A56F4F
:10E930000001AFEC56F0F4D7F051020810E1B66BCD
:10E94000F10EB56FF56BF55125EC3AF0000907E0D3
:10E95000F52B0101A56F0001AFEC56F0F4D7F05193
:10E96000030810E1B66BF10EB56FF56BF55134ECA1
:10E970003AF0000907E0F52B0101A56F0001AFECAB
:10E9800056F0F4D7F051040810E1B66BF10EB56FF4
:10E99000F56BF55143EC3AF0000907E0F52B010166
:10E9A000A56F0001AFEC56F0F4D7F051050810E167
:10E9B000B66BF10EB56FF56BF55152EC3AF00009FC
:10E9C00007E0F52B0101A56F0001AFEC56F0F4D77D
:10E9D000F051060810E1B66BF10EB56FF56BF5510D
:10E9E00061EC3AF0000907E0F52B0101A56F000189
:10E9F000AFEC56F0F4D7F051070810E1B66BF10E0A
:10EA0000B56FF56BF55170EC3AF0000907E0F52BA6
:10EA10000101A56F0001AFEC56F0F4D7F0510808E2
:10EA200010E1B66BF10EB56FF56BF5517FEC3AF076
:10EA3000000907E0F52B0101A56F0001AFEC56F0CE
:10EA4000F4D7F051090810E1B66BF10EB56FF56B14
:10EA5000F5518EEC3AF0000907E0F52B0101A56FA6
:10EA60000001AFEC56F0F4D7F051100810E1B66B8E
:10EA7000F10EB56FF56BF5519DEC3AF0000907E02A
:10EA8000F52B0101A56F0001AFEC56F0F4D7F05162
:10EA9000110810E1B66BF10EB56FF56BF551ACECEA
:10EAA0003AF0000907E0F52B0101A56F0001AFEC7A
:10EAB00056F0F4D7F051120810E1B66BF10EB56FB5
:10EAC000F56BF551BBEC3AF0000907E0F52B0101BD
:10EAD000A56F0001AFEC56F0F4D7040E01018E6F64
:10EAE00000013EEC59F001C0F5F0EFC0B6F0EEC009
:10EAF000B5F001C08FF1570E0101906F000177EC66
:10EB000059F0200E0101A56F0001AFEC56F0EA6A42
:10EB1000F10EE96E000EEF1010E0EACFF7F0E9CF4A
:10EB2000F6F0EFCFA5F1AFEC56F0F7C0EAFFF6C074
:10EB3000E9FFE92AD8B4EA2AEDD7070EEE25E96EF7
:10EB4000000EEF21EA6EEF6AEEC001F0B9EF75F04A
:10EB5000040E01018E6F00013EEC59F001C0EDF092
:10EB6000ED51A85D02E134AE19D0EF6BE50EEE6F0A
:10EB7000C1D6E3C0EFF0E4C0F0F0F26BE50EF16F48
:10EB8000010EF36F7FC0F5F07EC0F4F07BC0F7F0AC
:10EB90007AC0F6F0F4EC61F0EDC0A8F0349EF0EF2E
:10EBA0007BF0F86AD09E0D8EEA6AE96AC150C00B0C
:10EBB0000F09C16E070EB46E196A1A6A1B6A1C6AC5
:10EBC0001D6A1E6A1F6A206A216A226A236A246AF1
:10EBD000256A266A276A286A296A2A6A2B6A2C6AA1
:10EBE0002D6A2E6A2F6A306A316A326A336A34902B
:10EBF000356A366A376A386A396A3A6A3B6A3C6A01
:10EC00003D6A3E6A3F6A406A416A426A436A446AB0
:10EC1000456A466A476A486A496A4A6A4B6A4C6A60
:10EC20004D6A4E6A4F6A506A516A526A536A546A10
:10EC3000556A566A576A586A596A5A6A5B6A5C6AC0
:10EC40005D6A5E6A5F6A606A616A626A636A646A70
:10EC5000656A666A676A686A696A6A6A6B6A349230
:10EC6000349434963498349A349C349E6C6A6D6A29
:10EC70006E6A6F6A706A716A726A736A746A756AB8
:10EC8000766A776A786A796A7A6A7B6A7C6A7D6A68
:10EC90007E6A7F6A806B816B826B836B846B856B12
:10ECA000866B876B886B896B8A6B090E8B6F8C6F99
:10ECB0008D6F8E6F8F6F906F916F926F936F946F58
:10ECC000956F966F976F986F4D0E996F690E9A6F4B
:10ECD000730E9B6F650E9C6F200E9D6F610E9E6F75
:10ECE000200E9F6F6A0EA06F6F0EA16F750EA26F40
:10ECF000720EA36F2E0EA46FA56FA66FA76B630E87
:10ED0000A86FA96BAA6BB56BB66B540EBA6F720E77
:10ED1000BB6F690EBC6F700EBD6F4D0EBE6F650E82
:10ED2000BF6F720EC06F6F0EC16FC26B560EC36F96
:10ED3000650EC46F720EC56F200EC66F380EC76F9A
:10ED40002E0EC86F320EC96F330ECA6FCB6B560EC4
:10ED5000CC6F610ECD6F6C0ECE6F650ECF6F750EE2
:10ED6000D06F720ED16F730ED26F200ED36F440E20
:10ED7000D46F650ED56F660ED66F610ED76F750EA8
:10ED8000D86F740ED96FDA6B186AF2BE188EF29EC5
:10ED9000C80E0101C36F0001C3EC3CF018BEF28E37
:10EDA000C69A949A94889496000EC66EC76ED180C7
:10EDB000F10ED56E870ECD6E000ECA6E000ECB6EB4
:10EDC000B150480BB16E070EB46E92501A0E006E21
:10EDD000002EFED70000B450A19CB56A180ED26E6A
:10EDE000D76AD66ACF6ACE6A84EF3DF0040094EC0D
:10EDF0003DF001C0B7F0B72D0DD1186AF2BE188EE4
:10EE0000F29E060E0101C36FC76BC66BC56BC46B68
:10EE10000001D2EC3AF018BEF28E186AF2BE188EDB
:10EE2000F29E0A0E0101C36FC76BC66BC56BC46B44
:10EE30000001D2EC3AF018BEF28E120E01019C6F66
:10EE40009E6B530E9D6F0001EFEC3DF0AA6A240EFD
:10EE5000A96EA86AA69CA69EA684F2CF00F0F29E98
:10EE60000F01550EA76EAA0EA76EA682A6B2FED7F8
:10EE7000A6940050F212AA6A250EA96EA86AA69C52
:10EE8000A69EA684F2CF00F0F29E550EA76EAA0EA3
:10EE9000A76EA682A6B2FED7A6940050F212AA6A66
:10EEA000170EA96E410EA86EA69CA69EA684F2CF50
:10EEB00000F0F29E550EA76EAA0EA76EA682A6B20D
:10EEC000FED7A6940050F212F2CFE3F0F29EAA6AA7
:10EED000170EA96EA69CA69EA680A8500001E3BFAF
:10EEE000F28E656E65C0E3F093EC3EF0666A676A89
:10EEF000686A010E696E6A6E060E6B6E040001018F
:10EF0000896B68C08AF1000164EC3DF0010E0101DB
:10EF1000896F67C08AF1000164EC3DF0020E0101C7
:10EF2000896F66C08AF1000164EC3DF0040E0101B6
:10EF3000896F69C08AF1000164EC3DF0050E0101A2
:10EF4000896F6AC08AF1000164EC3DF0060E010190
:10EF5000896F6BC08AF1000164EC3DF0040E010181
:10EF6000526F600E516F000138EC3EF0186AF2BE2D
:10EF7000188EF29E050E0101C36FC46FC66BCC0ED6
:10EF8000C56FFF0EC86FE00EC76F040ECA6F600E2C
:10EF9000C96F0001B7EC3BF018BEF28E186AF2BEE2
:10EFA000188EF29E050E0101C36F700EC46FC66B02
:10EFB000CC0EC56FFF0EC86FE00EC76F040ECA6F90
:10EFC000600EC96F0001B7EC3BF018BEF28E210E47
:10EFD000E36FE46F020EE56FE76BFA0EE66F15EC78
:10EFE0003FF0140EB86FB8530FE0186AF2BE188ED7
:10EFF000F29E320E0101C36F0001C3EC3CF018BE5B
:10F00000F28E0400B807EFD70101526B516B00017B
:10F0100038EC3EF0F2CFE3F0F29EAA6A170EA96E2A
:10F02000A69CA69EA680A850E3BFF28E656E65C022
:10F03000E3F093EC3EF0040E0101526F600E516F4D
:10F04000000138EC3EF0186AF2BE188EF29E1D0EDA
:10F050000101C36F050EC46FC66BBA0EC56FFF0EFC
:10F06000C86FE00EC76F040ECA6F600EC96F000153
:10F07000B7EC3BF018BEF28E186AF2BE188EF29E04
:10F080001D0E0101C36F700EC46FC66BC30EC56F3A
:10F09000FF0EC86FE00EC76F040ECA6F600EC96F17
:10F0A0000001B7EC3BF018BEF28E200E01018F6F0D
:10F0B000906F610E916F926F010E936F946B966BD0
:10F0C000956B0001F1EC45F0210EE36FE46F020E49
:10F0D000E56FE76BFA0EE66F15EC3FF01C6A1B6AF2
:10F0E0001E6A1D6A1A6A196A3490226A216A246AA1
:10F0F000236AB86BB85104080DE3D890B835036A99
:10F10000270FE96E000E0320EA6EEC6AED52EF6AFB
:10F11000B82BF0D7336A0F0EB86FB8530FE0186AE8
:10F12000F2BE188EF29E190E0101C36F0001C3ECEE
:10F130003CF018BEF28E0400B807EFD73494349236
:10F14000646A8CEF46F0015202E10400FAD7040031
:10F15000120EE36FA1EF46F002C063F001C062F04F
:10F16000060EE36FC3EC46F003C045F002C044F066
:10F1700001C043F000C042F00A0EE36FC3EC46F05A
:10F1800003C049F002C048F001C047F000C046F09B
:10F1900045C04DF044C04CF043C04BF042C04AF073
:10F1A00049C051F048C050F047C04FF046C04EF043
:10F1B00049C059F048C058F047C057F046C056F013
:10F1C000F2CFE3F0F29EAA6A240EA96EA69CA69E38
:10F1D000A680A850E3BFF28E6C6EF2CFE3F0F29EF1
:10F1E000AA6A250EA96EA69CA69EA680A850E3BF7B
:10F1F000F28E6D6E6CC0E3F0E8EC46F08A6B3488FA
:10F20000348A348C348EF28AA084C00EF212040048
:10F21000348604007BEC47F003C055F002C054F084
:10F2200001C053F000C052F034B20AD055C08DF185
:10F2300054C08CF153C08BF152C08AF1DCEC47F022
:10F2400034B40AD055C08EF154C08DF153C08CF146
:10F2500052C08BF1FCEC47F034A0A4D0D8903334EA
:10F26000036A270F016E000E032201C0E3F003C002
:10F27000E4F0CEEF4CF0E4C0EAFFE3C0E9FFEC6A53
:10F28000ED5201C0EFFF332A33500508D8B4336A7A
:10F29000326A316AB86BB851040811E3D890B835B6
:10F2A000036A270FE96E000E0320EA6EECCF03F02D
:10F2B000ED52EF50312603503222B82BECD732C03A
:10F2C0009DF131C09CF101019F6B050E9E6F000105
:10F2D000FAEC4DF002C00EF101C00DF10001BEECE0
:10F2E00049F003C0DEF002C0DDF001C0DCF000C078
:10F2F000DBF0DEC0F8F0DDC0F7F0DCC0F6F0DBC01C
:10F30000F5F0C3EC4CF003C0E2F002C0E1F001C044
:10F31000E0F000C0DFF0D882DEC010F1DDC00FF1F8
:10F32000DCC00EF1DBC00DF1E2C014F1E1C013F15D
:10F33000E0C012F1DFC011F1D9EC49F000C0E3F0F8
:10F3400001C0E4F002C0E5F003C0E6F003C00CF138
:10F3500002C00BF101C00AF100C009F10101106BFC
:10F360000F6B0E6B7E0E0D6F000163EC49F00DE329
:10F37000E2C00CF1E1C00BF1E0C00AF1DFC009F11D
:10F38000A0EC49F001C08AF00DD0E2C00CF1E1C060
:10F390000BF1E0C00AF1DFC009F1A0EC49F0010E69
:10F3A00001248A6F000EB9B1010E010A016EE8B0A6
:10F3B00002D0B99101D0B981040094EC3DF001C0B4
:10F3C000B7F0B75102081EE1010E6D266D5002081C
:10F3D000D8A06D6AAA6A250EA96E6DC0A8FFA69C6A
:10F3E000A69EA684F2CF00F0F29E0F01550EA76EE6
:10F3F000AA0EA76EA682A6B2FED7A6940050F2125D
:10F4000034860001B75103081EE1FF0E6C1AAA6A88
:10F41000240EA96E6CC0A8FFA69CA69EA684F2CF5F
:10F4200000F0F29E0F01550EA76EAA0EA76EA682DF
:10F43000A6B2FED7A6940050F2126CC0E3F0000111
:10F44000E8EC46F034860400B751050819E1010ED6
:10F450000101996F230E9A6F830E9B6F820E9C6F32
:10F460009E6B9D6B000110EC40F085EF5FF0186A19
:10F47000F2BE188EF29ED7EC3CF018BEF28E3486A7
:10F4800034A6BCD0186AF2BE188EF29ED7EC3CF0BF
:10F4900018BEF28E65C0E3F093EC3EF03488348AF7
:10F4A000348C348E6C5210E0010E0101996F230EE2
:10F4B0009A6F830E9B6F820E9C6FFF0E9E6F9D6FE7
:10F4C000000110EC40F006D00101526B516B0001BD
:10F4D00038EC3EF0010E0101996F220E9A6F830EF7
:10F4E0009B6F220E9C6F7BC09EF17AC09DF1000144
:10F4F00073EC44F0540E0101996F010E9A6F540E93
:10F500009B6F210E9C6F85C09EF184C09DF1000110
:10F5100073EC44F0550E0101996F010E9A6F820E43
:10F520009B6F010E9C6F85C09EF184C09DF1000110
:10F5300073EC44F0550E01018F6F020E906F830E35
:10F54000916F210E926F010E936F946F7BC096F1B5
:10F550007AC095F10001F1EC45F0540E0101996F6C
:10F56000130E9A6F830E9B6F130E9C6F85C09EF1D6
:10F5700084C09DF1000173EC44F0540E0101996FB9
:10F58000140E9A6F830E9B6F140E9C6F85C09EF1B4
:10F5900084C09DF1000173EC44F0540E0101996F99
:10F5A000150E9A6F830E9B6F150E9C6F9E6B9D6B55
:10F5B000000173EC44F0540E0101996F160E9A6F1E
:10F5C000830E9B6F160E9C6F85C09EF184C09DF1CB
:10F5D000000173EC44F0540E0101996F170E9A6FFD
:10F5E000830E9B6F170E9C6F85C09EF184C09DF1AA
:10F5F000000173EC44F03496A194A0848AC0E3F037
:10F6000006EF63F0B75107080BE1000E34B4010EAA
:10F61000010A016EE8B002D0349401D03484348AF7
:10F62000B7510C080BE1000E34B2010E010A016E55
:10F63000E8B002D0349201D034823488B7510A083D
:10F640001CE1496A486A476A466A516A506A4F6AC9
:10F650004E6A186AF2BE188EF29E0A0E0101C36F3E
:10F6600049C0C7F148C0C6F147C0C5F146C0C4F1A2
:10F670000001D2EC3AF018BEF28EB7533CE134A24E
:10F680001CD0456A446A436A426A4D6A4C6A4B6AB6
:10F690004A6A186AF2BE188EF29E060E0101C36F06
:10F6A00045C0C7F144C0C6F143C0C5F142C0C4F172
:10F6B0000001D2EC3AF018BEF28E34A41CD0496A94
:10F6C000486A476A466A516A506A4F6A4E6A186ABF
:10F6D000F2BE188EF29E0A0E0101C36F49C0C7F137
:10F6E00048C0C6F147C0C5F146C0C4F10001D2EC24
:10F6F0003AF018BEF28E04006D5005E0010A26E0D3
:10F70000030A46E067D0010EE36FE46F53EF66F043
:10F71000000E34B4010EE76F000EB9B1010EE86FB0
:10F72000020EE56F530EE66F01EF67F0000E34B284
:10F73000010EE36F000EB9B1010EE86F020EE56F26
:10F74000230EE66FE3C0E7F0C8EF68F0000E34B2B6
:10F75000010EE76F000EB9B1010EE86F0D0EE56FF7
:10F76000040EE66FBFEC6BF0000E34B4010EE76FD1
:10F77000000EB9B1010EE86F0D0EE56F130EE66FC6
:10F7800074EC6DF0010EE36F360EE46FA7EF72F0CC
:10F79000000E34B2010EE76F000EB9B1010EE86F32
:10F7A0000D0EE56F040EE66FBFEC6BF0000E34B487
:10F7B000010EE76F000EB9B1010EE86F0D0EE56F97
:10F7C000130EE66F74EC6DF0010EE36F360EE46F0E
:10F7D00055EF73F05A0EE36F190EE46FA8EF75F052
:04F7E00018D5030035
:020000040030CA
:0E00000000C61F170087C5000FC00FE00F409D
:00000001FF
